:100000000C94650A0C94860A0C94860A0C94DD0FF5
:100010000C9417100C94860A0C94860A0C94860A89
:100020000C94860A0C94860A0C94860A0C94860A10
:100030000C94860A0C94860A0C94860A0C9432134B
:100040000C94860A0C94860A0C94860A0C94860AF0
:100050000C94860A0C94E7630C94860A0C94860A26
:100060000C94860A0C9462640C94860A0C94860A9A
:100070000C94860A0C94860A0C94860A0C94860AC0
:100080000C94DF770C94860A0C94860A0C94860AEA
:100090000C9491640C94860A0C94860A0C94860A3B
:1000A0000C94860A0C94860A0C94860A0C94860A90
:1000B0000C94860A0C94860A0C94860A0C94860A80
:1000C0000C94860A0C94860A0C94860A0C94860A70
:1000D0000C94860A0C94860A0C94860A0C94860A60
:1000E0000C94860A0C941D6B0C94276B0C94136B68
:1000F0000C94D36A0C94536B0C94496B0C943D6B29
:100100000C94316B0C94860A0C94860A0C94860A23
:100110000C94860A0C94860A0C94860A0C94860A1F
:100120000C94860A0C94860A0C94860A0C94860A0F
:100130000C94860A0D7E2C7EA57E977FB77FD77F95
:10014000DF7F8C7F084AD73B3BCE016E84BCBFFD6E
:10015000C12F3D6C74319ABD56833DDA3D00C77F97
:1001600011BED9E4BB4C3E916BAAAABE0000008030
:100170003F07634236B79BD8A71A39685618AEBAFC
:10018000AB558C1D3CB7CC5763BD6DEDFD753EF690
:10019000177231BF000000803F08000000BE9224AB
:1001A00049123EABAAAA2ABECDCCCC4C3E000000E0
:1001B00080BEABAAAAAA3E00000000BF00000080DB
:1001C0003F0000000000084178D3BB4387D1133DB6
:1001D000190E3CC3BD4282AD2B3E68EC8276BED97F
:1001E0008FE1A93E4C80EFFFBE01C4FF7F3F0000BE
:1001F000000000000C94A7740C94F2870C943566F0
:100200000C942C7E0C94F0840C94E2100C9449779E
:100210000C9418810C9471650C94145A0C940D7EF6
:100220000C944F840C94B1770C94E0720C946E6B28
:100230000C94F1150C94E5720C946B0E0C94617295
:100240000C9494720C94E8720C9475370C94A57EFF
:100250000C9475680C94E31C0C94D6720C94BA67D9
:100260000C948F760C948A760C94DB720C94510E5D
:100270000C94284C0C948C7F0C941F860C94FF6675
:100280000C94FE140C94DD680C94906C0C94D17258
:100290000C94864C0C949E710C94F2640C94F38034
:1002A0000C9492760C94DF7F0C9408670C945F8119
:1002B0000C94977F0C94A2810C9438720C94C88093
:1002C0000C9440660C94AA710C9445650C94834B75
:1002D0000C945A6A0C942E770C94B77F0C94306966
:1002E0000C94BA770C94D77F6E616E00696E6600CD
:1002F00025630025730A005854414C5F5452494D00
:100300003D25640025730A0025730A005465737443
:1003100020362025730A0054657374203520257318
:100320000A005465737420342025730A00546573E1
:100330007420332025730A005465737420322025FD
:10034000730A005465737420312025730A006368B2
:10035000616E3D25640A0074787077723D25640AE9
:10036000003530306B0A003235306B0A00313135E0
:100370006B0A0035366B0A0033386B0A0025730AA6
:1003800000765F6C6F773D252D332E32660A00258F
:10039000730A0073656E743D252D75206475703D7C
:1003A000252D752069676E6F7265643D252D75205A
:1003B00074746C5F7A65726F3D252D750A00253760
:1003C0002E33662025372E33660025352E326620E3
:1003D000004572726F72203020566F6C74004E6F41
:1003E0007420737570706F727465640A0045727260
:1003F0006F72203020566F6C74004572726F7220DD
:100400003020566F6C740062756C6B5F64656C6154
:10041000793D252D750062756C6B3D252D75005657
:10042000616C7565206E6F7420616C6C6F776564AC
:100430000062756C6B3A206D61783D257520737490
:100440006172743D25752C20656E643D25752C20E8
:10045000696E5F7573653D25750A007062323D25D2
:10046000730A00256C7500416C6C6F7765642073AE
:100470007065656420312F31302F3130302F3430AA
:1004800030206B6269742F730025630074746C3DB7
:10049000252D64200074746C3D252D6420004E656C
:1004A000772074746C3D252D6420002563004D5326
:1004B0003536313120503D252D372E326620252D01
:1004C000372E32666D0A00424D5030383520256C8B
:1004D000642050612020252D372E32666D00256363
:1004E00000545F484541545F4944583D252D352E01
:1004F00032662000545F4445573D252D352E326627
:10050000200041483D252D352E32662000545F5392
:10051000485432583D252D352E3266200052485F12
:1005200053485432583D252D352E32662000545FF5
:1005300052483D252D342E3166200052483D252D50
:10054000342E3166200025630025630025630025D5
:1005500063002563007265706F72745F616C6C3D3F
:10056000007265706F72743D00256300256300257D
:100570006300256300204F534343414C3D256420D5
:100580000020467573653A2065653D253032782038
:1005900068663D25303278206C663D253032782003
:1005A0006C623D25303278004D43553D2530366C28
:1005B000780025630074785F6C656E3D252D6C7541
:1005C0002C765F6C6F773D252D6C752C73687432BB
:1005D000783D252D6C752C62756C6B3D252D6C75E9
:1005E000002563004F4B0A00256300256300256347
:1005F0000025630025630025630025630025630053
:1006000064656275675F616C6C3D00646562756707
:100610003D0064656275673D0025730A0064656589
:10062000700A006E6F6E650A00707772733D00701D
:1006300062323D25730A007062313D25730A0069FC
:100640006E74725F7365635F70313D252D372E3395
:10065000660A00696E74725F70313D252D6C640A04
:1006600000696E74725F7365635F70303D252D376E
:100670002E33660A00696E74725F70303D252D6CF2
:10068000640A00765F6D63753D252D352E32660A4E
:1006900000745F6D63753D252D352E32660A00703E
:1006A0007077723D25730A0064656275673D00725C
:1006B000636D643D25730A0025730A006175746FCC
:1006C0000A006C6F675F6D6F64653D007573625FF4
:1006D0007077723D25730A0072656C61793D2573F0
:1006E0000A0074746C3D252D640A0052494D455F23
:1006F000616464723D252D642E252D640A006E65AB
:10070000696768626F725F7461626C655F73697A52
:10071000653D25640A00765F6C6F773D252D332E8D
:1007200032660A00747870773D25640A0063686158
:100730006E3D25640A0069643D006932635F62753D
:10074000733D006932635F73706565643D252D6C90
:10075000750A007478743D25730A005379737465C3
:100760006D2053756D6D6172790A002530366C7895
:100770000041744D65676132353652465232004150
:10078000744D656761313238524652320041744DC2
:100790006567613634524652320041744D65676177
:1007A00031323852464131004D43553D006D617341
:1007B0006B3D002C00696E74657276616C3D252D71
:1007C000750023252D642C00745F686561745F6972
:1007D000647800745F64657700616800705F6D73B2
:1007E000353631310072685F736874327800745F37
:1007F0007368743278007061007000616434006165
:10080000643300616432006164310061330061323D
:1008100000613100765F696E007268006572720077
:10082000757074696D650070315F6C737400703140
:100830005F740070310070305F6C73740070305FF3
:100840007400703000765F6D637500745F6D637562
:100850000074310074006964006536340074787483
:10086000002D002B006175746F006E6F6E65006265
:10087000756C6B00706F7765725F736176655F6C26
:10088000656472790072656C61795F6C656479008A
:10089000636F6D7061737300616363656C00707288
:1008A000657300705F707772006165730070315F0F
:1008B0006C6564790070305F6C65647200657665A4
:1008C0006E74006C6564006F7700706B74007478F0
:1008D0005F6C6564790072785F6C656472006F703C
:1008E0006572006E6F6E65002530327800765F614C
:1008F00064343D252D382E3666002000765F616415
:10090000333D252D382E3666002000765F61643237
:100910003D252D382E3666002000765F6164313D1E
:10092000252D382E3666002000765F6C6967687466
:100930003D252D382E3666002000765F61323D253C
:100940002D372E3366002000765F61313D252D372F
:100950002E3366002000765F696E3D252D352E32E0
:100960006600204E657665722D757365642073741C
:1009700061636B203E2025642062797465730A00F0
:10098000757074696D653D252D642D646179732DD5
:10099000253032643A253032643A253032642D688D
:1009A0006F7572730A0074657374205B6F66667C82
:1009B000317C327C337C347C355D2020202020202B
:1009C00020202D2074657374206D6F6465730A0D8B
:1009D000007478205B706B74207061796C6F616457
:1009E0005D2020202020202020202020202D20736A
:1009F000656E6420726164696F20706B74206B6532
:100A000079626F6172640A0D00776474205B6F6EA7
:100A10007C6F66667C746573745D202020202020C6
:100A200020202020202D207761746368646F670A7E
:100A30000D00765F6C6F77205B765F6C6F775D2063
:100A400020202020202020202020202020202D2099
:100A50006C6F77657374207265706F727420766F37
:100A60006C746167650A0D00757067722020202024
:100A70002020202020202020202020202020202076
:100A8000202020202D207265626F6F7420766961AE
:100A900020626F6F746C6F616465720A0D0075611E
:100AA0007274205B33386B7C35366B7C3131356B3F
:100AB0007C3235306B7C3530306B5D202D2073659A
:100AC00074207465726D2F75617274207370656522
:100AD000640A0D00626F6F742020202020202020E7
:100AE0002020202020202020202020202020202006
:100AF0002D207265626F6F740A0D0070777273201B
:100B00005B646565707C6E6F6E655D2020202020C3
:100B1000202020202020202D206D637520736C65FF
:100B20006570206D6F64650A0D00726573742065D1
:100B30006570726F6D202020202020202020202032
:100B40002020202020202D20726573746F72652074
:100B5000656570726F6D0A0D0070707772205B6F43
:100B60006E7C6F66665D20202020202020202020C3
:100B700020202020202D2070726F6772616D6D61C2
:100B8000626C65207077720A0D0070623220205B03
:100B90006F6E7C6F66665D20202020202020202044
:100BA0002020202020202D2070726F6772616D6DD3
:100BB00061626C652070696E2062320A0D0070629D
:100BC0003120205B6F6E7C6F66665D2020202020C8
:100BD000202020202020202020202D2062756C6BDA
:100BE000204750494F2070696E0A0D0074787420B8
:100BF0005B737472696E675D2020202020202020A6
:100C000020202020202020202D2053657420726574
:100C1000706F7274207465787420737472696E6773
:100C20000A0D0074787077205B31352D305D2020FF
:100C30002020202020202020202020202020202DA7
:100C4000205458205077722E204869676865737465
:100C5000203020283364426D290A0D0074746C2002
:100C60005B302D31355D20202020202020202020C9
:100C700020202020202020202D2074696D652D74D7
:100C80006F2D6C69766520666F72207061636B658D
:100C900074730A0D00737320202020202020202050
:100CA0002020202020202020202020202020202044
:100CB000202D2073797374656D2073756D6D61726D
:100CC000790A0D007273202020202020202020206F
:100CD0002020202020202020202020202020202014
:100CE0002D20726164696F2073746174730A0D0042
:100CF0007269205B236E5D205B696E745D2020202D
:100D00002020202020202020202020202D2072653F
:100D1000706F727420696E74657276616C0A0D0072
:100D200072636D64205B6F6E7C6F66665D20202051
:100D30002020202020202020202020202D20616C19
:100D40006C6F7720636D642066726F6D206E6574C2
:100D50006F726B0A0D007265205B236E5D205B2B4A
:100D60007C2D5D205B6D61736B7C6175746F2C6D88
:100D700061736B5D202D206D6F7465207265706FDF
:100D80007274207365742F6D6F646966790A0D0043
:100D90006F772020202020202020202020202020AD
:100DA0002020202020202020202020202D206F6E99
:100DB000652D776972652073656E736F72730A0DA6
:100DC000006C6F67205B6175746F7C6F6E7C6F6603
:100DD000665D20202020202020202020202D206D36
:100DE0006F7465732064617461206F6E2055534287
:100DF0000A0D006E65205B666C7573685D202020AF
:100E00002020202020202020202020202020202DD5
:100E1000206E65696768626F72207461626C650A32
:100E20000D0065727220202020202020202020200C
:100E300020202020202020202020202020202D20A5
:100E40006572726F722073746174730A0D006D6342
:100E5000752020202020202020202020202020203D
:100E6000202020202020202020202D206D63752090
:100E7000696E666F0A0D00693263205B70726F6283
:100E8000657C737065656420236E5D2020202020C2
:100E90002020202D206932632070726F62652062ED
:100EA00075737C73657420627573207370656564F7
:100EB0000A0D006964205B72657365745D202020F3
:100EC0002020202020202020202020202020202D15
:100ED0002069642068616E646C696E670A0D006841
:100EE000756D202020202020202020202020202060
:100EF00020202020202020202020202D2068756DFB
:100F000069646974792073656E736F720A0D00727B
:100F1000656C6179205B6F6E7C6F66667C73746153
:100F200074735D20202020202020202D2072656CED
:100F30006179206E6574776F726B207265706F7265
:100F400074730A0D006465205B6D61736B5D202016
:100F50002020202020202020202020202020202091
:100F6000202D2064656275670A0D006368616E203C
:100F70005B31312D32365D202020202020202020A2
:100F8000202020202020202D206368616E20313118
:100F90002D32362028322E3430352D323438302060
:100FA0004D687A290A0D0063616C69205B5B765F8E
:100FB000696E7C61317C61325D20766F6C747C720D
:100FC000657365747C6E6F6E655D202D2063616C4A
:100FD0006962726174650A0D0062756C6B205B5BFF
:100FE00073686F777C666C7573685D205B7365747E
:100FF0002074687273682064656C61795D5D20207F
:101000002D2062756C6B696E67207061636B65740F
:1010100073200A0D006164632020202020202020FE
:1010200020202020202020202020202020202020C0
:10103000202D2073686F7720765F696E2C206131D8
:101040002C20613220766F6C74616765730A0D0025
:10105000752020202020202020202020202020203B
:101060002020202020202020202020202D207570CE
:1010700074696D650A0D0076202020202020202034
:101080002020202020202020202020202020202060
:101090002020202D2076657273696F6E0A0D00681E
:1010A0002020202020202020202020202020202040
:1010B00020202020202020202020202D2068656C4A
:1010C000700A0D00256300756E6B6E6F776E20637E
:1010D0006D640A00484D43353838330025730025C8
:1010E0007300202573002025362E3266200025301F
:1010F00032780074656D705F65787465726E3D2539
:101100002D362E326600202573002025362E3266BD
:10111000204F6E2D426F617264002530327800746A
:10112000656D705F626F6172643D252D362E32668B
:10113000000A0042756C6B2072656D3A2073746111
:1011400072743D25752C20656E643D25752C2069D3
:101150006E5F7573653D25750A0042756C6B206185
:1011600064643A2073746172743D25752C20656E39
:10117000643D25752C20696E5F7573653D25750A84
:101180000042756C6B207468726573683A207469EC
:101190006D65723D25750A00503A20256C6420501B
:1011A000612020252D372E3266206D0A00493243FA
:1011B0003A20004A54414720726573657474210ACD
:1011C000005761746368646F67207265736574218A
:1011D0000A0042726F776E6F757420726573657462
:1011E000210A0045787465726E616C2072657365C2
:1011F00074210A00506F7765722D6F6E20726573CF
:101200006574212E0A004F6E6C696E650A00526F7C
:101210007574696E6720456E61626C65640A005280
:10122000504C20456E61626C65640A002573202570
:10123000732C206368616E6E656C202575202C20F0
:10124000636865636B207261746520257520487A38
:1012500020747820706F7765722025750A000A2A3D
:101260002A2A2A2A2A2A426F6F74696E67202573F8
:101270002A2A2A2A2A2A2A0A004A54414720726521
:10128000736574210A005761746368646F67207224
:1012900065736574210A0042726F776E6F757420F2
:1012A0007265736574210A0045787465726E616CAD
:1012B000207265736574210A00506F7765722D6F17
:1012C0006E2072657365742E0A00726E67206973F2
:1012D000737565732025640A00454550524F4D20B3
:1012E000697320636F72727570742C2072657772E7
:1012F0006974696E672077697468206465666175D2
:101300006C74732E0A006C6F63616C686F73740089
:1013100041544D4547413235367266723200020003
:1013200000FFFE000001452025642E256420636C2B
:101330006F636B20256C752063707520256C75209C
:101340006C706D20256C752069727120256C75207C
:10135000676C656420256C7520796C656420256C4C
:101360007520726C656420256C7520747820256C5E
:1013700075206C697374656E20256C752073656EBD
:10138000736F727320256C752073657269616C20B0
:10139000256C750A0000407A10F35A00A0724E18AE
:1013A000090010A5D4E80000E87648170000E40B17
:1013B00054020000CA9A3B000000E1F505000080DD
:1013C000969800000040420F000000A08601000037
:1013D00000102700000000E8030000000064000087
:1013E0000000000A00000000000100000000002CC6
:1013F00076D888DC674F0823DFC1DFAE59E1B1B78B
:1014000096E5E3E453C63AE651997696E8E6C28457
:1014100026EB898C9B62ED407C6FFCEFBC9C9F406F
:10142000F2BAA56FA5F490055A2AF75C936B6CF994
:10143000676DC11BFCE0E40D47FEF520E6B500D06A
:10144000ED902E0300943577050080841E0800007F
:10145000204E0A000000C80C333333330F986E124D
:10146000831141EF8D2114893BE65516CFFEE6DB53
:1014700018D1844B381BF77C1D901DA4BBE424209D
:101480003284725E228100C9F124ECA1E53D274E31
:10149000414E494E495459494E46CDCCCC3D0AD7D0
:1014A000233C17B7D13877CC2B329595E6241FB162
:1014B0004F0A000020410000C84200401C4620BCEA
:1014C000BE4CCA1B0E5AAEC59D7411241FBECFEF71
:1014D000D1E8DEBFCDBF00E00CBF1AE0A0E0B2E073
:1014E000E2E4FAE201E00BBF02C007900D92A033E4
:1014F000B107D9F729E3A0E3BAE001C01D92A73EE6
:10150000B207E1F70E94C1620C941F950C94000091
:101510002F923F924F925F926F927F928F929F9203
:10152000AF92BF92CF92DF92EF92FF920F931F93F1
:10153000CF93DF93CDB7DEB763970FB6F894DEBFD6
:101540000FBECDBF6C014B012A01FC011782168230
:10155000838181FF43C3AE014F5F5F4F3A01F601C4
:101560009381F40193FD859193FF81914F0188232D
:1015700009F430C3853239F493FD859193FF81914D
:101580004F01853239F4B60190E00E94EB9152018F
:101590002501E5CF10E0F12C20E02032A0F48B32C1
:1015A00069F030F4803259F0833269F420612CC044
:1015B0008D3239F0803339F4216026C022602460F6
:1015C00023C0286021C027FD27C030ED380F3A30F6
:1015D00078F426FF06C0FAE01F9F300D1124132F68
:1015E00013C04AE0F49E300D1124F32E20620CC08B
:1015F0008E3221F426FDEEC2206406C08C3611F432
:10160000206802C0883641F4F40193FD859193FF70
:1016100081914F018111C1CF9BEB980F933018F44A
:101620002061805E06C09BE9980F933008F071C17D
:101630002F7E26FF16E02F73322E853619F4206494
:10164000322E08C0863621F4F22FF0683F2E02C0F9
:101650001111115037FE07C01C3350F4EE24E394EF
:10166000E10E27E00BC0183038F027E017E005C086
:1016700027E04CE3E42E02C0212FE12C520144E08C
:10168000A40EB11CF20160817181828193810E2DC3
:10169000A3010E9462902C01098100FF02C003FF98
:1016A00007C031FC08C032FE09C030E2232E07C05B
:1016B0002DE2222E04C09BE2292E01C0212C802F76
:1016C0008C7019F0211068C2A8C237FE0FC0E40C5C
:1016D00004FF04C08A81813309F4EA941E1474F56E
:1016E000F8E0FE1578F588E0E82E2CC036FC2AC01C
:1016F000812F90E0841595059CF02CEF42162FEF7A
:10170000520674F0432D4068342E0AC0E2E0F0E047
:10171000EC0FFD1FE10FF11D8081803319F4115092
:101720001111F4CF37FE0EC0EE24E394E10E812FA9
:1017300090E0481659062CF4141904C0EE24E394E2
:1017400001C010E037FE06C01414150434F4C201C1
:10175000019605C085E090E002C081E090E0211094
:101760000196112331F0212F30E02F5F3F4F820F80
:10177000931F2F2D30E08217930714F4F81A01C03D
:10178000F12C832D897049F4FF2039F0B60180E2F5
:1017900090E00E94EB91FA94F7CF222029F0B60155
:1017A000822D90E00E94EB9133FC09C0FF2039F0BC
:1017B000B60180E390E00E94EB91FA94F7CF37FEF8
:1017C0005AC0942D852D57FE02C090E080E0292E4E
:1017D000382E20E030E0A2014E1951095D874C8778
:1017E000A201421953095F874E87612F70E0442799
:1017F0005527461B570B598B488B5FEF251635062F
:1018000049F4B6018EE290E02A8B3B8B0E94EB916B
:101810003B892A89421453046CF04C855D8542153E
:10182000530544F4EE85FF85E20FF31FE60DF71D27
:10183000818101C080E351E0251A31082F5F3F4FBD
:1018400048895989241635064CF0B60190E02A8B58
:101850003B8B0E94EB912A893B89CFCF241435041E
:1018600039F49A81963318F4953311F404FF81E327
:10187000B60190E04BC08A81813309F00F7EB6013A
:1018800090E00E94EB91111105C034FC18C085E670
:1018900090E017C0B6018EE290E00E94EB9182E0EA
:1018A000EE24E394E80EF301E80FF11D8081B60108
:1018B00090E00E94EB9111508E2D91F7E6CF85E4D8
:1018C00090E0B6010E94EB9157FC05C04114510411
:1018D00039F404FF05C05194419451088DE201C0D0
:1018E0008BE2B60190E00E94EB9180E39AE049160A
:1018F00051042CF08F5F5AE0451A5108F7CFB6011A
:1019000090E00E94EB91B601C201C0960E94EB915B
:1019100057C1833631F0833779F0833509F058C0E9
:1019200021C05201E2E0AE0EB11CF2018081898338
:1019300001E010E0230114C05201F2E0AF0EB11C2F
:10194000F2014080518026FF03C0612F70E002C089
:101950006FEF7FEFC2012A8B0E9497918C012A8939
:101960002F7715C05201F2E0AF0EB11CF20140809A
:10197000518026FF03C0612F70E002C06FEF7FEF40
:10198000C2012A8B0E944C918C012A892068322E38
:1019900023FD1AC08F2D90E008171907A8F4B6018F
:1019A00080E290E00E94EB91FA94F4CFF20137FCD0
:1019B000859137FE81912F01B60190E00E94EB9155
:1019C000F110FA94015011090115110579F7F8C0C9
:1019D000843611F0893659F5520127FF09C0F4E029
:1019E000AF0EB11CF20160817181828193810AC0C6
:1019F000F2E0AF0EB11CF20160817181072E000C84
:101A0000880B990B2F76322E97FF09C09095809501
:101A1000709561957F4F8F4F9F4F2068322E2AE03F
:101A200030E0A3010E94FC92E82EE6183FC0022F8E
:101A3000853721F40F7E2AE030E01DC0097F8F3604
:101A400091F018F4883559F0C5C0803719F08837FF
:101A500011F0C0C0006104FF09C0046007C024FF8A
:101A600008C0066006C028E030E005C020E130E094
:101A700002C020E132E0520107FF09C0F4E0AF0EDE
:101A8000B11CF201608171818281938108C0F2E012
:101A9000AF0EB11CF2016081718180E090E0A30182
:101AA0000E94FC92E82EE6180F77302E36FE0BC00F
:101AB000332D3E7FE11650F434FE0AC032FC08C0DC
:101AC000332D3E7E05C00E2D332D03C00E2D01C0DB
:101AD000012F34FF0CC0FE01EE0DF11D808180331B
:101AE00011F4397E08C032FF05C00E5F04C0832F99
:101AF000867809F00F5F33FD13C030FF06C01E2D3E
:101B00000F1518F41F0D101B0F2D0F1568F4B601DB
:101B100080E290E03B8B0E94EB910F5F3B89F5CF19
:101B20000F1510F4F01A01C0F12C34FF12C0B601E9
:101B300080E390E03B8B0E94EB913B8932FF17C022
:101B400031FD03C088E790E002C088E590E0B6016F
:101B50000CC0832F867859F031FF02C08BE201C0A0
:101B600080E237FD8DE2B60190E00E94EB91E11634
:101B700038F4B60180E390E00E94EB911150F7CF6A
:101B8000EA94F301EE0DF11D8081B60190E00E9410
:101B9000EB91E110F5CF14C0F4E0FF1558F584E0A7
:101BA000F81A33FE1EC0211026C003FF2AC008EE1B
:101BB00012E0F32DF0713F2EF8018491811124C0C1
:101BC000FF2009F4E5CCB60180E290E00E94EB91A1
:101BD000FA94F6CFF6018681978126C08FEF9FEFAA
:101BE00023C0B60180E290E00E94EB91FA94F110DC
:101BF000F8CFD9CFF12CB601822D90E00E94EB9165
:101C0000D4CF0CEE12E0D5CF31108052B60190E067
:101C10000E94EB910F5F1F4FCFCF23E02F1510F4E1
:101C200083E0BECFF12CC1CF63960FB6F894DEBF30
:101C30000FBECDBFDF91CF911F910F91FF90EF901D
:101C4000DF90CF90BF90AF909F908F907F906F90DC
:101C50005F904F903F902F9008958115910511F05E
:101C60000197F1F7089589E296E09F938F930E9480
:101C700037928091660290916702A0916802B091BC
:101C800069020F900F9093FF03C083E296E002C0B9
:101C90008DE196E09F938F930E9437920F900F9063
:101CA0000895E091E21CEF73F0E0ED5CF24E80836A
:101CB0008091E21C8F5F8093E21C80918335886065
:101CC000809383354CE452E061E1CA010E94D26EF8
:101CD00080E090E00895CF93DF93EC018091891329
:101CE00090918A13A0918B13B0918C1386FF1DC025
:101CF0008E811F928F938D811F928F938C811F9263
:101D00008F938B811F928F938A811F928F9389EE7D
:101D100092E09F938F930E9423928DB79EB70C966B
:101D20000FB6F8949EBF0FBE8DBFBE018BE79AE041
:101D30000E94CB6FBE0188E092E0DF91CF910C94BE
:101D4000587052985A981DBAE9E6F0E08081806296
:101D50008083EA9A53985B98EB9A808180688083AD
:101D6000E8E6F0E08081816080830895E8E9FDE1A4
:101D70001182128210820895CF92DF92EF92FF9229
:101D80000F931F93CF93DF93EC019B018091981DDC
:101D9000843108F0BBC080919A1D64E10E94B28634
:101DA00090939A1DC090B530D090B630E090B73087
:101DB000F090B830092F10E08DE8989FD0011124E1
:101DC000A856B24E1396CD92DD92ED92FC921697E4
:101DD0004115510559F0FA018081FD01EA57FF4F85
:101DE0008083FA018181A957BF4F8C932097A9F076
:101DF00089819DE8909FF001919FF00D1124E85694
:101E0000F24EDF01A657BF4F8C93E557FF4F8881F5
:101E10008F70808388818F70808321153105E1F177
:101E2000D90116964C9116975DE8509FC001519FBD
:101E3000900D11248856924EFC01E757FF4F4083C6
:101E400015964C9115973197408334961B964D917A
:101E50005D916D917C911E97452F562F672F7727A7
:101E6000518340837C01BEE8EB0EF11CF901238510
:101E7000348545855685A4E6B0E00E944D87672FDE
:101E8000782F892F992724E630E040E050E00E9427
:101E9000E686D7016D937C938DE8809FD001819F6A
:101EA000B00D1124A156B24EFE0132968FE701907B
:101EB0000D928A95E1F780919A1D8F5F80939A1D0C
:101EC0009091981D9F5F9093981D40918913509118
:101ED0008A1360918B1370918C1360FF2DC01F9239
:101EE0009F931F928F938091991D1F928F938AE5E4
:101EF00091E19F938F930E943792EDB7FEB738968A
:101F00000FB6F894FEBF0FBEEDBF16C08091C5306E
:101F10009091C630A091C730B091C8300196A11DF4
:101F2000B11D8093C5309093C630A093C730B09355
:101F3000C83080E090E002C081E090E0DF91CF9176
:101F40001F910F91FF90EF90DF90CF900895209117
:101F5000981D222361F18091991D8F5F215020935C
:101F6000981D64E10E94B2869093991D4091891357
:101F700050918A1360918B1370918C1360FF1AC07B
:101F80001F922F9380919A1D1F928F931F929F9360
:101F900083E391E19F938F930E9437928DB79EB711
:101FA00008960FB6F8949EBF0FBE8DBF03C080E0A9
:101FB00090E0089581E090E008951F920F920FB68F
:101FC0000F9211248F939F93AF93BF9380916800DA
:101FD00080FF24C080915E3590915F35A09160357F
:101FE000B09161350196A11DB11D80935E3590932E
:101FF0005F35A0936035B0936135809189139091DE
:102000008A13A0918B13B0918C1387FF07C074982B
:1020100082E090E09093920280939102BF91AF9101
:102020009F918F910F900FBE0F901F9018951F9248
:102030000F920FB60F9211248F939F93AF93BF937C
:102040008091680080FF24C0809162359091633553
:10205000A0916435B09165350196A11DB11D8093A5
:10206000623590936335A0936435B0936535809164
:10207000891390918A13A0918B13B0918C1390FFC8
:1020800007C0739882E090E090939202809391024F
:10209000BF91AF919F918F910F900FBE0F901F90A6
:1020A000189580937C0080917B00877F80937B00D4
:1020B00080917C00806C80937C0085E080937A0026
:1020C00080917A00806880937A0080917B0087FFFE
:1020D000FCCF80917B0085FFFCCF80917A008064EB
:1020E00080937A0080917A0086FDFCCF109279006F
:1020F0001092780084E090E060E070E020917A0037
:10210000206420937A0020917A0026FDFCCF209154
:10211000780030917900620F731F019779F7109260
:102120007C0080917A008F7780937A00769567950E
:102130007695679580E090E00E94BB8A089580E0E4
:102140000E9451102091890230918A0240918B02A5
:1021500050918C020E94B58C21EE3AE744E95EE38F
:102160000E94268908950F931F93CF93DF930FE169
:1021700010E0CBE5DEE00093510182E991E00E949E
:102180002D0E8091510185FD0DC00031110521F00A
:102190002CF0CB54D10903C0C4ECD9E0E297015034
:1021A0001109E9CFBE0180E090E00E94BB8A20E0E7
:1021B00030E04AE754E40E94098ADF91CF911F91F1
:1021C0000F910895CF93DF93EC0188819981009757
:1021D00099F0863D914121F01982188283E011C067
:1021E000623171F40E94B3106093B1307093B230D9
:1021F0008093B3309093B43086ED91E199838883D6
:1022000081E0DF91CF91089580917B008860809379
:102210007B0089EC80937C0085E080937A0080913C
:102220007A00806880937A0080917B0087FFFCCFE2
:1022300080917B0085FFFCCF80917A008064809341
:102240007A0080917A0086FDFCCF80917A008064CC
:1022500080937A0080917A0086FDFCCF60917800AF
:102260007091790080917A008F7780937A0080E076
:1022700090E00E94BB8A27ED33EA40E95FE30E94C9
:10228000B58C26E636E648E853E40E942589089591
:10229000CF92DF92EF92FF921F93CF93DF93CDB750
:1022A000DEB729970FB6F894DEBF0FBECDBF6C0125
:1022B000109283138FEF89878BEEE82E8CE1F82E36
:1022C00010E089858823E9F11830D9F1BE016F5FEC
:1022D0007F4FCE0109960E94D05D99859F3F11F0F6
:1022E0009E3F19F4909383132CC0CE010196C11424
:1022F000D10481F40E94E95D80938035A8E7B5E3BD
:10230000FE01319688E08E0F91919D938E13FCCF44
:1023100081E018C00E94E95DF7018087FE013196D7
:1023200020E030E08191D701A20FB31F8C932F5F83
:102330003F4F28303105B1F71F5FF9E0EF0EF11C78
:10234000C0CF812F29960FB6F894DEBF0FBECDBF48
:10235000DF91CF911F91FF90EF90DF90CF90089584
:1023600081E391E19F938F930E9437920F900F909A
:1023700008952F923F924F925F926F927F928F9229
:102380009F92AF92BF92CF92DF92EF92FF920F9304
:102390001F93CF93DF93EC015B01009711F427E0CB
:1023A00003C0019749F426E04AE250E06BE270E096
:1023B00089E290E00E94B05CCE010E9448119E012B
:1023C0002C573C4E6901D9018C93CD2B69F0CBEE93
:1023D000DCE1E12CF12C86EE282E80E1382E92EE05
:1023E000892E90E1992E9EC088E795E30E947C5E3D
:1023F000BC01990F880B990B0E94BD8A6B017C016F
:10240000AB2869F020E030E048EC52E40E94098AF1
:102410009F938F937F936F938FE191E1A4C0C8E75F
:10242000D5E30AE111E189911F928F931F930F93D6
:102430000E9437920F900F900F900F90B5E3C03825
:10244000DB0789F720E030E048EC52E4C701B60131
:102450000E94098A9F938F937F936F938AE091E103
:102460009F938F930E9437920F900F900F900F9031
:102470000F900F9080918035811103C08CE893E01C
:1024800002C088E193E09F938F9386E091E19F9350
:102490008F930E9437920F900F900F900F906DC006
:1024A00000E010E0FE01E00FF11F80811F928F938A
:1024B000AEEEB0E1BF93AF930E9437920F5F1F4F14
:1024C0000F900F900F900F900830110559F720E0F2
:1024D00030E048EC52E4C301B2010E94098A9F93A4
:1024E0008F937F936F933F922F920E9437920F901A
:1024F0000F900F900F900F900F908885811151C011
:102500008CE893E09F938F939F928F920E943792D3
:102510000E94B011FFEFEF1AFF0A29960F900F905B
:102520000F900F90D6018C9190E0E816F906E4F533
:10253000CE010E947C5EBC01990F880B990B0E9412
:10254000BD8A2B013C01A114B10409F4A9CF20E0FC
:1025500030E048EC52E40E94098A9F938F937F9366
:102560006F9383EF90E19F938F930E9437920F9028
:102570000F900F900F900F900F90DF91CF911F91C0
:102580000F91FF90EF90DF90CF90BF90AF909F9012
:102590008F907F906F905F904F903F902F900C9412
:1025A000B01188E193E0AECFDF91CF911F910F91F1
:1025B000FF90EF90DF90CF90BF90AF909F908F9063
:1025C0007F906F905F904F903F902F900895CF93A2
:1025D000DF931F921F92CDB7DEB7E8E7F5E3818165
:1025E000898387818A83CE0101960E94FC720F90B5
:1025F0000F90DF91CF910895CF93DF93EC0120915D
:1026000078353091793540917A3550917B356091AC
:102610007C3570917D3580917E3590917F35AFEF1F
:102620000E941989E1F427E04AE250E06BE270E091
:1026300089E290E00E94B05C80E090E00E94481146
:10264000CC57DC4E888349E050E06EE070E088E7CC
:1026500095E30E940295DF91CF910C94E712DF91F0
:10266000CF9108951F920F920FB60F9211240BB6BF
:102670000F92FF920F931F932F933F934F935F936C
:102680006F937F938F939F93AF93BF93CF93DF937A
:10269000EF93FF938091833582608093833580919F
:1026A000660286FD2B9A8091660287FD2B9A8091A7
:1026B0009102909192021816190614F4749A739A62
:1026C0008091891390918A13A0918B13B0918C13F0
:1026D00085FF02C07498739880910602909107025A
:1026E00001979093070280930602892B09F04CC151
:1026F00080913E0A90913F0A019690933F0A809301
:102700003E0A8091B5309091B630A091B730B0912B
:10271000B8300196A11DB11D8093B5309093B630AD
:10272000A093B730B093B83080E190E09093070267
:10273000809306028091660280FD02C01D9B05C049
:10274000109288131092871306C081E090E0909356
:102750008813809387138091891390918A13A09195
:102760008B13B0918C1397FF08C0809187139091C1
:102770008813892B49F0749A739802E91CE1CAEC1A
:10278000D0E3FF24F39421C0739A7498F6CF80911C
:102790003E0A90913F0A01960E94BE86892BE1F085
:1027A000F8016085718561157105A1F5F8016085F5
:1027B00071856115710509F03FC0065F1F4F2596B1
:1027C000F0E3CE3DDF0709F44CC0F8016085718568
:1027D0006115710529F3DBCF4281417020E030E0C3
:1027E00050E060E070E080E090E0A0E00E94198995
:1027F000B9F277988091891390918A13A0918B13E5
:10280000B0918C1392FFCCCF7498109292021092D8
:102810009102C6CF80913E0A90913F0A01960E9494
:10282000BE86892B19F61C821B82AE0162E184E20E
:1028300092E00E94D26EBACF80913E0A90913F0AF8
:102840000E94BE86892B09F0B8CFF8821A830983CB
:102850001C821B82AE0162E182E492E00E94D26E91
:10286000ACCF60916C0270916D0261157105A1F1A0
:1028700080913E0A90913F0A0E94BE86892B61F5A5
:1028800080915E3590915F35A0916035B091613552
:102890004091A7285091A8286091A9287091AA2852
:1028A000841B950BA60BB70B8093BA1C9093BB1C93
:1028B000A093BC1CB093BD1C80915E3590915F3598
:1028C000A0916035B09161358093A7289093A82896
:1028D000A093A928B093AA2860916A0270916B0214
:1028E00061157105A1F180913E0A90913F0A0E9405
:1028F000BE86892B61F58091623590916335A091F8
:102900006435B09165354091AB285091AC28609109
:10291000AD287091AE28841B950BA60BB70B809346
:10292000BE1C9093BF1CA093C01CB093C11C80918F
:10293000623590916335A0916435B091653580938F
:10294000AB289093AC28A093AD28B093AE2880918B
:10295000660286FD2B988091660290916702A09195
:102960006802B091690291FF0FC00E94F8678A3136
:1029700019F0C1E0C80F01C0CBE00E9435668C2F72
:102980000E9410680E94FF6640E050E060E085EB26
:1029900092E00E94D26EFF91EF91DF91CF91BF91B3
:1029A000AF919F918F917F916F915F914F913F91E7
:1029B0002F911F910F91FF900F900BBE0F900FBEA4
:1029C0000F901F9018958091E21C9091C930891B3F
:1029D00008950E94E314882371F0E091C930EF73E9
:1029E000F0E0ED5CF24E808190E02091C9302F5FE5
:1029F0002093C93008958FEF9FEF0895CF93DF9311
:102A0000EC0110926F0A10926E0A888199810097EA
:102A1000C1F0843E934021F01982188283E0BDC04A
:102A2000613109F0B9C00E94E914992790936A0AAC
:102A30008093690A8D30910509F444C08F3F910558
:102A400049F40E94E3148111EECF84EE93E0998360
:102A50008883A2C08231910509F45AC08F3791054D
:102A600009F052C08091670A9091680A18161906F9
:102A70000CF56091E1397091E23988E090E00E94B4
:102A8000EB916091E1397091E23980E290E00E942F
:102A9000EB916091E1397091E23988E090E00E9419
:102AA000EB918091670A9091680A01979093680A68
:102AB0008093670A8091670A9091680A8F37910521
:102AC00009F0BFCF1092C9301092E21C8091670AC2
:102AD0009091680AFC01E252FF4C108290936F0AB9
:102AE00080936E0A1092680A1092670A809181356D
:102AF00090918235009709F4A4CF40E050E06091B6
:102B000081130E94D26E9DCF8830910571F5AACFB6
:102B10006091E1397091E2398DE090E00E94EB9193
:102B20001092660A1092650A2091650A3091660A31
:102B30008091670A9091680A281739070CF0BACF7C
:102B4000F901E252FF4C80816091E1397091E239E4
:102B500090E00E94EB918091650A9091660A01963F
:102B60009093660A8093650ADFCF6091E139709196
:102B7000E2390E94EB912091670A3091680A8091B6
:102B8000690AF901E252FF4C80832F5F3F4F309377
:102B9000680A2093670A8ECF81E0DF91CF91089574
:102BA0008091871390918813892BD1F080916602D0
:102BB00090916702A0916802B091690293FD10C0E4
:102BC0000E94356683B7817F866083BFF89483B7A0
:102BD000816083BF7894889583B78E7F83BF789414
:102BE0000895CF93DF93FC012081318121153105B8
:102BF00051F02930324129F0FC011182108283E02A
:102C000015C0653891F4EC010E9436650E94D0151C
:102C100040E050E065E88091CB149091CC140E9484
:102C2000D26E89E092E19983888381E0DF91CF9130
:102C30000895CF93DF931F921F92CDB7DEB7892BF4
:102C400081F05F934F938FED90E19F938F93698312
:102C50007A830E9437920F900F900F900F907A8195
:102C600069817F936F938CED90E19F938F930E9486
:102C700037920F900F900F900F900F900F90DF9161
:102C8000CF910895EF92FF920F931F93CF93DF930D
:102C90000E94366580EB0E94095F81111CC00E9472
:102CA0006D5F8091AF2C9091B02C81609093B02C8F
:102CB0008093AF2C81E293E09F938F938CED90E112
:102CC0009F938F930E9437920F900F900F900F90C9
:102CD000C1E0D0E002C0C0E0D0E01EB11470729A32
:102CE0000E9436658EE40E94095F811117C00E9420
:102CF0006D5F8091AF2C9091B02C82609093B02C3E
:102D00008093AF2C7E018FEFE81AF80A43E159E077
:102D100069E273E0CE010E941916E701111101C0AA
:102D200072980E9436658EEE0E94095F811116C06E
:102D30000E946D5F8091AF2C9091B02C8460909335
:102D4000B02C8093AF2C8E010F5F1F4F43E159E0F1
:102D500061E373E0CE010E941916E8010E94366516
:102D600086EA0E94095F811116C00E946D5F809102
:102D7000AF2C9091B02C88609093B02C8093AF2CA6
:102D80008E010F5F1F4F43E159E068E373E0CE010E
:102D90000E941916E8010E9436658CE30E94095FC3
:102DA00081111EC00E946D5F8091AF2C9091B02C5C
:102DB00080619093B02C8093AF2C8E010F5F1F4FDA
:102DC00043E159E060E473E0CE010E94191684EDFE
:102DD00090E19F938F930E9437920F900F90E8019C
:102DE0000E94366582ED0E94095F811116C00E9423
:102DF0006D5F8091AF2C9091B02C80629093B02C3D
:102E00008093AF2C8E010F5F1F4F43E159E068E4C0
:102E100073E0CE010E941916E8010E94366580E831
:102E20000E94095F811116C00E946D5F8091AF2CD6
:102E30009091B02C91609093B02C8093AF2C8E0128
:102E40000F5F1F4F43E159E061E573E0CE010E943F
:102E50001916E8010E94366580ED0E94095F811114
:102E600016C00E946D5F8091AF2C9091B02C80684D
:102E70009093B02C8093AF2C8E010F5F1F4F43E1D6
:102E800059E067E573E0CE010E941916E8010E943F
:102E900036658CEE0E94095F811116C00E946D5F3D
:102EA0008091AF2C9091B02C92609093B02C809335
:102EB000AF2C8E010F5F1F4F43E159E06FE573E0C8
:102EC000CE010E941916E80107E010E00E94366565
:102ED0008CE70E94095F811113C00E946D5F809191
:102EE000AF2C9091B02C80649093B02C8093AF2C39
:102EF00043E159E066E673E0CE010E94191603C073
:102F00000150110919F70E946D5FDF91CF911F9158
:102F10000F91FF90EF900C94B011CF93DF931F921D
:102F20001F92CDB7DEB74A8369830E94445F6981EF
:102F3000862F0E94755F4A81842F0E94755F0F90D3
:102F40000F90DF91CF910C946D5FAF92BF92CF92B3
:102F5000DF92EF92FF920F931F93CF93DF9300D0F6
:102F6000CDB7DEB7182F022F4A835B8369830E9497
:102F7000445F6981862F0E94755F812F81600E9466
:102F80006B5F4A81A42E5B81B52E10E0E12CF12C01
:102F9000680181E0C81AD108E016F10689F0EC1446
:102FA000FD0419F40E94905F02C00E94865FF50143
:102FB0008083FFEFEF1AFF0A8FEFA81AB80AECCF51
:102FC0000F900F900F90DF91CF911F910F91FF9075
:102FD000EF90DF90CF90BF90AF900C946D5FBF9259
:102FE000CF92DF92EF92FF920F931F93CF93DF93D5
:102FF000CDB7DEB760970FB6F894DEBF0FBECDBF7A
:10300000F82EE42E6623D9F18E010F5F1F4F80E169
:10301000F80111928A95E9F728E0A80168E980EBA8
:103020000E94A517FF2041F08FE693E09F938F93B6
:103030000E9423920F900F9026E7C22E23E0D22EFB
:1030400037E0B32EB00EF80181918F011F928F935C
:10305000DF92CF920E9423920F900F900F900F90CB
:10306000B012F1CF88851F928F938BEC93E09F93E2
:103070008F930E9423920F900F900F900F90EE204D
:10308000D9F18E010F5F1F4F80E1F80111928A95EF
:10309000E9F720E1A80160E880EB0E94A517FF2076
:1030A00041F08BE793E09F938F930E9423920F90C0
:1030B0000F9086E7E82E83E0F82E9FE0D92ED00E01
:1030C000F80181918F011F928F93FF92EF920E94DE
:1030D00023920F900F900F900F90D012F1CF88890C
:1030E0001F928F938BEC93E09F938F930E94239278
:1030F0000F900F900F900F9060960FB6F894DEBF70
:103100000FBECDBFDF91CF911F910F91FF90EF9038
:10311000DF90CF90BF9008950F931F93CF93DF93CD
:103120001F921F92CDB7DEB71A82198222E0AE013C
:103130004F5F5F4F6AEA8EEE0E94A51703E71DE11D
:10314000898190E0982F88272A81822BF80191832A
:10315000808322E0AE014F5F5F4F6CEA8EEE0E94EB
:10316000A517898190E0982F88272A81822BF80162
:103170009383828322E0AE014F5F5F4F6EEA8EEE53
:103180000E94A517898190E0982F88272A81822B99
:10319000F8019583848322E0AE014F5F5F4F60EBBF
:1031A0008EEE0E94A517898190E0982F88272A81AA
:1031B000822BF801938B828B22E0AE014F5F5F4F31
:1031C00062EB8EEE0E94A517898190E0982F8827E8
:1031D0002A81822BF801958B848B22E0AE014F5F10
:1031E0005F4F64EB8EEE0E94A517898190E0982FC7
:1031F00088272A81822BF801978B868B22E0AE01EB
:103200004F5F5F4F66EB8EEE0E94A517898190E0BD
:10321000982F88272A81822BF8019783868322E0C2
:10322000AE014F5F5F4F68EB8EEE0E94A51789815C
:1032300090E0982F88272A81822BF8019187808738
:1032400022E0AE014F5F5F4F6AEB8EEE0E94A51742
:10325000898190E0982F88272A81822BF801958711
:10326000848722E0AE014F5F5F4F6CEB8EEE0E94D1
:10327000A517898190E0982F88272A81822BF80151
:103280009787868722E0AE014F5F5F4F6EEB8EEE31
:103290000E94A517898190E0982F88272A81822B88
:1032A000F801918B808B0F900F90DF91CF911F9140
:1032B0000F9108952F923F924F925F926F927F925B
:1032C0008F929F92AF92BF92CF92DF92EF92FF9236
:1032D0000F931F93CF93DF93CDB7DEB76C970FB6E5
:1032E000F894DEBF0FBECDBF182F042F2D8B19828F
:1032F0001A821B828091971D811107C06C8F0E94DA
:103300008C1881E08093971D6C8D662309F472C040
:103310004EE264EF8EEE0E948D1762E174E380E06E
:1033200090E00E94E75E22E0AE014F5F5F4F66EFE4
:103330008EEE0E94A5172981822F90E0A0E0B0E0D8
:103340004427582F692F7A2F8A81482B8091891D15
:1033500090918A1D9A01AB01281B390B4109510933
:10336000A091871DB091881D0E944D876B017C0143
:103370003FE0F594E794D794C7943A95D1F76091DC
:10338000811D7091821DCB01770FAA0BBB0BBC0175
:10339000CD014BE0660F771F881F991F4A95D1F723
:1033A0002091831D3091841D4901330FAA08BB0869
:1033B000A7019601280D391D4A1D5B1D0E94088733
:1033C000C20ED31ED0927E1DC0927D1D28E0C20E7B
:1033D000D11C54E0D594C7945A95E1F70D2C000CFC
:1033E000EE08FF08C0928B1DD0928C1DE0928D1DBF
:1033F000F0928E1D812F8295880F880F807C8C5CC7
:103400008887212E312CA3E0B0E0012E02C0AA0F44
:10341000BB1F0A94E2F72AE63AE00E9446879B0126
:10342000AC012E5F3F4F4F4F5F4F29873A874B8745
:103430005C8780E593ECA0E0B0E09C01AD0104C0A6
:1034400055954795379527951A95D2F7298B3A8B3D
:103450004B8B5C8B10E0412C512C320188E090E0CA
:10346000AC01421953095B8F4A8F101709F43EC112
:10347000488564EF8EEE0E948D1769857A858B856D
:103480009C850E94E75E23E0AE014F5F5F4F66EFD1
:103490008EEE0E94A517E0917D1DF0917E1DE05AF1
:1034A000FF409F01DF010E942F876C837D838E8305
:1034B0009F838091751D9091761D9E878D872091A9
:1034C000731D3091741D388B2F872091771D30919B
:1034D000781D0E942F876B017C01ADE0F594E79485
:1034E000D794C794AA95D1F7A091791DB0917A1D70
:1034F0002C813D814E815F818CE0559547953795B4
:1035000027958A95D1F70E945887BB2797FDB095DC
:10351000AB2F8C0D9D1DAE1DBF1D0296A11DB11DB3
:1035200032E0B595A795979587953A95D1F79C0187
:10353000AD0130584F4F5F4FA091851DB091861D52
:103540000E944D874B015C014FE0B694A79497947D
:1035500087944A95D1F739818A8190E0A0E0B0E064
:10356000BA2FA92F982F8827A32B2B81822B9C0160
:10357000AD010A8C04C055954795379527950A9457
:10358000D2F72E8B3F8B488F598F4F8558896A0110
:10359000550FEE08FF0862E0CC0CDD1CEE1CFF1C92
:1035A0006A95D1F7A0917B1DB0917C1D2C813D8146
:1035B0004E815F810E9458879B01AC0177E1559550
:1035C0004795379527957A95D1F72C833D834E8380
:1035D0005F832D853E85DF010E942F87DC01CB01B3
:1035E000EBE0B595A79597958795EA95D1F72C814E
:1035F0003D814E815F81820F931FA41FB51FC80EAE
:10360000D91EEA1EFB1E022C04C0CC0CDD1CEE1CD5
:10361000FF1C0A94D2F732E0C30ED11CE11CF11C4E
:10362000F2E0F594E794D794C794FA95D1F72E89F0
:103630003F89488D598D2C193D094E095F096989CB
:103640007A898B899C890E94A28697FD0BC0660FA0
:10365000771F881F991FA50194010E94E6866901C2
:103660007A010AC0A50194010E94E68669017A01E7
:10367000CC0CDD1CEE1CFF1C9927F7FC9A958F2DB6
:103680007E2D6D2D9B01AC010E94A2869B01AC0199
:10369000AEEDBBE00E944D874C01BB2497FCB0947B
:1036A000AB2CA3E4B3EEA70196010E945B87BB2776
:1036B00097FDB095AB2F880E991EAA1EBB1E4FEC2E
:1036C000840E4EE0941EA11CB11C44E0B594A79456
:1036D000979487944A95D1F7C80CD91CEA1CFB1C17
:1036E0004C0C5D1C6E1C7F1C1F5FBFCE112381F034
:1036F000212F30E040E050E0C301B2010E94E68695
:1037000020938F1D3093901D4093911D5093921DD7
:103710005D89552389F160918F1D7091901D809175
:10372000911D9091921D611571058105910521F101
:103730000E94BD8A20E836EE45EC57E40E94098AD3
:1037400021E03EED42E45EE30E94228D9B01AC014C
:1037500060E070E080E89FE30E9425892BE43AE373
:103760004DEB57E30E94098A6093931D7093941D5B
:103770008093951D9093961D6C960FB6F894DEBFBE
:103780000FBECDBFDF91CF911F910F91FF90EF90B2
:10379000DF90CF90BF90AF909F908F907F906F9071
:1037A0005F904F903F902F9008950F931F93CF936A
:1037B000DF9300D000D0CDB7DEB78E010F5F1F4F73
:1037C00086E0F80111928A95E9F78091891C8111B0
:1037D00013C040E061E386EA0E948D174AE06CE284
:1037E00086EA0E948D1781E08093891C68EF7CE750
:1037F00080E090E00E94E75E48E06DE286EA0E9489
:103800008D1768EF7CE780E090E00E94E75E26E09D
:10381000A80162E386EA0E94A51747E06DE286EA06
:103820000E948D178A8190E0982F88272981822B0A
:103830009093841C8093831C2C8130E0322F2227AC
:103840004B81242B3093861C2093851C4E8150E0A5
:10385000542F44276D81462B5093881C4093871C1E
:103860005F934F933F932F939F938F938FE793E0B3
:103870009F938F930E9423920FB6F894DEBF0FBEE2
:10388000CDBF26960FB6F894DEBF0FBECDBFDF9139
:10389000CF911F910F910895CF92DF92EF92FF92F7
:1038A0000F931F93CF93DF93CDB7DEB72A970FB651
:1038B000F894DEBF0FBECDBF8E010F5F1F4F86E0B5
:1038C000F80111928A95E9F741E062E08CE30E94E9
:1038D0008D1748E560E08CE30E948D1764E278E67E
:1038E00080E090E00E94E75E26E0A80163E08CE3C0
:1038F0000E94A51743E062E08CE30E948D170981C6
:1039000010E0102F00278A81082BE3E6FCE11183E9
:103910000083EB80F12CFE2CEE248C81E82AF382CC
:10392000E282CD80D12CDC2CCC248E81C82AD58299
:10393000C482B801012E000C880B990B0E94BD8A2D
:103940009B01AC01B7010F2C000C880B990B2F8346
:10395000388749875A870E94BD8A2F8138854985D3
:103960005A850E94A58920EE3EE245E652E40E9477
:10397000B58C20E030E044E353E40E9426899F9315
:103980008F937F936F93DF92CF92FF92EF921F936B
:103990000F938DE893E09F938F930E9423920FB62D
:1039A000F894DEBF0FBECDBF2A960FB6F894DEBFE7
:1039B0000FBECDBFDF91CF911F910F91FF90EF9080
:1039C000DF90CF900895CF93DF93EC0188819981A8
:1039D000009759F1823F914121F01982188283E0CA
:1039E00071C08CE49AE00E94606D892B51F1809146
:1039F000891390918A13A0918B13B0918C1393FD2E
:103A000022C08091891390918A13A0918B13B09159
:103A10008C1394FD49C08091891390918A13A091D1
:103A20008B13B0918C1395FD46C040E850E060E0E8
:103A300070E08CE49AE00E94426D82EF91E19983FC
:103A4000888381E03FC08091AF2C82FFDACF21E0F4
:103A500048E061E083E00E945A198091961D8F939F
:103A60008091951D8F938091941D8F938091931DCC
:103A70008F938091921D8F938091911D8F93809150
:103A8000901D8F9380918F1D8F9388E991E19F9373
:103A90008F930E9437928DB79EB70A960FB6F8940F
:103AA0009EBF0FBE8DBFADCF8091AF2C83FFB3CF34
:103AB0000E94D51BB0CF8091AF2C84FFB6CF0E945F
:103AC0004C1CB3CFDF91CF910895CF93C82F8CEECC
:103AD0000E946B5F8C2F0E94755F6AE67AE080E03F
:103AE00090E00E94E75E8DEE0E946B5F0E94865F11
:103AF000C82F0E94905F2C2F30E0322F2227A9017F
:103B0000482BCA01CF9108950F931F93CF93DF9352
:103B1000C82F8CEE0E946B5F8C2F0E94755F64E251
:103B200078E680E090E00E94E75E8CEE0E946B5F9A
:103B300080E00E94755F6AE67AE080E090E00E9493
:103B4000E75E8DEE0E946B5F0E94865FC82F0E9429
:103B5000865FD82F0E94905F4D2F50E060E070E0AC
:103B6000762F652F542F44276C2B8A019B01082B3D
:103B7000C901B801DF91CF911F910F9108952F9244
:103B80003F924F925F926F927F928F929F92AF92ED
:103B9000BF92CF92DF92EF92FF920F931F93CF933A
:103BA000DF93CDB7DEB7CB54D1090FB6F894DEBFA3
:103BB0000FBECDBF8091040290910502892BD1F1F7
:103BC00010920502109204028CEE0E946B5F8EE14F
:103BD0000E94755F66E37CE980E090E00E94E75E0A
:103BE00082EA0E94651D90933D0A80933C0A84EA14
:103BF0000E94651D90933B0A80933A0A86EA0E94D0
:103C0000651D9093390A8093380A88EA0E94651DE1
:103C10009093370A8093360A8AEA0E94651D909332
:103C2000350A8093340A8CEA0E94651D9093330A0A
:103C30008093320A88E40E94841D6DAB7EAB8FAB0B
:103C400098AF88E50E94841D4B015C018091340A85
:103C50009091350A8C0120E030E040E050E0BA015C
:103C600022968FAF229723961FAF239724962FAFCC
:103C7000249725963FAF259726964FAF26972796F0
:103C80005FAF279728966FAF289729967FAF299720
:103C90009C0140E050E060E070E080E090E008E0EF
:103CA0000E94BB880E9474883901B42FA52FF62F7B
:103CB000E72F8C019401A50160E070E080E090E0C6
:103CC0005301CB2EDA2EEF2EFE2E0E94F2882CA36B
:103CD0003BA34B83252E362E472E582E792E632D4F
:103CE000742D852D972D315041095F4F6F4F7F4FB8
:103CF0008F4F9F4F88248394912C21153F4F4F4F16
:103D00005140610571058105910509F010F4812C80
:103D1000912C9A8289820091320A1091330A5801BB
:103D2000C12CD12CE12CF12C00E010E02CA13BA106
:103D30004B81522D632D742D852D972D0E94608708
:103D4000F22E032F142FB52FF62FE72FD82EE92EA2
:103D5000A0E00E94198984F42150310940485F4F46
:103D60006F4F7F4F8F4F9F4FF22E032F142FB52F82
:103D7000F62FE72FD82EE92E2F2D302F412F5B2F36
:103D80006F2F7E2F8D2D9E2D07E10E94D4882B8FC3
:103D90003C8F4D8F5E8F6F8F78A389A39AA320539A
:103DA000384F4F4F5F4F6F4F7F4F8F4F9F4F2B8B32
:103DB0003C8B4D8B5E8B6F8B788F898F9A8F2056C3
:103DC000304F4F4F5F4F6F4F7F4F8F4F9F4F243D6F
:103DD000304341055105610571058105910529F0C3
:103DE00020F0F4013196FA83E98380903A0A9090AA
:103DF0003B0A940140E050E060E070E080E090E039
:103E000000E10E94BB882C833D834E835F83662E36
:103E100078874C014091360A5091370AACA0BBA07C
:103E2000CB80D22CE32CF42C052D172D9A0140E0E9
:103E300050E060E070E080E090E00E946087F22E49
:103E4000032F142FB52FF62FE72FD82EE92EA0E041
:103E50000E9419895CF4AFE70E94FB88F22E032FC1
:103E6000142FB52FF62FE72FD82EE92E2F2D302F18
:103E7000412F5B2F6F2F7E2F8D2D9E2D07E00E94EF
:103E8000D48859016A017B018C012C813D814E81CE
:103E90005F81662D7885C4010E94F2882C833D8362
:103EA0004E835F8368877E878F87988B2E5F3F4F17
:103EB000434051096E4F7F4F8F4F9F4F2230310546
:103EC000494F5F4F644071058105910539F030F02D
:103ED00009811A810F5F1F4F1A83098360913C0A81
:103EE00070913D0A80E090E020E030E840E050E052
:103EF0000E94B98729873A874B875C87662E7D8722
:103F00004C014091380A5091390AACA0BBA0CB803B
:103F1000D22CE32CF42C052D172D9A0140E050E013
:103F200060E070E080E090E00E946087F22E032F56
:103F3000142FB52FF62FE72FD82EE92EA0E00E94E0
:103F4000198984F421503F4F4F4F5F4F6F4F7F4F80
:103F50008F4F9F4FF22E032F142FB52FF62FE72FE1
:103F6000D82EE92E2F2D302F412F5B2F6F2F7E2F34
:103F70008D2D9E2D08E00E94D48859016A017B0195
:103F80008C0129853A854B855C85662D7D85C4012C
:103F90000E94F28829873A874B875C876D87798BE7
:103FA0008A8B692E2F5F3F4F41405109610971098A
:103FB00081099109213030484C4F5F4761407105BC
:103FC0008105910539F030F029813A812F5F3F4F0B
:103FD0003A8329832B893C894D895E896F89788D45
:103FE000898D9A8D2F3C374041055105610571053A
:103FF0008105910511F00CF0A4C1ACA0BBA0CB8051
:10400000D22CE32CF42C052D172D95014C2D522D7F
:10401000632D742D852D972D0E946087A12CB12CC6
:10402000C12CE0E8DE2EE12CF12C00E010E00E9433
:10403000E68729AF3AAF4BAF5CAF6DAF7EAF8FAFC6
:1040400021969FAF2197AB8CBC8CCD8CDE8CEF8CF6
:10405000F8A009A11AA19501A601B701C8010E9403
:10406000608759016A017B01E82F192F02E00E9445
:10407000BB880E2F0E94F2887901142F552EF62F3F
:10408000E72F6C01922EAF2CB42E052F462EB72FA2
:10409000782E8D2CA0E00E9419895CF4A1E00E948A
:1040A000FB88922EA32EB42E052F462EB72F782EE6
:1040B000892E292D3A2D4B2D502F642D7B2F872DA6
:1040C000982D01E00E94D4882AA7732E4A012C96CD
:1040D0006FAF2C972B967FAF2B978BA79CA72B832B
:1040E0003BA34CA39DA26EA37FA388A799A7B52D40
:1040F0009701412F552D6F2F7E2FC601A0E00E9402
:1041000019894CF4A3E00E94FB887901142FB52F84
:10411000F62FE72F6C019701412F5B2F6F2F7E2F1A
:10412000C60102E00E94D4882DA73EA74FA758AB36
:1041300069AB7AAB8BAB9CAB2901B42FA52F229630
:104140006FAF2297F72F1C012B893C894D895E891F
:104150006F89788D898D9A8D24323A4F4F4F5F4FFA
:104160006F4F7F4F8F4F9F4F0CF08BC02B8D3C8D2F
:104170004D8D5E8D6F8D78A189A19AA12455324F06
:104180004F4F5F4F6F4F7F4F8F4F9F4F59016A01C6
:104190007B018C010E94608719012A01B62FA72F8D
:1041A000FC0103E00E94BB8851016201EB2EFA2E54
:1041B0008F010E94078959016A017B018C012AA5A0
:1041C000372DA4012C966FAD2C972B967FAD2B9796
:1041D0008BA59CA50E94F2882B833BA34CA35DA3D7
:1041E0006EA37FA388A799A79101A2016B2F7A2FB5
:1041F000CF0102E00E94BB8851016201EB2EFA2E32
:104200008F010E94078902E00E94BB880E2F0E9446
:104210000789122FD32EE42EB52FF62FE72FF82E75
:10422000092FA0E00E9419895CF4A1E00E94FB889C
:10423000122FD32EE42EB52FF62FE72FF82E092FAD
:10424000212F3D2D4E2D5B2F6F2F7E2F8F2D902FE9
:1042500001E00E94D48859016A017B018C012DA5DF
:104260003EA54FA558A969A97AA98BA99CA90E9426
:10427000F2882901B42FA52F22966FAF2297F72F2E
:104280001C012C813D814E815F8168857E858F85F3
:104290009889AB80BBA0CCA0DDA0EEA0FFA008A5B4
:1042A00019A50E9407892C833D834E835F8368870D
:1042B0007E878F87988B29853A854B855C856D85B0
:1042C00079898A89962D5201CB2EDA2E2296EFAC6F
:1042D0002297FF2E81010E94078929873A874B8701
:1042E0005C876D87798B8A8B692E2B893C894D89F8
:1042F0005E896F89788D898D9A8DA9ACBAACCBAC6B
:10430000DCACEDACFEAC0FAD21961FAD21970E9449
:1043100007892056304F4F4F5F4F6F4F7F4F8F4F62
:104320009F4F243D304341055105610571058105CD
:10433000910539F030F009811A810F5F1F4F1A8300
:1043400009834DA95EA96FA978AD9A01AB0160E020
:1043500070E0CB0122962FAF229723963FAF239791
:1043600024964FAF249725965FAF259726966FAF7B
:10437000269727967FAF279728968FAF289729965D
:104380009FAF2997A984BA84CB84DC84ED84F98813
:104390000A89162D60E070E080E090E00E9460875E
:1043A000122FD32EE42EB52FF62FE72FF82E092F3C
:1043B000A0E00E94198984F421503109404E5F4FDA
:1043C0006F4F7F4F8F4F9F4F122FD32EE42EB52F5D
:1043D000F62FE72FF82E092F212F3D2D4E2D5B2F85
:1043E0006F2F7E2F8F2D902F05E10E94D488AC80F7
:1043F000BD80CE80DF80E884FE840F8518890E940E
:104400000789122FD32EE42EB52FF62FE72FF82E83
:10441000092FA0E00E94198984F4215030484F4FA1
:104420005F4F6F4F7F4F8F4F9F4F122FD32EE42E32
:10443000B52FF62FE72FF82E092F212F3D2D4E2DCA
:104440005B2F6F2F7E2F8F2D902F0FE00E94D4882F
:1044500039014A015B016C0179018A011B012C01C0
:10446000285E3340410951096109710981099109A7
:10447000283D304D4140510561057105810591058B
:1044800031F028F0E981FA813196FA83E9830E94BC
:104490006D5F29813A81232B51F09301A401B5016D
:1044A000C6010E94748879018A011B012C019701C1
:1044B000A801B101C2010E94B58A20E030E048ECB9
:1044C00052E40E94098AC55BDF4F0FB6F894DEBF45
:1044D0000FBECDBFDF91CF911F910F91FF90EF9055
:1044E000DF90CF90BF90AF909F908F907F906F9014
:1044F0005F904F903F902F9008954F925F926F92F0
:104500007F928F929F92AF92BF92CF92DF92EF9263
:10451000FF922B013C0169017A0123EC35EF4CE855
:1045200051E4C701B6010E94B58C4B015C0128EB38
:104530003EE143E753E4C701B6010E9426899B018F
:10454000AC01C501B4010E94098A0E94838A4B0113
:104550005C0120E030E048EC52E4C301B2010E946B
:10456000098A21E835E943EC50E40E94B58CA501A5
:1045700094010E94B58C4B015C0123E333E948E8C8
:1045800053E4C701B6010E9426899B01AC01C50115
:10459000B4010E94098A23E333EB48E553E40E9407
:1045A000B58CFF90EF90DF90CF90BF90AF909F9031
:1045B0008F907F906F905F904F9008954F925F9291
:1045C0006F927F928F929F92AF92BF92CF92DF9223
:1045D000EF92FF9269017A010E94298C20E030E07D
:1045E00040E050E40E94258922E93CE54EED5EE37F
:1045F0000E94098A4B015C0123EC35EF4CE851E441
:10460000C701B6010E94B58C2B013C0128EB3EE1AD
:1046100043E753E4C701B6010E9426899B01AC0120
:10462000C301B2010E94098A9B01AC01C501B4011A
:104630000E9426896B017C0128EB3EE143E753E4AD
:104640000E94B58C4B015C01A701960163EC75EFEC
:104650008CE891E40E9425899B01AC01C501B4015D
:104660000E94098AFF90EF90DF90CF90BF90AF90AB
:104670009F908F907F906F905F904F9008954F9292
:104680005F926F927F928F929F92AF92BF92CF92E2
:10469000DF92EF92FF922B013C0169017A0123EC3A
:1046A00035EF4CE851E4C701B6010E94B58C4B01CF
:1046B0005C0128EB3EE143E753E4C701B6010E94E9
:1046C00026899B01AC01C501B4010E94098A0E94A0
:1046D000838A4B015C0120E030E048EC52E4C301E6
:1046E000B2010E94098AA50194010E94B58C20E0C4
:1046F00030E040E251E40E94258924EE38E34EE0A8
:104700005FE30E94B58C9B01AC01C701B6010E941A
:104710002689FF90EF90DF90CF90BF90AF909F9051
:104720008F907F906F905F904F90089580E80E94E7
:104730006B5F81110DC08EEF0E94755F811108C003
:1047400066E37CE980E090E00E94E75E0C946D5F98
:104750000E946D5F8091C1309091C230A091C330B2
:10476000B091C4300196A11DB11D8093C1309093CA
:10477000C230A093C330B093C4300895FC01DC0173
:10478000AC014E5F5F4F90E031E38D91982788E058
:10479000292F220F97FF03C0922F932701C0922F3A
:1047A0008150B1F7A417B50781F721E030E082818D
:1047B000981711F020E030E0C9010895DF92EF92E0
:1047C000FF920F931F93CF93DF930E94962380E86D
:1047D0000E946B5F81116DC08AEF0E94755F81112D
:1047E00068C08FE00E94755F811163C06AE67AE05D
:1047F00080E090E00E94E75E81E80E946B5F81119B
:1048000058C00E94865FD82F0E94865F0E94865FF4
:10481000182F0E94865F0E94865F082F0E94865F85
:104820000E94905FF82E80E80E946B5F811141C06A
:104830008CEF0E94755F81113CC089EC0E94755F0E
:10484000811137C06AE67AE080E090E00E94E75E7E
:1048500081E80E946B5F0E94865FE82E0E94865F5F
:10486000D82E0E94865F0E94865FC82F0E94905FAC
:104870001F92DF921F92EF921F92FF921F920F934F
:104880001F921F931F92DF931F928F931F92CF93BC
:1048900082EA93E09F938F930E9423920E946D5F20
:1048A0008DB79EB742960FB6F8949EBF0FBE8DBFD0
:1048B00017C00E946D5F8091C1309091C230A0916D
:1048C000C330B091C4300196A11DB11D8093C13099
:1048D0009093C230A093C330B093C4300E9496230B
:1048E00020E030E040E050E060E070E080E090E008
:1048F000DF91CF911F910F91FF90EF90DF9008957E
:10490000EF92FF920F931F93CF93DF9300D0CDB719
:10491000DEB78C0180E80E946B5F811154C00115E5
:10492000110551F085EE0E94755F81114CC062E067
:104930007EE281E090E009C083EE0E94755F811104
:1049400042C062E375E783E090E00E94E75E81E8A1
:104950000E946B5F811137C00E94865FE82E8983B9
:104960000E94865FF82E8A830E94905F8B830E944C
:104970006D5FCE0101960E94BE23892B21F16F2D20
:1049800070E07E296C7F80E090E0012B69F00E944E
:10499000BB8A20E030E04AEF5AE30E94B58C20E069
:1049A00030E040EC50E40CC00E94BB8A22E538EBBA
:1049B0004FE25BE30E94B58C26E636E64BE352E419
:1049C0000E9425891BC00E946D5F8091C13090912B
:1049D000C230A091C330B091C4300196A11DB11D69
:1049E0008093C1309093C230A093C330B093C43051
:1049F0000E94962360EF7FEF89E794E40F900F9079
:104A00000F90DF91CF911F910F91FF90EF9008953C
:104A10000F931F93CF93DF93729A8091660283FF67
:104A200008C08EE40E94095F811165C0C0E5D0E036
:104A300009C0C0E5D0E08FED97E00E942D0E2197D0
:104A4000D1F7EFCF8FED97E00E942D0E2197D1F790
:104A50008FE40E94095F0E94865FD82FDF730E9457
:104A6000865F082F0E94865FC82F0E94905F182FD4
:104A70000E946D5F8091660283FF72986D2F70E0D7
:104A8000762F6627600F711D80E090E00E94BB8A40
:104A900020E134E048EC5BE30E94B58C6093A328EE
:104AA0007093A4288093A5289093A6286C2F70E07B
:104AB000762F6627610F711D7695679576956795B8
:104AC00080E090E00E94BB8A24EA3CEF44E25CE391
:104AD0000E94B58C20E030E040E252E40E9425893B
:104AE00060938435709385358093863590938735B0
:104AF00080E090E002C081E090E0DF91CF911F91D3
:104B00000F9108957298729A8EE40E94095F80EA6C
:104B10000E94755F80E00E94755F80E00E94755F73
:104B20008FE40E94095F0E94865F8EE40E94095F05
:104B300080E80E94755F80E00E94755F80E00E94BF
:104B4000755F0E946D5F80E090E0089587EC90E1D2
:104B50009F938F930E943792809180020F900F90C5
:104B6000882361F01F928F9384EC90E19F938F9341
:104B70000E9437920F900F900F900F9008958FE939
:104B800090E19F938F930E94379287E790E19F93E4
:104B90008F930E94379280E590E19F938F930E94BC
:104BA000379285E190E19F938F930E94379289ED30
:104BB0009FE09F938F930E94379287EA9FE09F9395
:104BC0008F930E9437928BE69FE09F938F930E9472
:104BD000379285E49FE09F938F930E9437928FE0F6
:104BE0009FE09F938F930E9437928091AF2C90917A
:104BF000B02C827091702DB73EB72E5E3F4F0FB62E
:104C0000F8943EBF0FBE2DBF892B41F08FED9EE083
:104C10009F938F930E9437920F900F9083EB9EE0AB
:104C20009F938F930E94379287E79EE09F938F9385
:104C30000E9437928EE49EE09F938F930E9437925A
:104C400082E29EE09F938F930E94379283EF9DE0D4
:104C50009F938F930E94379281EC9DE09F938F9357
:104C60000E94379280E99DE09F938F930E94379234
:104C700086E59DE09F938F930E94379280E29DE0AE
:104C80009F938F930E94379280EF9CE09F938F9326
:104C90000E94379284EC9CE09F938F930E943792FE
:104CA00085E99CE09F938F930E9437928CE59CE06E
:104CB0009F938F930E94379283E29CE09F938F9300
:104CC0000E9437928CEE9BE09F938F930E943792C5
:104CD0008EEB9BE09F938F930E9437928DB79EB788
:104CE00080960FB6F8949EBF0FBE8DBF8AE89BE0FA
:104CF0009F938F930E94379289E59BE09F938F93B8
:104D00000E9437928AE29BE09F938F930E94379292
:104D10008BEF9AE09F938F930E94379284ED9AE0F5
:104D20009F938F930E9437928EE99AE09F938F937F
:104D30000E94379288E69AE09F938F930E94379261
:104D400082E39AE09F938F930E94379289E09AE0E2
:104D50009F938F930E94379281ED99E09F938F9359
:104D60000E94379286EA99E09F938F930E94379230
:104D70002DB73EB72A5E3F4F0FB6F8943EBF0FBE29
:104D80002DBF089581ED93E00C945F924F925F9256
:104D90006F927F928F929F92AF92BF92CF92DF924B
:104DA000EF92FF92CF93DF93CDB7DEB728970FB680
:104DB000F894DEBF0FBECDBF8091B5309091B63074
:104DC000A091B730B091B83089839A83AB83BC830C
:104DD0004090B5305090B6306090B7307090B83099
:104DE0008091B5309091B630A091B730B091B83085
:104DF0008D839E83AF83B8876091B5307091B63054
:104E00008091B7309091B8302CE3822E912CA12C58
:104E1000B12CA50194010E94E6867F936F9330E147
:104E2000C32E3EE0D32EE12CF12C6D817E818F814B
:104E30009885A70196010E94E686A50194010E942B
:104E4000E6863F932F9340E8842E41E5942EAA24D2
:104E5000A394B12CC301B201A50194010E94E6867E
:104E6000A70196010E94E6863F932F9369817A817C
:104E70008B819C81A50194010E94E6863F932F932C
:104E800080E899E09F938F930E9437920FB6F89431
:104E9000DEBF0FBECDBF28960FB6F894DEBF0FBEA3
:104EA000CDBFDF91CF91FF90EF90DF90CF90BF907B
:104EB000AF909F908F907F906F905F904F900895EC
:104EC000E7EEF9E3808191818234924479F0E75EE4
:104ED000F943FF93EF9382E699E09F938F930E94AB
:104EE00037920F900F900F900F9008953A96E53FEC
:104EF00081E8F80738F30895CF93DF93EC018C9A9B
:104F00000E949F109F938F937F936F9386E599E004
:104F10009F938F930E9437920F900F900F900F9056
:104F20000F900F90209719F00E94B01108C084E5EF
:104F300099E09F938F930E9437920F900F9081E09A
:104F40000E94511020918502309186024091870283
:104F5000509188020E94B58C9F938F937F936F939B
:104F600088E499E09F938F930E9437920F900F905F
:104F70000F900F900F900F90209719F00E94B01192
:104F800008C086E499E09F938F930E9437920F9018
:104F90000F9082E00E945110209181023091820294
:104FA00040918302509184020E94B58C9F938F930D
:104FB0007F936F938AE399E09F938F930E94379238
:104FC0000F900F900F900F900F900F90209719F067
:104FD0000E94B01108C088E399E09F938F930E94CC
:104FE00037920F900F9083E00E9451109F938F9300
:104FF0007F936F9389E299E09F938F930E943792FA
:105000008C980F900F900F900F900F900F9020970B
:1050100019F00E94B01108C087E299E09F938F9326
:105020000E9437920F900F908091AF2C87FF83C022
:1050300021E042E161E080ED0E94CD609F938F937B
:105040007F936F938AE199E09F938F930E943792A9
:105050000F900F900F900F900F900F90209719F0D6
:105060000E94B01108C088E199E09F938F930E943D
:1050700037920F900F9021E042E162E080ED0E94B4
:10508000CD609F938F937F936F938BE099E09F9375
:105090008F930E9437920F900F900F900F900F9068
:1050A0000F90209719F00E94B01108C089E099E094
:1050B0009F938F930E9437920F900F9021E042E1CF
:1050C00063E080ED0E94CD609F938F937F936F93F9
:1050D0008CEF98E09F938F930E9437920F900F90E0
:1050E0000F900F900F900F90CD2B19F00E94B011E0
:1050F00008C08AEF98E09F938F930E9437920F9099
:105100000F9021E042E164E080ED0E94CD609F932A
:105110008F937F936F938DEE98E09F938F930E9470
:1051200037920F900F900F900F900F900F90DF918C
:10513000CF910C94B011CD2BD1F3DF91CF91089585
:105140000F931F93CF93DF93882389F049E050E0BA
:105150006FEF70E088E795E30E94719149E050E0BD
:105160006EE070E088E795E30E94029513C0C8E7FF
:10517000D5E308EE18E089911F928F931F930F9348
:105180000E9437920F900F900F900F9085E3C038D8
:10519000D80789F7DF91CF911F910F910C94B0112F
:1051A000882311F0299A089529980895882311F0E9
:1051B0002A9A08952A980895CF93DF9360917E02EA
:1051C00070917F0280E090E00E945791EC016EE0C8
:1051D00074E00E947891892B99F4809166029091F5
:1051E0006702A0916802B0916902A4608093660290
:1051F00090936702A0936802B09369022A9A1BC039
:1052000061E174E0CE010E947891892BF1F48091E4
:10521000660290916702A0916802B0916902AB7F2B
:105220008093660290936702A0936802B09369022C
:1052300080E00E94D62844E050E06EE170E086E60F
:1052400092E0DF91CF910C9402952A9903C081E1FD
:1052500094E002C08EE094E09F938F938BE594E0FE
:105260009F938F930E9437920F900F900F900F9003
:10527000DF91CF910895CF92DF92EF92FF92CF937B
:10528000DF936B017C0160FF11C085E194E09F9387
:105290008F938CED90E19F938F930E9437920F90A4
:1052A0000F900F900F9081E090E002C080E090E0BE
:1052B000C1FE09C0EC01219643E159E06AE174E0C6
:1052C0000E941916CE01C2FE09C0EC01219643E1ED
:1052D00059E062E274E00E941916CE01C3FE09C0D3
:1052E000EC01219643E159E06AE274E00E9419164C
:1052F000CE01C4FE09C0EC01219643E159E06EE8FD
:1053000075E00E941916CE01C5FE09C0EC01219678
:1053100043E159E06EE274E00E941916CE01C6FE28
:1053200009C0EC01219643E159E062E374E00E9478
:105330001916CE01C7FE09C0EC01219643E159E0E0
:1053400068E374E00E941916CE01D0FE09C0EC019A
:10535000219643E159E060E474E00E941916CE0101
:10536000D1FE09C0EC01219643E159E068E474E004
:105370000E941916CE01D2FE09C0EC01219643E12C
:1053800059E06CE474E00E941916CE012091AF2C14
:105390003091B02C24703270232B59F0D3FE09C009
:1053A000EC01219643E159E062E574E00E94191690
:1053B000CE012091AF2C23FF0BC0D4FE09C0EC011D
:1053C000219643E159E067E574E00E941916CE0189
:1053D0002091AF2C24FF0BC0D5FE09C0EC01219613
:1053E00043E159E06DE574E00E941916CE01D6FE46
:1053F00009C0EC01219643E159E065E674E00E94A2
:105400001916CE01D7FE09C0EC01219643E159E0FF
:1054100060E774E00E941916CE01E0FE0CC043E183
:1054200059E061E874E0DF91CF91FF90EF90DF9059
:10543000CF900C941916CD28CE28CF2841F483EEB6
:1054400098E09F938F930E9437920F900F90DF9177
:10545000CF91FF90EF90DF90CF900895CF92DF92A1
:10546000EF92FF92CF93DF93EC01C12CD12C760108
:10547000209709F4A3C06EED78E0CE010E9443911D
:10548000892B11F46894C0F866ED78E0CE010E9493
:105490004391892B11F46894C1F86EEC78E0CE0149
:1054A0000E944391892B11F46894C2F86AEC78E069
:1054B000CE010E944391892B11F46894C3F867ECE4
:1054C00078E0CE010E944391892B11F46894C4F8CE
:1054D00063EC78E0CE010E944391892B11F468942B
:1054E000C5F86DEB78E0CE010E944391892B11F451
:1054F0006894C6F865EB78E0CE010E944391892B51
:1055000011F46894C7F86DEA78E0CE010E944391E7
:10551000892B11F46894D0F869EA78E0CE010E94F2
:105520004391892B11F46894D1F863EA78E0CE01B5
:105530000E944391892B11F46894D2F86EE978E0C7
:10554000CE010E944391892B11F46894D3F868E945
:1055500078E0CE010E944391892B11F46894D4F82D
:1055600060E978E0CE010E944391892B11F46894A0
:10557000D5F865E878E0CE010E944391892B11F4BB
:105580006894D6F864E778E0CE010E944391892BB5
:1055900011F46894D7F86FE678E0CE010E94439149
:1055A000892B11F46894E0F860917E0270917F027B
:1055B00080E090E00E945791EC015ACFC701B601FC
:1055C000DF91CF91FF90EF90DF90CF900895AF9251
:1055D000BF92CF92DF92EF92FF920F931F93CF93E0
:1055E000DF93122FD32FC42F052FF62EC72ED82EC0
:1055F000E92E217030E040E050E060E070E080E0B3
:1056000090E0A0E00E94198989F086E894E09F93D9
:105610008F938CED90E19F938F930E9437920F9020
:105620000F900F900F90E1E0F0E002C0E0E0F0E0BA
:105630008091AF2C80FF19C0212F247030E040E012
:1056400050E060E070E080E090E0A0E00E94198906
:1056500061F05F018FEFA81AB80A43E159E06AE8E8
:1056600074E0CF010E941916F501212F227030E05D
:1056700040E050E060E070E080E090E0A0E00E9458
:10568000198961F05F018FEFA81AB80A43E159E068
:105690006EE874E0CF010E941916F501212F2870E1
:1056A00030E040E050E060E070E080E090E0A0E0BA
:1056B0000E94198961F05F018FEFA81AB80A43E1CF
:1056C00059E066EA74E0CF010E941916F501212F16
:1056D000207130E040E050E060E070E080E090E079
:1056E000A0E00E94198961F05F018FEFA81AB80A43
:1056F00043E159E061E974E0CF010E941916F50118
:10570000212F207230E040E050E060E070E080E067
:1057100090E0A0E00E94198961F05F018FEFA81A64
:10572000B80A43E159E064E974E0CF010E94191618
:10573000F501212F207430E040E050E060E070E09F
:1057400080E090E0A0E00E94198961F05F018FEF96
:10575000A81AB80A43E159E06AE974E0CF010E944F
:105760001916F501212F207830E040E050E060E08C
:1057700070E080E090E0A0E00E94198961F05F0194
:105780008FEFA81AB80A43E159E060EA74E0CF014C
:105790000E941916F50120E03D2F317040E050E0E5
:1057A00060E070E080E090E0A0E00E94198961F084
:1057B0005F018FEFA81AB80A43E159E063EA74E089
:1057C000CF010E941916F50120E03D2F327040E014
:1057D00050E060E070E080E090E0A0E00E94198975
:1057E00061F05F018FEFA81AB80A43E159E068EA57
:1057F00074E0CF010E941916F50120E03D2F3470AE
:1058000040E050E060E070E080E090E0A0E00E94C6
:10581000198961F05F018FEFA81AB80A43E159E0D6
:105820006FEA74E0CF010E941916F50120E03D2FC8
:10583000387040E050E060E070E080E090E0A0E090
:105840000E94198961F05F018FEFA81AB80A43E13D
:1058500059E062EB74E0CF010E941916F50120E0D7
:105860003D2F307140E050E060E070E080E090E07B
:10587000A0E00E94198961F05F018FEFA81AB80AB1
:1058800043E159E067EB74E0CF010E941916F5017E
:1058900020E03D2F307240E050E060E070E080E0BA
:1058A00090E0A0E00E94198961F05F018FEFA81AD3
:1058B000B80A43E159E06EEB74E0CF010E9419167B
:1058C000F50120E030E040E050E06F2D647070E0C2
:1058D00080E090E0A0E00E94198961F05F018FEF05
:1058E000A81AB80A43E159E065EC74E0CF010E94C0
:1058F0001916F5018091AF2C81FF19C020E03D2FD2
:10590000307440E050E060E070E080E090E0A0E0C3
:105910000E94198961F05F018FEFA81AB80A43E16C
:1059200059E069EC74E0CF010E941916F5018091ED
:10593000AF2C9091B02C90FF19C020E030E040E0F7
:10594000502F507160E070E080E090E0A0E00E9495
:10595000198961F05F018FEFA81AB80A43E159E095
:105960006CEC74E0CF010E941916F5018091AF2C08
:105970009091B02C90FF19C020E030E040E0502F13
:10598000507260E070E080E090E0A0E00E94198931
:1059900061F05F018FEFA81AB80A43E159E06FEC9C
:1059A00074E0CF010E941916F5018091AF2C9091FF
:1059B000B02C90FF19C020E030E040E0502F507430
:1059C00060E070E080E090E0A0E00E94198961F062
:1059D0005F018FEFA81AB80A43E159E065ED74E062
:1059E000CF010E941916F50120E03D2F307840E0EC
:1059F00050E060E070E080E090E0A0E00E94198953
:105A000061F05F018FEFA81AB80A43E159E060EE38
:105A100074E0CF010E941916F50120E030E04C2F10
:105A2000417050E060E070E080E090E0A0E00E9413
:105A3000198961F05F018FEFA81AB80A43E159E0B4
:105A400065EE74E0CF010E941916F50120E030E008
:105A50004C2F427050E060E070E080E090E0A0E009
:105A60000E94198961F05F018FEFA81AB80A43E11B
:105A700059E068EE74E0CF010E941916F50120E0AC
:105A800030E04C2F447050E060E070E080E090E047
:105A9000A0E00E94198961F05F018FEFA81AB80A8F
:105AA00043E159E06BEE74E0CF010E941916F50155
:105AB0008091AF2C87FF19C020E030E04C2F487058
:105AC00050E060E070E080E090E0A0E00E94198982
:105AD00061F05F018FEFA81AB80A43E159E06EEE5A
:105AE00074E0CF010E941916F5018091AF2C87FF59
:105AF00019C020E030E04C2F407150E060E070E0D1
:105B000080E090E0A0E00E94198961F05F018FEFD2
:105B1000A81AB80A43E159E062EF74E0CF010E948D
:105B20001916F5018091AF2C87FF19C020E030E0F5
:105B30004C2F407250E060E070E080E090E0A0E028
:105B40000E94198961F05F018FEFA81AB80A43E13A
:105B500059E066EF74E0CF010E941916F5018091BB
:105B6000AF2C87FF19C020E030E04C2F407450E08C
:105B700060E070E080E090E0A0E00E94198961F0B0
:105B80005F018FEFA81AB80A43E159E06AEF74E0A9
:105B9000CF010E941916F5018091AF2C82FF19C028
:105BA00020E030E04C2F407850E060E070E080E092
:105BB00090E0A0E00E94198961F05F018FEFA81AC0
:105BC000B80A43E159E061E276E0CF010E9419167C
:105BD000F5018091AF2C82FF19C020E030E040E059
:105BE000502F517060E070E080E090E0A0E00E94F3
:105BF000198961F05F018FEFA81AB80A43E159E0F3
:105C00006EEF74E0CF010E941916F5018091AF2C60
:105C10009091B02C90FF19C020E030E040E0502F70
:105C2000527060E070E080E090E0A0E00E9419898E
:105C300061F05F018FEFA81AB80A43E159E061E013
:105C400075E0CF010E941916F5018091AF2C90915B
:105C5000B02C90FF19C020E030E040E0502F54708D
:105C600060E070E080E090E0A0E00E94198961F0BF
:105C70005F018FEFA81AB80A43E159E069E075E0C7
:105C8000CF010E941916F5018091AF2C9091B02C94
:105C900091FF1EC020E030E040E0502F587060E0DF
:105CA00070E080E090E0A0E00E94198989F043E173
:105CB00059E062E175E0CF01DF91CF911F910F9123
:105CC000FF90EF90DF90CF90BF90AF900C9419169B
:105CD000212F3D2F4C2F502F6F2D7C2D8D2D9E2D44
:105CE000A0E00E94198941F48AE698E09F938F937F
:105CF0000E9437920F900F90DF91CF911F910F91DB
:105D0000FF90EF90DF90CF90BF90AF900895AF924B
:105D1000BF92DF92EF92FF920F931F93CF93DF9387
:105D2000EC015B01FB01108265E678E00E94439183
:105D3000892B59F58091AF2C3DE4F32E00E882FFCA
:105D400003C024E8E22E02C094E0E92E10E0D12C3A
:105D500081FD00EC26E04AE250E06BE270E089E26F
:105D600090E00E94B05C81E090E00E94481188239E
:105D700011F08DE5F82E8091AF2C9091B02C90FD14
:105D800016E091FF07C0186005C0F12C00E0E12C7F
:105D900010E0D12C63E678E0CE010E944391892B7C
:105DA00061F481E0F501808360917E0270917F0251
:105DB00080E090E00E945791EC0161E678E0CE012E
:105DC0000E944391892B61F48FEFF50180836091EC
:105DD0007E0270917F0280E090E00E945791EC017A
:105DE000209709F424C16DE578E0CE010E9443912B
:105DF000892B19F4FF2DF160FF2E69E578E0CE01C3
:105E00000E944391892B19F48F2D8460F82E66E54A
:105E100078E0CE010E944391892B19F4EF2DE260C6
:105E2000FE2E64E578E0CE010E944391892B19F49F
:105E3000FF2DF860FF2E61E578E0CE010E944391CE
:105E4000892B19F48F2D8061F82E6BE478E0CE0158
:105E50000E944391892B19F4EF2DE062FE2E65E438
:105E600078E0CE010E944391892B19F4FF2DF06454
:105E7000FF2E62E478E0CE010E944391892B19F451
:105E80008F2D8068F82E6DE378E0CE010E9443915B
:105E9000892B09F4016066E378E0CE010E9443910A
:105EA000892B09F4026063E378E0CE010E944391FC
:105EB000892B09F404606EE278E0CE010E944391E0
:105EC000892B09F4086067E278E0CE010E944391D3
:105ED000892B09F4006160E278E0CE010E944391D1
:105EE000892B09F400626CE178E0CE010E944391B5
:105EF000892B19F4ED2DE460DE2E69E178E0CE0106
:105F00000E944391892B09F4006464E178E0CE019A
:105F10000E944391892B09F4006861E178E0CE0189
:105F20000E944391892B19F4FE2DF160EF2E6EE053
:105F300078E0CE010E944391892B19F48E2D826066
:105F4000E82E6BE078E0CE010E944391892B19F492
:105F5000EE2DE460EE2E67E078E0CE010E944391E2
:105F6000892B19F4FE2DF860EF2E63E078E0CE0166
:105F70000E944391892B19F48E2D8061E82E6FEFDA
:105F800077E0CE010E944391892B19F4EE2DE06257
:105F9000EE2E6BEF77E0CE010E944391892B19F42E
:105FA000FE2DF064EF2E69EF77E0CE010E94439161
:105FB000892B19F48E2D8068E82E66EF77E0CE01EC
:105FC0000E944391892B09F411606EEE77E0CE01B7
:105FD0000E944391892B09F4126065EE77E0CE01AF
:105FE0000E944391892B09F414606CED77E0CE0197
:105FF0000E944391892B09F4186069ED77E0CE0186
:106000000E944391892B09F4106163ED77E0CE0182
:106010000E944391892B09F4106268EC77E0CE016D
:106020000E944391892B09F0D2CE1064D0CE2F2D3F
:10603000302F4E2D512F6D2D70E080E090E0DF91DC
:10604000CF911F910F91FF90EF90DF90BF90AF9095
:1060500008955F926F927F928F929F92AF92BF92BC
:10606000CF92DF92EF92FF920F931F93CF93DF9324
:10607000782EC2E9DCE100E010E082ECE82E87E057
:10608000F82E872D8170582E872D8270682E9DEAFC
:10609000C92E97E0D92E25EBA22E27E0B22E33EBA6
:1060A000832E37E0932E772051F01F930F93FF92AA
:1060B000EF920E9437920F900F900F900F90552003
:1060C000A1F089858F9388858F93BF92AF920E94AC
:1060D00037920F900F900F900F906620C1F09F9213
:1060E0008F920E9437920F900F90662081F0DF927E
:1060F000CF920E943792288139814A815B816C81DD
:106100007D818E819F810E94E72A0F900F900E94CF
:10611000B0110F5F1F4F2A960430110521F6DF9151
:10612000CF911F910F91FF90EF90DF90CF90BF9094
:10613000AF909F908F907F906F905F90089588EAC6
:1061400097E09F938F930E94379280919F28909120
:10615000A028A091A128B091A2280F900F90813083
:1061600027EA92072EE1A207B10519F48AE997E020
:106170001DC0823026EA92072EE1A207B10519F46C
:106180008DE897E013C0823027EA92072EE1A2073C
:10619000B10519F48FE797E009C0823028EA920729
:1061A0002EE1A207B10549F481E797E09F938F9311
:1061B0000E9437920F900F900895BF93AF939F93D3
:1061C0008F938BE697E09F938F930E9437920F9067
:1061D0000F900F900F900F900F9008958BE597E020
:1061E0009F938F930E9437920E94C2260E949F30F5
:1061F0000E94B01189E79CE19F938F9383E597E01C
:106200009F938F930E943792609160027091610218
:10621000809162029091630228EE33E040E050E00A
:106220000E94E6865F934F933F932F9383E497E01A
:106230009F938F930E9437928AE397E09F938F9367
:106240000E9437920E9442168091AF2C2DB73EB724
:10625000225F3F4F0FB6F8943EBF0FBE2DBF80FFA9
:1062600005C041E061E081E00E94EF1786E397E01E
:106270009F938F930E94379280E00E94A0280E94F3
:10628000C626809165021F928F938DE297E09F93BF
:106290008F930E943792809186131F928F9384E28E
:1062A00097E09F938F930E943792809190028F93F3
:1062B00080918F028F9380918E028F9380918D02B7
:1062C0008F9386E197E09F938F930E9437921F925E
:1062D00080E48F938EEF96E09F938F930E94379286
:1062E00080918E371F928F9380918D371F928F935D
:1062F0008BEE96E09F938F930E9437928091640279
:106300001F928F9382EE96E09F938F930E94379215
:106310008091660290916702A0916802B091690233
:106320002DB73EB7225E3F4F0FB6F8943EBF0FBE6B
:106330002DBF96FD03C081E194E002C08EE094E0A1
:106340009F938F9388ED96E09F938F930E9437924F
:1063500083E00E9429300F900F900F900F901D99AD
:1063600003C081E194E002C08EE094E09F938F939C
:106370008CEC96E09F938F930E94379282EC96E08C
:106380009F938F930E943792809166020F900F9097
:106390000F900F900F900F9081FF09C08CEB96E04B
:1063A0009F938F930E9437920F900F9013C080FDA0
:1063B00003C081E194E002C08EE094E09F938F934C
:1063C00088EB96E09F938F930E9437920F900F90E7
:1063D0000F900F908091660290916702A0916802E1
:1063E000B091690297FD03C081E194E002C08EE0A4
:1063F00094E09F938F938FEA96E09F938F930E94F0
:10640000379288EA96E09F938F930E94379260912B
:10641000891370918A1380918B1390918C130E9431
:106420003B290E94B0110F900F900F900F900F908A
:106430000F90779B03C081E194E002C08EE094E06E
:106440009F938F938FE996E09F938F930E9437924B
:106450000E94330E0E9404119F938F937F936F933A
:1064600081E996E09F938F930E9437920E94B31028
:106470009F938F937F936F9383E896E09F938F937F
:106480000E94379281E090E00E947C2780915E35E7
:1064900090915F35A0916035B0916135BF93AF9316
:1064A0009F938F9385E796E09F938F930E943792F7
:1064B000809173358F93809172358F938091713570
:1064C0008F93809170358F9381E696E09F938F93A1
:1064D0000E9437928091623590916335A091643526
:1064E000B0916535BF93AF939F938F9383E596E00B
:1064F0009F938F930E9437928DB79EB782960FB667
:10650000F8949EBF0FBE8DBF809177358F93809199
:1065100076358F93809175358F93809174358F93F5
:106520008FE396E09F938F930E94379261E070E033
:1065300080E090E00E94B91161E070E081E090E0BD
:106540000E94B9110F900F900F900F900F900F9025
:10655000299903C081E194E002C08EE094E09F930A
:106560008F9387E396E09F938F930E9437920F90CB
:106570000F900F900F902A9903C081E194E002C020
:106580008EE094E09F938F938FE296E09F938F939A
:106590000E9437920F900F900F900F900895F894EB
:1065A00091E2E0E0F0E0909357008491E2E0F0E0C7
:1065B000909357002491E4E0F0E090935700E49129
:1065C00090E0A0E0B0E0BC0155274427822F90E086
:1065D000A0E0B0E0BA2FA92F982F8827840F951F2D
:1065E000A61FB71F8E0F911DA11DB11D80939F285F
:1065F0009093A028A093A128B093A22878940895FE
:10660000CF93DF93CDB7DEB761970FB6F894DEBFB7
:106610000FBECDBF48E250E062E270E082E99CE14B
:106620000E94E4942091921C3091931C4091941C00
:106630005091951C6091961C7091971C8091981CAC
:106640009091991CAFEF0E94198909F05DC08DE40B
:106650008093921C80E88093931C84E08093941C28
:106660001092951C1092961C1092971C1092981CD8
:106670001092991C8CE390E090939B1C80939A1C41
:1066800010929C1C10929D1C10929E1C10929F1C9C
:106690001092A01C1092A11C1092A21C1092A31C7C
:1066A0001092A51C1092A41C1092A61C1092A71C5C
:1066B0001092A81C1092A91C1092AA1C1092AB1C3C
:1066C0001092AC1C1092AD1C1092AF1C1092AE1C1C
:1066D0001092B01C1092B11C1092B21C1092B31CFC
:1066E0001092B41C1092B51C1092B61C1092B71CDC
:1066F0001092B91C1092B81C48E250E062E270E0BF
:1067000082E99CE10E94029544E050E06EE170E075
:10671000CE010B960E94E4948B859C85AD85BE8549
:106720008F3F2FEF9207A207B207A9F48AE090E407
:10673000A0E0B0E08093660290936702A0936802A5
:10674000B093690244E050E06EE170E086E692E0CA
:106750000E94029508C08093660290936702A093FE
:106760006802B09369028091660290916702A091DD
:106770006802B0916902A2FF02C02A9A03C080E0B9
:106780000E94D62844E050E06AE570E0CE010B9606
:106790000E94E4948B859C85AD85BE858F3F2FEF4D
:1067A0009207A207B20789F41092891310928A13F4
:1067B00010928B1310928C1344E050E06AE570E065
:1067C00089E893E10E94029508C080938913909311
:1067D0008A13A0938B13B0938C1349E050E06EE0C2
:1067E00070E088E795E30E94E4940E94E71244E099
:1067F00050E06EE470E0CE010B960E94E4948B852D
:106800009C85AD85BE8544E050E06EE470E08F3F2E
:106810009F4FAF4FBF4F29F485E892E00E94029549
:1068200004C085E892E00E94E49444E050E06AE409
:1068300070E0CE010B960E94E4948B859C85AD851B
:10684000BE8544E050E06AE470E08F3F9F4FAF4F59
:10685000BF4F29F481E892E00E94029504C081E8CC
:1068600092E00E94E49444E050E062E570E0CE01E2
:106870000B960E94E4948B859C85AD85BE8544E093
:1068800050E062E570E08F3F9F4FAF4FBF4F29F45C
:1068900089E892E00E94029504C089E892E00E9493
:1068A000E49441E050E06DE170E0CE0141960E9439
:1068B000E494898941E050E06DE170E08F3F29F474
:1068C00086E893E10E94029504C086E893E10E9465
:1068D000E49441E050E06CE170E0CE0141960E940A
:1068E000E494898941E050E06CE170E08F3F29F445
:1068F00085E692E00E94029504C085E692E00E943F
:10690000E49441E050E06BE170E0CE0141960E94DA
:10691000E494898941E050E06BE170E08F3F29F415
:1069200084E692E00E94029504C084E692E00E9410
:10693000E4944AE050E064E070E0CE0101960E94E9
:10694000E49489814AE050E064E070E08F3F29F4EC
:1069500089E79CE10E94029504C089E79CE10E94BE
:10696000E49444E050E066E570E0CE010B960E94AE
:10697000E4948B859C85AD85BE8544E050E066E55A
:1069800070E08F3F9F4FAF4FBF4F29F48DE892E0EB
:106990000E94029504C08DE892E00E94E49444E0D5
:1069A00050E067E170E0CE010B960E94E4948B8585
:1069B0009C85AD85BE8544E050E067E170E08F3F87
:1069C0009F4FAF4FBF4F29F480E692E00E9402959F
:1069D00004C080E692E00E94E49442E050E062E06D
:1069E00070E0CE010F960E94E4948F85988942E072
:1069F00050E062E070E08F3F910529F48FE793E16A
:106A00000E94029504C08FE793E10E94E49442E063
:106A100050E060E070E0CE010F960E94E4948F8514
:106A2000988942E050E060E070E08F3F910529F4E2
:106A30008DE793E10E94029504C08DE793E10E94E7
:106A4000E49461960FB6F894DEBF0FBECDBFDF9120
:106A5000CF910895CF92DF92EF92FF9260917E02E4
:106A600070917F0280E090E00E9457916BE175E0A9
:106A70000E947891892B09F03BC18DE48093921C90
:106A800080E88093931C84E08093941C1092951C62
:106A90001092961C1092971C1092981C1092991CA0
:106AA0008CE390E090939B1C80939A1C10929C1C0A
:106AB00010929D1C10929E1C10929F1C1092A01C64
:106AC0001092A11C1092A21C1092A31C1092A51C43
:106AD0001092A41C1092A61C1092A71C1092A81C25
:106AE0001092A91C1092AA1C1092AB1C1092AC1C04
:106AF0001092AD1C1092AF1C1092AE1C1092B01CE4
:106B00001092B11C1092B21C1092B31C1092B41CC3
:106B10001092B51C1092B61C1092B71C1092B91CA2
:106B20001092B81C48E250E062E270E082E99CE119
:106B30000E9402958AE090E4A0E0B0E080936602B3
:106B400090936702A0936802B093690244E050E01A
:106B50006EE170E086E692E00E9402951092891341
:106B600010928A1310928B1310928C1344E050E011
:106B70006AE570E089E893E10E94029582E2C82EFE
:106B8000DD24DA948CECE82E8BE3F82EC09285029B
:106B9000D0928602E0928702F092880244E050E0B0
:106BA0006EE470E085E892E00E940295C092810256
:106BB000D0928202E0928302F092840244E050E09C
:106BC0006AE470E081E892E00E94029587ED94E328
:106BD000AFEEBCE38093890290938A02A0938B026C
:106BE000B0938C0244E050E062E570E089E892E006
:106BF0000E9402958AE999E9A9E1B0E480938D02A7
:106C000090938E02A0938F02B093900244E050E0E4
:106C100066E570E08DE892E00E940295109286137E
:106C200080E00E94226941E050E06DE170E086E87A
:106C300093E10E9402958AE1809365020E94FB67BE
:106C400041E050E06CE170E085E692E00E94029540
:106C50008FE08093640241E050E06BE170E084E6F5
:106C600092E00E9402958AE0E9E7FCE1DF011D92D3
:106C70008A95E9F74AE050E064E070E0CF010E94B5
:106C8000029580EA96E8A1E0B0E0809360029093DC
:106C90006102A0936202B093630244E050E067E1B6
:106CA00070E080E692E00E940295109280131092AC
:106CB0007F1342E050E062E070E08FE793E10E94D2
:106CC000029510927E1310927D1342E050E060E036
:106CD00070E08DE793E10E94029581E00E94A02878
:106CE00080E090E0FF90EF90DF90CF900C94FC124A
:106CF000FF90EF90DF90CF9008950E941E656C9AF0
:106D00006B9A6A9A6F9A729A749A739A779A809821
:106D100080B3897F80BB8398849887E080937E00CE
:106D2000549A0E94CF320E9400330E94A10E80E04C
:106D300090E00E94FC12609160027091610280916B
:106D40006202909163020E94F45E0E94B31060930D
:106D5000B1307093B2308093B3309093B43080915F
:106D6000660286FD239A219A229A239A0E94B60EE1
:106D70001D9B05C01092881310928713089581E01F
:106D800090E090938813809387130895CF93DF93B7
:106D900090E04091891350918A1360918B13709108
:106DA0008C1341FD08C02091660220FD04C021FF24
:106DB0008CC01D9B8AC02DE8289FE001299FD00D23
:106DC0001124CE018156924E9F938F9382E295E0DB
:106DD0009F938F930E942392FE01E856F24EDF01AB
:106DE000AA57BF4F2C910F900F900F900F90438197
:106DF0005481658176818091B5309091B630A091B3
:106E0000B730B091B830841B950BA60BB70B22237B
:106E1000D1F1BF93AF939F938F93DF01A257BF4FE1
:106E200011968C9111978F938C918F931297119645
:106E30008C9111978F938C918F9313978C911F92B4
:106E40008F9311978C911F928F9313968C911F9211
:106E50008F9311978C911F928F93E957FF4F8081E9
:106E60001F928F931F922F9388E295E09F938F93A9
:106E70000E9423928DB79EB746960FB6F8949EBF98
:106E80000FBE8DBF10C0BF93AF939F938F938FE6BC
:106E900095E09F938F930E9423920F900F900F90F5
:106EA0000F900F900F900E94B01180918002882364
:106EB00061F01F928F9380EF92E09F938F930E94D7
:106EC00037920F900F900F900F90DF91CF91089510
:106ED0008091981D882341F08091991D90E00E9437
:106EE000C6360E94A70FF4CF0895CF93DF93EC012D
:106EF000888199818D3C2EE09207F1F018F4892B5E
:106F0000C1F04BC0853D2EE0920709F44CC0893D8D
:106F10009E4009F042C080E49AE00E94606D892B97
:106F200009F43FC080E49AE00E944C6D80E00E942A
:106F3000D0288DEC9EE02EC0623199F5299A4091BF
:106F40007D1350917E135695542F4427579547959E
:106F500060E070E080E49AE00E94426D80918913C5
:106F600090918A13A0918B13B0918C13A0FF10C045
:106F700080917E138F9380917D138F9381E891E1AF
:106F80009F938F930E9437920F900F900F900F90C6
:106F900085ED9EE09983888304C01982188283E07E
:106FA00019C081E017C080E49AE00E94606D892BCF
:106FB000C1F380E49AE00E944C6D0E94683740E281
:106FC00050E060E070E080E49AE00E94426D89ED5C
:106FD0009EE0E0CFDF91CF9108952F923F924F92A4
:106FE0005F926F927F928F929F92AF92BF92CF9259
:106FF000DF92EF92FF920F931F93CF93DF93CDB762
:10700000DEB72B970FB6F894DEBF0FBECDBF9B87C0
:107010008A873A01FC0180819181892B11F00C94BF
:10702000654B60917E0270917F02CA010E94579168
:1070300060E870E0C3010E949791009759F4609155
:10704000E1397091E2398AE090E00E94EB9181E0B1
:107050000C946A4B8130910561F4F3011081912EFB
:10706000990C9908892C092D292C392C492C592C3B
:10707000B9C082309105B9F4F3018081082E000C6B
:10708000990B982F88272181820F911D27FD9A95B2
:10709000182F992E892E880C8808082D282C382C1A
:1070A000482C582C9FC083309105B1F5F301208105
:1070B000922F990F990B392F492F592F692F792F1B
:1070C000892F00E10E94BB8819012A014B01B82FCA
:1070D000A92F2181922F990F990B392F492F592FC1
:1070E000692F792F892F08E00E94BB8859016A0116
:1070F0007B018C019101A201B4018B2F9A2F0E9478
:10710000F288A2801A2D110F110BB12EC12ED12E93
:10711000E12EF12E012F55C004970CF45BC0F30152
:107120002081922F990F990B392F492F592F692FB1
:10713000792F892F08E10E94BB8819012A014B0190
:10714000B82FA92F2181922F990F990B392F492FF1
:10715000592F692F792F892F00E10E94BB8859018F
:107160006A017B018C019101A201B4018B2F9A2F3E
:107170000E94F288A3801A2D110F110BB12EC12E7F
:10718000D12EE12EF12E012F0E94F28819012A0141
:107190004B01B82FA92F2281922F990F990B392FCC
:1071A000492F592F692F792F892F08E00E94BB881A
:1071B00059016A017B018C019101A201B4018B2F5D
:1071C0009A2F0E94F288122F932E842E052F1B01D6
:1071D0002C0108C01AE0912C812C00E0212C312CCC
:1071E000412C512C0E94B011212F392D482D502FA8
:1071F000B101C2012537F3E63F07FDE64F07510510
:10720000610571058105910511F40C944D462537F2
:10721000E3E63E07EDE64E07510561057105810580
:10722000910511F008F0B1C12337F2E73F0741059E
:107230005105610571058105910511F40C94E6482D
:107240002337E2E73E0741055105610571058105D8
:10725000910511F008F0B8C02536F4E63F07410566
:107260005105610571058105910509F41CC7253695
:10727000E4E63E074105510561057105810591056B
:1072800011F008F040C0A6E70E94198911F40C948F
:10729000D5420E94198909F068F4A8E60E9419896C
:1072A00009F452C7A5E70E94198911F40C94BF4252
:1072B0000C94634B212F392D482D502FB101C20161
:1072C0002436F1E63F074105510561057105810549
:1072D000910511F40C940E492537E2E63E0741056D
:1072E0005105610571058105910509F47DC42A33B5
:1072F000364241055105610571058105910509F485
:1073000032C30C94634B212F392D482D502FB101DE
:10731000C2012737EFE63E074105510561057105BA
:107320008105910511F40C94B3462737FFE63F071A
:1073300041055105610571058105910509F0C8F404
:107340002436E9E63E0741055105610571058105D1
:10735000910511F40C94984225363E46410551059D
:10736000610571058105910511F40C94E7460C94B3
:10737000634B212F392D482D502FB101C2012536E5
:10738000E2E73E074105510561057105810591055B
:1073900011F40C94B3472936F2E73F074105510534
:1073A000610571058105910511F40C94954823330D
:1073B000314741055105610571058105910511F0C0
:1073C0000C94634B0C940E49212F392D482D502FCE
:1073D000B101C2012236F5E63F07F4E64F07510539
:1073E000610571058105910509F45DC62236E5E662
:1073F0003E07E4E64E0751056105710581059105DB
:1074000011F008F05BC02133F4E63F07F1E64F07C7
:107410005105610571058105910509F4B8C2213353
:10742000E4E63E07E1E64E07510561057105810579
:10743000910509F0C0F42337F3E73F0741055105F3
:10744000610571058105910511F40C94FA482837FE
:10745000344741055105610571058105910509F420
:1074600082C20C94634B212F392D482D502FB1012E
:10747000C2012837F4E63F07F1E64F0751056105E1
:1074800071058105910509F47EC22C36E5E73E07BA
:10749000E2E64E075105610571058105910509F484
:1074A000A3C3233634464146510561057105810564
:1074B000910511F00C94634B0C940E49212F392D3A
:1074C000482D502FB101C2012D36E5E73E07E8E611
:1074D0004E075105610571058105910511F40C9464
:1074E00024492D36F5E73F07F8E64F0751056105BA
:1074F00071058105910509F0E0F42237E2E73E07C6
:10750000E5E64E075105610571058105910511F408
:107510000C94FE4523363D464846510561057105EC
:107520008105910511F00C94634B0E944C1C0C9446
:10753000654B212F392D482D502FB101C201243622
:10754000E3E63E07ECE64E0751056105710581054E
:10755000910511F40C9461452736FFE63F07FCE6E0
:107560004F075105610571058105910511F40C94D2
:10757000644523363243494651056105710581054D
:10758000910511F00C94634B22C2212F392D482D07
:10759000502FB101C2012037FCE63F07F5E64F0747
:1075A000F8E65F07610571058105910509F4CCC511
:1075B0002037ECE63E07E5E64E07E8E65E076105A4
:1075C00071058105910511F008F0E2C02437F8E754
:1075D0003F07F4E74F0751056105710581059105E6
:1075E00011F40C9441432437E8E73E07E4E74E07E3
:1075F0005105610571058105910511F008F060C024
:107600002033F1E33F07F1E74F07510561057105AD
:107610008105910511F40C94FE452033E1E33E070A
:10762000E1E74E075105610571058105910509F0F6
:10763000D8F42133F2E63F07F0E74F075105610523
:1076400071058105910509F49AC2223332464047FB
:107650005105610571058105910511F00C94634B8D
:107660000E94DC280C94654B212F392D482D502F7A
:10767000B101C2012037F5E63F07F2E74F07510598
:10768000610571058105910511F40C94B3472C3601
:10769000E4E73E074E075105610571058105910537
:1076A00011F40C94894A2133314341475105610556
:1076B00071058105910511F00C94634B0C944D46B6
:1076C000212F392D482D502FB101C2012B36ECE668
:1076D0003E07E5E74E07E2E65E07610571058105B5
:1076E000910509F481C22B36FCE63F07F5E74F0709
:1076F000F2E65F07610571058105910509F0E0F487
:107700002437E4E63E07E7E74E07510561057105BA
:107710008105910511F40C94D74A24373F464F4612
:107720005246610571058105910511F00C94634B7A
:107730000C9400000C94654B212F392D482D502FAF
:10774000B101C2012E36E1E63E07E8E64E07E3E668
:107750005E07610571058105910509F466C7263349
:10776000F9E63F07F5E74F07F5E65F0761057105A5
:107770008105910509F4ECC429363C46414653463F
:10778000610571058105910511F00C94634BC9C227
:10779000212F392D482D502FB101C2012437F3E795
:1077A0003F07F5E64F07F2E75F07610571058105C1
:1077B000910511F40C9463472437E3E73E07E5E6AF
:1077C0004E07E2E75E07610571058105910511F03D
:1077D00008F062C02337F5E63F07F2E74F07F0E70E
:1077E0005F07610571058105910511F40C94D44979
:1077F0002337E5E63E07E2E74E07E0E75E0761056F
:1078000071058105910509F0D0F42136FDE63F07A9
:10781000F5E74F07F8E65F076105710581059105FA
:1078200011F40C94D1462237374740475047610541
:1078300071058105910509F4A6C10C94634B212FB4
:10784000392D482D502FB101C2012436FDE63F07E6
:10785000F3E64F07F2E75F076105710581059105C2
:1078600009F481C52136ECE63E07E5E64E07E2E77E
:107870005E07610571058105910509F486C423370A
:10788000324747475047610571058105910511F061
:107890000C94634B0C946647212F392D482D502FA3
:1078A000B101C2012437E2E73E07E1E64E07E5E712
:1078B0005E07610571058105910509F4AFC524379F
:1078C000F2E73F07F1E64F07F5E75F07610571054E
:1078D0008105910509F0C8F42437E3E73E07E5E6A2
:1078E0004E07E4E75E07610571058105910509F41E
:1078F000F3C627373047484754476105710581056E
:10790000910509F468C60C94634B212F392D482D3D
:10791000502FB101C2012F36ECE63E07EFE54E07CE
:10792000E6E75E07610571058105910509F4C6C4A6
:107930002C36F1E63F07F4E74F07F8E75F076105EC
:1079400071058105910511F40C94564A223737468A
:1079500040475547610571058105910511F00C946B
:10796000634B0C943D4583E08093663510926835F7
:107970001092673546E655E362E182E492E00E94A8
:10798000D26E0C94654B0E94D51B0C94654B21E084
:1079900042E161E080ED0E94CD6021E042E161E0E2
:1079A00080ED0E94CD6021E042E161E080ED0E9427
:1079B000CD6021E042E161E080ED0E94CD6021E0F8
:1079C00042E161E080ED0E94CD600C94654B6091D6
:1079D0007E0270917F0280E090E00E9457916BE7F9
:1079E00075E00E947891892B09F0C5C060917E02F4
:1079F00070917F0280E090E00E9457918C01009787
:107A000009F497C064E673E00E947891892BE1F451
:107A100088EE93E0A0E0B0E0809360029093610272
:107A2000A0936202B093630268EE73E080E090E09E
:107A30000E94F45E44E050E067E170E080E692E08E
:107A40000E9402950C94654B61E875E0C8010E94A4
:107A50007891892BE1F480E197E2A0E0B0E0809397
:107A6000600290936102A0936202B093630260E1AE
:107A700077E280E090E00E94F45E44E050E067E14D
:107A800070E080E692E00E9402950C94654B64E8F9
:107A900075E0C8010E947891892BE1F480EA96E8AC
:107AA000A1E0B0E08093600290936102A093620233
:107AB000B093630260EA76E881E090E00E94F45EB1
:107AC00044E050E067E170E080E692E00E940295B9
:107AD0000C94654B68E875E0C8010E947891892B89
:107AE000E1F480E89AE1A6E0B0E080936002909330
:107AF0006102A0936202B093630260E87AE186E0DB
:107B000090E00E94F45E44E050E067E170E080E6BF
:107B100092E00E9402950C94654B87E694E09F9357
:107B20008F930E9437920E94B0110F900F900C9487
:107B3000654B609160027091610280916202909148
:107B4000630228EE33E040E050E00E94E6865F9357
:107B50004F933F932F9383E694E09F938F930E94DC
:107B600037920E94B0110F900F900F900F900F90CE
:107B70000F900C94654B0E9442160C94654B0E942A
:107B8000DC280C94654B60917E0270917F0280E04E
:107B900090E00E9457918C016EE074E00E94789111
:107BA000892B19F477980C94654B61E174E0C80156
:107BB0000E947891892B19F4779A0C94654B779BE6
:107BC00003C081E194E002C08EE094E09F938F9324
:107BD00089E196E09F938F930E9437920F900F90C8
:107BE0000F900F900C94654B60917E0270917F0214
:107BF00080E090E00E9457918C016CE875E00E9453
:107C00007891892BD1F48091981D1F928F93809148
:107C10009A1D1F928F938091991D1F928F931F928F
:107C200084E18F9381E394E09F938F930E94379236
:107C30000FB6F894DEBF0FBECDBF61E975E0C80195
:107C40000E947891892B19F40E94683766C069E90F
:107C500075E0C8010E947891892BF1F560917E0250
:107C600070917F0280E090E00E945791009709F4A4
:107C700054C00E9444908531910528F5909380135B
:107C800080937F1342E050E062E070E08FE793E181
:107C90000E94029560917E0270917F0280E090E0E8
:107CA0000E9457910097C9F10E94449090937E13CF
:107CB00080937D1342E050E060E070E08DE793E157
:107CC0000E9402952AC08FE194E09F938F930E94B7
:107CD00037920F900F9021C0809180138F938091E5
:107CE0007F138F9386E194E09F938F930E94379246
:107CF0000E94B01180917E138F9380917D138F939A
:107D000087E094E09F938F930E9437920E94B01176
:107D10000FB6F894DEBF0FBECDBF0E94B0110C9419
:107D2000654B60917E0270917F0280E090E00E943E
:107D300057918C0165EE74E00E947891892B09F0CF
:107D400077C060917E0270917F0280E090E00E9497
:107D500057918C01009711F40C94654B67E975E01D
:107D60000E947891892BB1F482E29FEFACECBBE3E7
:107D70008093850290938602A0938702B093880235
:107D800044E050E06EE470E085E892E00E940295E5
:107D90000C94654B6DE975E0C8010E947891892BC0
:107DA000B1F482E29FEFACECBAE38093850290934A
:107DB0008602A0938702B093880244E050E06EE40C
:107DC00070E085E892E00E9402950C94654BC80132
:107DD0000E9440902B013C0120E030E0A9010E946C
:107DE000048A8823D9F081E00E9451109B01AC01E4
:107DF000C301B2010E94098A6093850270938602D2
:107E0000809387029093880244E050E06EE470E033
:107E100085E892E00E9402950C94654B8AEF93E00E
:107E20009F938F930E9437920F900F900C94654B05
:107E300068EE74E0C8010E947891892B09F077C040
:107E400060917E0270917F0280E090E00E945791E5
:107E50008C01009711F40C94654B67E975E00E9462
:107E60007891892BB1F482E29FEFACECBBE3809375
:107E7000810290938202A0938302B093840244E033
:107E800050E06AE470E081E892E00E9402950C9470
:107E9000654B6DE975E0C8010E947891892BB1F4BA
:107EA00082E29FEFACECBAE380938102909382026E
:107EB000A0938302B093840244E050E06AE470E04F
:107EC00081E892E00E9402950C94654BC8010E94E3
:107ED00040902B013C0120E030E0A9010E94048A7F
:107EE0008823D9F082E00E9451109B01AC01C301AC
:107EF000B2010E94098A609381027093820280938A
:107F000083029093840244E050E06AE470E081E8E8
:107F100092E00E9402950C94654B8DEE93E09F9346
:107F20008F930E9437920F900F900C94654B60EEE8
:107F300074E0C8010E947891892B09F073C06091A8
:107F40007E0270917F0280E090E00E9457918C0148
:107F5000009711F40C94654B67E975E00E947891E5
:107F6000892BB1F487ED94E3AFEEBCE380938902F3
:107F700090938A02A0938B02B0938C0244E050E06D
:107F800062E570E089E892E00E9402950C94654BEE
:107F90006DE975E0C8010E947891892B51F48EED4E
:107FA00093E09F938F930E9437920F900F900C94C1
:107FB000654BC8010E9440902B013C0120E030E05D
:107FC000A9010E94048A882319F180E00E945110BF
:107FD0004B015C0121EE3AE744E95EE3C301B201E3
:107FE0000E942589A50194010E94098A6093890253
:107FF00070938A0280938B0290938C0244E050E04D
:1080000062E570E089E892E00E9402950C94654B6D
:1080100081ED93E09F938F930E9437920F900F9082
:108020000C94654B0E949F109F938F937F936F9347
:108030008AEC93E09F938F930E94379282E00E9494
:10804000511020918102309182024091830250911F
:1080500084020E94B58C162F072FF82EE92E81E09E
:108060000E945110EF92FF920F931F93209185026F
:108070003091860240918702509188020E94B58C0F
:108080009F938F937F936F938EEB93E09F938F9348
:108090000E9437920E94B0110FB6F894DEBF0FBE57
:1080A000CDBF0C94654B60917E0270917F0280E0A1
:1080B00090E00E945791009711F10E942E2A0091A2
:1080C000891310918A1320918B1330918C136017B0
:1080D00071078207930739F16093891370938A13AC
:1080E00080938B1390938C1344E050E06AE570E02A
:1080F00089E893E10E94029582E196E002C08BE05C
:1081000096E09F938F930E943792609189137091AC
:108110008A1380918B1390918C130E943B290E94AB
:10812000B0110F900F9080E096E09F938F930E9484
:1081300037926FEF7FEFCB010E943B290E94B01175
:108140000F900F900C94654B0E94BF250C94654BCB
:10815000F3018481843329F440E061E080E00E94EF
:10816000EF1780918002882311F40C94654B1F92C5
:108170008F938DEF95E09F938F930E9437920F908E
:108180000F900F900F900C94654BF3018481893709
:1081900009F080C060917E0270917F0280E090E0E3
:1081A0000E9457918C016EE074E00E947891892BB7
:1081B00051F48091660290916702A0916802B0919B
:1081C0006902906410C061E174E0C8010E94789176
:1081D000892BD1F48091660290916702A091680288
:1081E000B09169029F7B8093660290936702A0938F
:1081F0006802B093690244E050E06EE170E086E608
:1082000092E00E94029546C062EA75E0C8010E94B1
:108210007891892B21F58091911C8F938091901CEE
:108220008F9380918F1C8F9380918E1C8F93809160
:108230008D1C8F9380918C1C8F9380918B1C8F93BE
:1082400080918A1C8F9383E993E09F938F930E9480
:1082500037920FB6F894DEBF0FBECDBF1BC0809122
:10826000660290916702A0916802B091690296FD42
:1082700003C081E194E002C08EE094E09F938F936D
:108280008FE893E09F938F930E9437920F900F9007
:108290000F900F9080918002882311F40C94654B0D
:1082A0001F928F938AEF95E09F938F930E9437924E
:1082B0000F900F900F900F900C94654BF3018481F9
:1082C0008737E9F560917E0270917F0280E090E04F
:1082D0000E9457910097D9F00E9440902B013C01D9
:1082E00020E030E0A9010E94048A882381F04092B6
:1082F0008D0250928E0260928F027092900244E042
:1083000050E066E570E08DE892E00E940295809171
:1083100090028F9380918F028F9380918E028F9322
:1083200080918D028F9381E893E09F938F930E94B9
:1083300037920F900F900F900F900F900F908091A9
:108340008002882311F40C94654B1F928F9387EF62
:1083500095E09F938F930E9437920F900F900F900C
:108360000F900C94654B60917E0270917F0280E0CB
:1083700090E00E9457918C016EE074E00E94789129
:1083800040906602509067026090680270906902A7
:10839000892B19F4689457F809C061E174E0C801A9
:1083A0000E947891892B99F4E89457F840926602DC
:1083B00050926702609268027092690244E050E055
:1083C0006EE170E086E692E00E94029513C057FCD1
:1083D00003C081E194E002C08EE094E09F938F930C
:1083E0008DE793E09F938F930E9437920F900F90A9
:1083F0000F900F9080918002882311F40C94654BAC
:108400001F928F9384EF95E09F938F930E943792F2
:108410000F900F900F900F900C94654B60917E021F
:1084200070917F0280E090E00E9457918C0168EA91
:1084300075E00E947891892B11F489E108C06CEAFB
:1084400075E0C8010E947891892B49F480E18093FE
:10845000C4001092C50082E08093C00055C060EB5C
:1084600075E0C8010E947891892B11F488E0EFCF64
:1084700065EB75E0C8010E947891892B39F06AEBB1
:1084800075E0C8010E947891892B11F483E0DFCF59
:108490008091C400893141F488E793E09F938F93E2
:1084A0000E9437920F900F908091C400803141F468
:1084B00083E793E09F938F930E9437920F900F90E2
:1084C0008091C400883041F48DE693E09F938F93B0
:1084D0000E9437920F900F908091C400833041F436
:1084E00087E693E09F938F930E9437920F900F90AF
:1084F0008091C400883041F481E693E09F938F938C
:108500000E9437920F900F9080918002882311F47F
:108510000C94654B1F928F9381EF95E09F938F93FF
:108520000E9437920F900F900F900F900C94654B14
:1085300060917E0270917F0280E090E00E945791EE
:1085400067E975E00E947891892B11F481E001C000
:1085500080E00E94A02880918002882311F40C946E
:10856000654B1F928F938EEE95E09F938F930E94A1
:1085700037920F900F900F900F900C94654B0E94C4
:10858000C62680918002882311F40C94654B1F92BB
:108590008F938BEE95E09F938F930E9437920F906D
:1085A0000F900F900F900C94654B0E94C226809103
:1085B0008002882311F40C94654B1F928F9388EEF0
:1085C00095E09F938F930E9437920F900F900F909A
:1085D0000F900C94654B60917E0270917F0280E059
:1085E00090E00E9457910E944490803170F48093F3
:1085F00086130E94226941E050E06DE170E086E858
:1086000093E10E9402950C94654B809186131F9212
:108610008F9387E593E09F938F930E9437920F90FB
:108620000F900F900F900C94654B60917E027091AB
:108630007F0280E090E00E9457910E94449095EF65
:10864000980F903170F4809365020E94FB6741E0BF
:1086500050E06CE170E085E692E00E9402950C9497
:10866000654B809165021F928F938EE493E09F93F8
:108670008F930E9437920F900F900F900F900C9451
:10868000654B60917E0270917F0280E090E00E94D5
:108690005791009789F04AE050E0BC0189E79CE1DE
:1086A0000E9488914AE050E064E070E089E79CE134
:1086B0000E9402950C94654B89E79CE19F938F93F0
:1086C0008FEB95E09F938F930E9423920F900F90D2
:1086D0000F900F900C94654B60917E0270917F0219
:1086E00080E090E00E9457918C0164E673E00E9464
:1086F0007891892BD9F4219A809166029091670232
:10870000A0916802B09169028061809366029093A3
:108710006702A0936802B093690244E050E06EE102
:1087200070E086E692E00E940295CFC769EE74E0A1
:10873000C8010E947891892BD9F4229A809166020F
:1087400090916702A0916802B09169028062809363
:10875000660290936702A0936802B093690244E0B6
:1087600050E06EE170E086E692E00E940295ADC7AF
:1087700066E473E0C8010E947891892BD9F4239AAA
:108780008091660290916702A0916802B09169029F
:1087900080648093660290936702A0936802B0930E
:1087A000690244E050E06EE170E086E692E00E94EB
:1087B00002958BC76CE874E0C8010E947891892B00
:1087C000D9F4239A8091660290916702A091680281
:1087D000B091690280688093660290936702A093CB
:1087E0006802B093690244E050E06EE170E086E612
:1087F00092E00E94029569C76EE373E0C8010E948F
:108800007891892B71F581E08093CA3082E99CE1EF
:108810009093CC308093CB301092CE301092CD30EC
:108820008091660290916702A0916802B0916902FE
:1088300091608093660290936702A0936802B09360
:10884000690244E050E06EE170E086E692E00E944A
:1088500002954AEC50E362E182E492E00E94D26E1B
:1088600034C76DE673E0C8010E947891892B11F539
:10887000E2ECFCE1119211922CE1E23EF207D1F719
:108880008091660290916702A0916802B09169029E
:1088900092608093660290936702A0936802B093FF
:1088A000690244E050E06EE170E086E692E00E94EA
:1088B00002950BC761E174E0C8010E947891409174
:1088C0006602509167026091680270916902892B7B
:1088D000C1F44F705C7F40936602509367026093CF
:1088E0006802709369022B9A44E050E06EE170E0F8
:1088F00086E692E00E94029580916F350E94106892
:10890000E4C644FD03C081E194E002C08EE094E03F
:108910009F938F9383E493E09F938F930E9437926A
:10892000809166020F900F900F900F9085FD03C00D
:1089300081E194E002C08EE094E09F938F9388E3FE
:1089400093E09F938F930E943792809166020F90DD
:108950000F900F900F9086FD03C081E194E002C05C
:108960008EE094E09F938F938DE293E09F938F939B
:108970000E943792809166020F900F900F900F9097
:1089800087FD03C081E194E002C08EE094E09F93F4
:108990008F9382E293E09F938F930E94379280910E
:1089A000660290916702A0916802B09169020F90EF
:1089B0000F900F900F9090FD03C081E194E002C0F2
:1089C0008EE094E09F938F9387E193E09F938F9342
:1089D0000E9437928091660290916702A09168028E
:1089E000B09169020F900F900F900F9091FD03C00E
:1089F00081E194E002C08EE094E09F938F938CE03D
:108A000093E09F938F930E9437928091660290919A
:108A10006702A0916802B09169020F900F900F90C9
:108A20000F9091FF52C687EC95E00E945F9292EC06
:108A3000E92E9CE1F92E00E010E02FEC822E25E0DB
:108A4000922EF70180819181F2E0EF0EF11C9F934D
:108A50008F93C8010B969F938F939F928F920E9442
:108A600023920F5F1F4F0F900F900F900F900F905A
:108A70000F900031110529F728C684EE95E09F93E9
:108A80008F930E943792809180020F900F908823DD
:108A900061F01F928F9381EE95E09F938F930E94D8
:108AA00037920F900F900F900F90F89498E088E114
:108AB0000FB6F894A895809360000FBE9093600065
:108AC000FFCF0E947E6001C660917E0270917F029E
:108AD00080E090E00E9457918C016EE074E00E946B
:108AE0007891892BE9F40E94FF668091660290914B
:108AF0006702A0916802B09169028D7F81608093C6
:108B0000660290936702A0936802B093690244E002
:108B100050E06EE170E086E692E00E940295D5C5D5
:108B200061E174E0C8010E947891892BE1F40E9410
:108B300035668091660290916702A0916802B091BB
:108B400069028C7F8093660290936702A09368020B
:108B5000B093690244E050E06EE170E086E692E096
:108B60000E940295B2C56AED75E0C8010E94789135
:108B7000892BE9F40E943566809166029091670224
:108B8000A0916802B09169028E7F82608093660234
:108B900090936702A0936802B093690244E050E0AA
:108BA0006EE170E086E692E00E9402958EC58091AB
:108BB000660281FF0FC08AED95E09F938F9388E056
:108BC00093E09F938F930E9437920F900F900F9096
:108BD0000F907BC580FD03C081E194E002C08EE070
:108BE00094E09F938F9384E093E09F938F930E94F0
:108BF00037920F900F900F900F9067C58091C830FB
:108C00008F938091C7308F938091C6308F938091DE
:108C1000C5308F938091C4308F938091C3308F93F0
:108C20008091C2308F938091C1308F938091C030FA
:108C30008F938091BF308F938091BE308F938091BE
:108C4000BD308F938091BC308F938091BB308F93D8
:108C50008091BA308F938091B9308F9385EB95E0F6
:108C60009F938F930E9437920E94B011809180024F
:108C70000FB6F894DEBF0FBECDBF882309F425C51B
:108C80001F928F9382EB95E09F938F930E94379270
:108C90000F900F900F900F9018C5F89489E021E085
:108CA00030E0F90180935700C895E02C20E030E0D7
:108CB000F90180935700C895F02C7894F89423E03C
:108CC00030E0F90180935700C895002D22E030E094
:108CD000F90180935700C895102D78948091A228AF
:108CE0008F938091A1288F938091A0288F9380915A
:108CF0009F288F9388EA95E09F938F930E943792E5
:108D00001F92EF921F92FF921F920F931F921F9339
:108D100081E895E09F938F930E9437920E9460278D
:108D2000809166001F928F9385E795E09F938F93C4
:108D30000E9437920E94B011809180020FB6F89481
:108D4000DEBF0FBECDBF882309F4BFC41F928F932F
:108D500082E795E09F938F930E9437920F900F9038
:108D60000F900F90B2C460E070E080E090E00E944D
:108D7000B91160E070E081E090E00E94B91180914B
:108D80008002882309F4A1C41F928F938FE695E097
:108D90009F938F930E9437920F900F900F900F9098
:108DA00094C40E9482250E94B01180918002882381
:108DB00009F48BC41F928F938CE695E09F938F9359
:108DC0000E9437920F900F900F900F907EC4609189
:108DD0007E0270917F0280E090E00E94579161E9ED
:108DE00075E00E947891892B31F5F8948BE79AE031
:108DF0000E94AB6F8C01892B69F0C8010F960E940D
:108E0000186CB80188E092E00E945870C8010E9476
:108E10000C70F0CF8BE79AE00E94FF6F892B29F04E
:108E20008BE79AE00E94BF6FF5CF8BE79AE00E9434
:108E3000A76F789436C08BE79AE00E94AB6F8C01E5
:108E40008FEDE82E85E0F82E0115110551F1F8019E
:108E500086811F928F9380851F928F9385811F92A9
:108E60008F9381851F928F9387811F928F93848127
:108E70001F928F9383811F928F9382811F928F9372
:108E800082851F928F93FF92EF920E942392C801D6
:108E90000E940C708C010FB6F894DEBF0FBECDBFE0
:108EA000D3CF80918002882309F40FC41F928F933F
:108EB00089E695E09F938F930E9437920F900F90D1
:108EC0000F900F9002C40E942A35FFC360917E026A
:108ED00070917F0280E090E00E9457918C016EE1DA
:108EE00076E00E947891892BD1F48091660290916E
:108EF0006702A0916802B0916902977F8093660231
:108F000090936702A0936802B093690244E050E036
:108F10006EE170E086E692E00E940295D6C36DE9AC
:108F200075E0C8010E947891892BD1F48091660286
:108F300090916702A0916802B09169029860809355
:108F4000660290936702A0936802B093690244E0BE
:108F500050E06EE170E086E692E00E940295B5C3B3
:108F60000E94330EB2C360917E0270917F0280E056
:108F700090E00E945791FC0120812332C1F44AE025
:108F800050E060E070E001960E94DE8D7B836A8392
:108F900060917E0270917F0280E090E00E94579184
:108FA0002A813B81243031050CF096C002C01B821F
:108FB0001A82009709F490C01982BE016F5F7F4F3B
:108FC0000E94872E19013A014B01B82FA92F8AE080
:108FD0002A813B81829FF001839FF00D1124EE5680
:108FE000F34E4080518032813C8383818D83948114
:108FF0009E8325812F8336813887878189879101D8
:10900000A301B4018B2F9A2F5201CC80DD80EE801A
:10901000FF80088519850E94108909F460C0898144
:10902000811103C0208231822AC0181684F442289C
:1090300053289C81692A2D81722A3E81832A8F813F
:10904000982A9885B92B2985A22B408217C0209495
:1090500030946094709480949094B095A09524205E
:1090600053203C8163228D8178229E8189222F8129
:1090700092223885B3238985A82320825182628277
:10908000738284829582B683A78348E250E062E2CD
:1090900070E082E99CE10E94029581E695E09F9351
:1090A0008F930E9437928AE02A813B81829FF00150
:1090B000839FF00D1124EE56F34E208131814281C1
:1090C000538164817581868197810E94E72A0E947D
:1090D000B0110F900F9003C082E00E94293085E507
:1090E00095E09F938F930E9437922FEF3FEF4FEFC2
:1090F0005FEF6FEF7FEF8FEF9FEF0E94E72A0E94F5
:10910000B011809180020F900F90882309F4DDC286
:109110001F928F9382E595E09F938F930E943792E1
:109120000F900F900F900F90D0C260917E027091BF
:109130007F0280E090E00E945791FC012081233261
:10914000A1F44AE050E060E070E001960E94DE8DFC
:109150008B0160917E0270917F0280E090E00E941E
:10916000579104301105ECF402C000E010E00097C4
:10917000C1F04AE050E060E070E00E94098F2AE010
:10918000209FF001219FF00D1124EE56F34E7187C0
:10919000608748E250E062E270E082E99CE10E9470
:1091A000029581E00E94293080918002882309F491
:1091B0008CC21F928F938FE495E09F938F930E94B0
:1091C00037920F900F900F900F907FC20E949B706C
:1091D00080918002882309F478C21F928F938CE4D7
:1091E00095E09F938F930E9437920F900F900F906E
:1091F0000F906BC20E94EE3080918002882309F4A8
:1092000064C21F928F9389E495E09F938F930E948D
:1092100037920F900F900F900F9057C280E090E020
:109220000E947C2780918002882309F44EC21F92FD
:109230008F9386E495E09F938F930E9437920F90CF
:109240000F900F900F9041C28091AF2C81FF2DC0E5
:109250000E940825892B49F58091A6288F9380913B
:10926000A5288F938091A4288F938091A3288F9312
:109270008BE395E09F938F930E943792809187357F
:109280008F93809186358F93809185358F938091D0
:1092900084358F938EE295E09F938F930E9437924F
:1092A0000FB6F894DEBF0FBECDBF0E94B011809103
:1092B000AF2C9091B02C90FF63C081E090E00E94B1
:1092C00080247B011C0180E090E00E9480244B01FF
:1092D0008C010E94DE233F922F92FF92EF928DE14C
:1092E00095E09F938F930E9437921F930F939F92C5
:1092F0008F928DE095E09F938F930E943792240187
:1093000038019401A80147018101B701C1010E9400
:109310007D229F938F937F936F9382E095E09F933D
:109320008F930E943792242D352D462D572D6E2D6B
:10933000792D822D912F0E94DE229F938F937F9310
:109340006F9384EF94E09F938F930E943792242D24
:10935000352D462D572D6E2D792D822D912F0E9462
:109360003F239F938F937F936F9381EE94E09F931E
:109370008F930E9437920FB6F894DEBF0FBECDBF19
:109380000E94B01180918002882309F49EC11F922F
:109390008F938EED94E09F938F930E9437920F905E
:1093A0000F900F900F9091C18091AF2C82FF2BC036
:1093B00021E048E061E083E00E945A198091961D07
:1093C0008F938091951D8F938091941D8F938091A1
:1093D000931D8F938091921D8F938091911D8F93F8
:1093E0008091901D8F9380918F1D8F9387EC94E0D7
:1093F0009F938F930E9437920E94B0110FB6F894FA
:10940000DEBF0FBECDBF8091AF2C9091B02C91FFED
:109410003BC00E94BF1D20E030E048EC52E4162F14
:10942000072FF82EE92E0E94B58C20E836EE45EC89
:1094300057E40E94098A21E03EED42E45EE30E9487
:10944000228D9B01AC0160E070E080E89FE30E9408
:1094500025892BE43AE34DEB57E30E94098A9F9359
:109460008F937F936F93EF92FF920F931F938EEAE8
:1094700094E09F938F930E9437920E94B0110FB691
:10948000F894DEBF0FBECDBF80918002882309F41F
:109490001CC11F928F938BEA94E09F938F930E943D
:1094A00037920F900F900F900F900FC160917E0236
:1094B00070917F0280E090E00E94579163E276E035
:1094C0000E947891892B99F460917E0270917F02BD
:1094D00080E090E00E945791009709F4F6C00E9446
:1094E000449090915201892B80935201EEC080915B
:1094F00052018F701F928F9387EF92E09F938F930B
:109500000E9437920E94B0110F900F900F900F9011
:10951000DCC060917E0270917F0280E090E00E944A
:109520005791009711F14AE050E060E070E00E942E
:10953000DE8D603198F4609364021F926F938EE920
:1095400094E09F938F930E94379241E050E06BE14B
:1095500070E084E692E00E94029511C0809164025E
:109560001F928F9385E994E006C0809164021F9258
:109570008F938CE894E09F938F930E9437920F9083
:109580000F900F900F900E94B0118091800288235D
:1095900009F49BC01F928F9389E894E09F938F9367
:1095A0000E9437920F900F900F900F908EC0609195
:1095B0007E0270917F0280E090E00E9457918C01C2
:1095C0006EE074E00E947891892BE1F40E942A6594
:1095D0008091660290916702A0916802B091690241
:1095E00090618093660290936702A0936802B093A3
:1095F000690244E050E06EE170E086E692E00E948D
:10960000029563C061E174E0C8010E947891892BE2
:1096100099F5F8940E9438650FB6F894A895809152
:109620006000886180936000109260000FBE84B774
:10963000877F84BF80916000886180936000109272
:10964000600078948091660290916702A091680210
:10965000B09169029F7E8093660290936702A09307
:109660006802B093690244E050E06EE170E086E683
:1096700092E00E94029529C068E276E0C8010E944B
:1096800078914091660250916702609168027091F2
:109690006902892B21F454FF18C0F894FFCF54FDC0
:1096A00003C081E194E002C08EE094E09F938F9329
:1096B00083EF92E09F938F930E9437920F900F90C9
:1096C0000F900F9002C00E94A625EA85FB851182AB
:1096D000108283E02B960FB6F894DEBF0FBECDBF8D
:1096E000DF91CF911F910F91FF90EF90DF90CF907E
:1096F000BF90AF909F908F907F906F905F904F90B2
:109700003F902F900895CF93DF93EC01888199814A
:10971000009741F08B3C914109F48CC0198218826A
:1097200083E093C00E947D368091660280FD05C073
:1097300081FF01C01D9B0E943566809170008C7F67
:10974000809370008091B60080628093B600109282
:10975000B20082E08093B1008091B6008770E1F79B
:109760008091700081608093700061E57EE080E010
:1097700090E00E9407650E94C22680E00E94A02817
:109780008DEA91E19F938F930E9437920E94421637
:109790008091AF2C0F900F9086FD0E942A608091DF
:1097A000AF2C9091B02C90FD0E9496238091AF2C0D
:1097B00087FF06C021E04CE061E080ED0E94CD60B3
:1097C000809186130E942269809165020E94FB6746
:1097D0000E94F86780936B0A809165020E94FB6784
:1097E000809186131F928F9380916B0A1F928F93A3
:1097F0008DE296E09F938F930E94239210926D0AC0
:1098000010926C0A0F900F900F900F900F900F9086
:1098100086E592E0909382358093813583E290E0F3
:1098200090938213809381138BEC91E199838883C9
:1098300081E00BC06332E1F74EED50E360E070E091
:109840008CE69AE00E94ED37E3CFDF91CF91089547
:109850000F931F93CF93DF93EC018A018881998145
:10986000009711F1803E914121F01982188283E026
:1098700020C06231E9F4A80162E170E08CE69AE070
:109880000E94ED3784E0809366351092683510921F
:10989000673510936A350093693546E655E362E112
:1098A00082E492E00E94D26E80EE91E199838883F7
:1098B00081E0DF91CF911F910F910895843691053A
:1098C00014F19F938F9383E896E09F938F930E9468
:1098D00023928091B9309091BA30A091BB30B09171
:1098E000BC300196A11DB11D8093B9309093BA3060
:1098F000A093BB30B093BC300F900F900F900F909F
:1099000081E090E0089580E090E008952F923F92EA
:109910004F925F926F927F928F929F92AF92BF927F
:10992000CF92DF92EF92FF920F931F93CF93DF932B
:10993000CDB7DEB7CC59D1090FB6F894DEBF0FBE54
:10994000CDBFCB56DF4F99838883C559D0408A015C
:10995000633871F480E79AE0C456DF4F6883CC59CE
:10996000D0400E94EC71C456DF4F6881CC59D04082
:10997000CB56DF4FA881B981C559D0402D913C917C
:109980002837B1E13B0711F40C94CD5940F421156F
:10999000310581F02C3A3F4009F414C408C42A3838
:1099A00041E1340709F4E2C32139314111F40C9447
:1099B000D559FDC345E159E061E870E080E79AE0E0
:1099C0000E94D1718CEA9FE0C8C35A01E3E0F0E045
:1099D000EC0FFD1FE40FF51F1082CA010E945E4CC0
:1099E000892B81F720E030E040E050E0CC56DF4F9B
:1099F0006881C459D040627070E080E090E0A0E0DF
:109A00000E94198909F079C6212F287030E040E0C2
:109A100050E060E070E080E090E0A0E00E941989F2
:109A200099F127E04AE250E06BE270E089E290E0D1
:109A30000E94B05C88E795E30E947C5EBC01990FB0
:109A4000880B990B0E94BD8A20E030E048EC52E47C
:109A50000E94098A9F938F937F936F9387EB96E081
:109A60009F938F931F9287E78F93CE018A0D9B1D43
:109A700003969F938F930E948F92A80EB91E0FB6E4
:109A8000F894DEBF0FBECDBF212F207130E040E043
:109A900050E060E070E080E090E0A0E00E94198972
:109AA000E9F126E04AE250E06BE270E089E290E002
:109AB0000E94B05C81E090E00E9448118093851381
:109AC0008BEE9CE10E947C5EBC01990F880B990B88
:109AD0000E94BD8A20E030E048EC52E40E94098AEE
:109AE0009F938F937F936F9381EC96E09F938F93D7
:109AF0001F9287E78F93C501029621E030E02C0F7B
:109B00003D1F820F931F9F938F930E948F92A80EE9
:109B1000B91E0FB6F894DEBF0FBECDBFC257DF4FE0
:109B20002881CE58D04030E040E050E060E070E066
:109B300080E090E0A0E00E94198901F10E940411E8
:109B40009F938F937F936F938CEC96E09F938F936B
:109B50001F9287E78F93C5010296A1E0B0E0AC0F9A
:109B6000BD1F8A0F9B1F9F938F930E948F92A80EF9
:109B7000B91E0FB6F894DEBF0FBECDBF212F2074E3
:109B800030E040E050E060E070E080E090E0A0E095
:109B90000E94198931F18091B4308F938091B33054
:109BA0008F938091B2308F938091B1308F938AEDF3
:109BB00096E09F938F931F9287E78F93C50102963C
:109BC00021E030E02C0F3D1F820F931F9F938F9356
:109BD0000E948F92A80EB91E0FB6F894DEBF0FBE7A
:109BE000CDBF212F207830E040E050E060E070E011
:109BF00080E090E0A0E00E94198941F1F894809102
:109C00005E3590915F35A0916035B0916135789463
:109C1000BF93AF939F938F9388EE96E09F938F931C
:109C20001F9287E78F93C5010296A1E0B0E0AC0FC9
:109C3000BD1F8A0F9B1F9F938F930E948F92A80E28
:109C4000B91E0FB6F894DEBF0FBECDBF20E0302F97
:109C5000317040E050E060E070E080E090E0A0E033
:109C60000E94198909F05BC520E0302F327040E076
:109C700050E060E070E080E090E0A0E00E94198990
:109C800009F0CBC520E0302F347040E050E060E0B8
:109C900070E080E090E0A0E00E94198909F0EEC534
:109CA00020E0302F387040E050E060E070E080E06D
:109CB00090E0A0E00E94198909F00FC620E0302F43
:109CC000307140E050E060E070E080E090E0A0E0C3
:109CD0000E94198909F07FC620E0302F307240E0E1
:109CE00050E060E070E080E090E0A0E00E94198920
:109CF00009F0A1C620E030E040E050E0CC56DF4F54
:109D00006881C459D040647070E080E090E0A0E0C9
:109D10000E94198909F0BDC620E0C856DF4F38817E
:109D2000C859D04040E050E060E070E080E090E052
:109D3000A0E00E94198909F019C720E0C756DF4F3B
:109D40003881C959D04040E050E060E070E080E0E8
:109D500090E0A0E00E94198909F036C7CE56DF4F87
:109D60005881C259D0405170952E20E030E0452FE7
:109D700050E060E070E080E090E0A0E00E9419898F
:109D800009F050C720E030E0CE56DF4F4881C2597D
:109D9000D040427050E060E070E080E090E0A0E0F1
:109DA0000E94198909F071C720E030E0C657DF4FE3
:109DB0004881CA58D04050E060E070E080E090E018
:109DC000A0E00E94198909F093C720E030E0CE5648
:109DD000DF4F4881C259D040487050E060E070E0E9
:109DE00080E090E0A0E00E94198909F0ABC720E074
:109DF00030E0CE56DF4F4881C259D040407150E02C
:109E000060E070E080E090E0A0E00E94198909F035
:109E1000C9C720E030E0CE56DF4F4881C259D0405C
:109E2000407250E060E070E080E090E0A0E00E94CE
:109E3000198909F0E8C720E030E0CE56DF4F4881AD
:109E4000C259D040407450E060E070E080E090E0A3
:109E5000A0E00E94198911F00C943457CE56DF4FC0
:109E6000F881C259D040F0787F2E20E030E04F2FAB
:109E700050E060E070E080E090E0A0E00E9419898E
:109E800011F00C946757CD56DF4F2881C359D0404D
:109E90002170622E20E030E040E0562D60E070E05E
:109EA00080E090E0A0E00E94198911F40C94E85938
:109EB0008091AF2C82FD02C00C94AF5721E046E0A8
:109EC00061E083E00E945A1920E030E0472D50E025
:109ED00060E070E080E090E0A0E00E94198911F459
:109EE0000C94AF578091AF2C82FF02C00C94745732
:109EF00020E030E040E0CD56DF4F5881C359D040DC
:109F0000527060E070E080E090E0A0E00E9419896B
:109F100011F00C94E45720E030E040E0CD56DF4FE4
:109F20005881C359D040547060E070E080E090E008
:109F3000A0E00E94198911F00C94175820E030E03D
:109F400040E0CD56DF4F5881C359D040507160E09A
:109F500070E080E090E0A0E00E94198911F00C947C
:109F60004A5820E030E040E0CD56DF4F5881C359D9
:109F7000D040507260E070E080E090E0A0E00E948D
:109F8000198911F00C94895820E030E040E0CD565A
:109F9000DF4F5881C359D040507460E070E080E0DA
:109FA00090E0A0E00E94198911F00C94C85820E0BC
:109FB00030E040E0CD56DF4F5881C359D040587053
:109FC00060E070E080E090E0A0E00E94198911F06C
:109FD0000C94075920E030E040E0C656DF4F58812E
:109FE000CA59D04060E070E080E090E0A0E00E94BC
:109FF000198911F00C94385920E030E0492D50E0D7
:10A0000060E070E080E090E0A0E00E94198911F02B
:10A010000C946F59212F302FCE56DF4F4881C259F3
:10A02000D040CD56DF4F5881C359D040CC56DF4F7A
:10A030006881C459D0407D2DC956DF4F8881C759EA
:10A04000D0409C2DA0E00E94198911F00C947A59FF
:10A0500080916402806189838091640A8A83FE0111
:10A06000EA0DFB1D13828091891390918A13A091B0
:10A070008B13B0918C1385010D5F1F4F80FF0CC0B7
:10A080001F930F9388E798E09F938F930E942392EA
:10A090000F900F900F900F90B801CE0101960E9483
:10A0A000DB738091660282FF0AC02EE531E3A801CE
:10A0B000BE016F5F7F4F8EE692E00E949A5F8091B3
:10A0C000891390918A13A0918B13B0918C1382FD08
:10A0D00073980E94FF6680E79AE00E94EE7180917B
:10A0E000660290916702A0916802B091690290FDAA
:10A0F00002C00C94B1593FEFA31AB30A0E94F8674B
:10A10000F82E89E10E9410688091660290916702A2
:10A11000A0916802B091690290FD02C00C94AD5903
:10A1200073988091640A8F5F8093640A8A83B50173
:10A130006F5F7F4FCE0101960E94DB7380E79AE04C
:10A140000E94EE7140E050E065E88091CB14909160
:10A15000CC140E94D26E88E791E1CB56DF4FA881E4
:10A16000B981C559D0408D939C931EC088E59AE073
:10A170000E94606D892BC1F00E94FF66809166028B
:10A1800087FD2B9840E450E060E070E088E59AE0BD
:10A190000E94426D81E991E1CB56DF4FE881F98160
:10A1A000C559D0409183808381E00C94F859CB56F7
:10A1B000DF4FA881B981C559D0401D921C9283E020
:10A1C0000C94F859623181F7809066029090670292
:10A1D000A0906802B090690291FCF4CBF8018081F4
:10A1E000813021F50180F281E02D108101812281F1
:10A1F000CE56DF4F2883C259D0403381CD56DF4F32
:10A200003883C359D0404481CC56DF4F4883C4596A
:10A21000D040D5805681C956DF4F5883C759D040AA
:10A22000C780E084F184212C312C52C08230B9F4F3
:10A2300023803480E12CF12C11E000E0CE56DF4F7A
:10A240001882C259D040B0E8CD56DF4FB883C35909
:10A25000D040CC56DF4F1882C459D04032C0833032
:10A26000D1F0843009F0AECBE12CF12C212C312C33
:10A2700015E000E0CE56DF4F1882C259D040CD56CF
:10A28000DF4F1882C359D040E2E0CC56DF4FE8835D
:10A29000C459D04016C0E12CF12C212C312C15E0F2
:10A2A00000E0CE56DF4F1882C259D040CD56DF4F66
:10A2B0001882C359D040F1E0CC56DF4FF883C4591F
:10A2C000D040D12CC956DF4F1882C759D040C12C7D
:10A2D0004090B1305090B2306090B3307090B43054
:10A2E00020918D0230918E0240918F025091900208
:10A2F000C657DF4F288339834A835B83CA58D040CF
:10A300002DEC3CEC4CE45EE3C657DF4F688179816D
:10A310008A819B81CA58D0400E9426899B01AC014A
:10A32000C301B2010E94E28B87FD0BC0E894A0F844
:10A330008092660290926702A0926802B0926902CF
:10A3400046C0C657DF4F288139814A815B81CA5890
:10A35000D040C301B2010E94048A87FF38C08091B7
:10A36000BD309091BE30A091BF30B091C030019609
:10A37000A11DB11D8093BD309093BE30A093BF301E
:10A38000B093C030A0FC1ECB6894A0F88092660207
:10A3900090926702A0926802B092690215E400E20E
:10A3A000CE56DF4F1882C259D040CD56DF4F1882AB
:10A3B000C359D04034E0CC56DF4F3883C459D04025
:10A3C000D12CC956DF4F1882C759D040C12CCE5668
:10A3D000DF4F4881C259D0404470C657DF4F488391
:10A3E000CA58D04020E030E050E060E070E080E00B
:10A3F00090E0A0E00E94198909F08C9A512F5072C8
:10A40000C257DF4F5883CE58D040252F30E040E070
:10A4100050E060E070E080E090E0A0E00E941989E8
:10A4200011F00E940411802F8074C856DF4F88837A
:10A43000C859D04020E0382F40E050E060E070E0A4
:10A4400080E090E0A0E00E94198911F00E940825A8
:10A45000902F9078C756DF4F9883C959D04020E09D
:10A46000392F40E050E060E070E080E090E0A0E054
:10A470000E94198951F00E949F1060936B35709370
:10A480006C3580936D3590936E35212F217030E0BF
:10A4900040E050E060E070E080E090E0A0E00E94EA
:10A4A0001989F1F089E79CE19F938F9387E996E002
:10A4B0009F938F931F9287E78F93CE0103969F936D
:10A4C0008F930E948F924C010E945E4C0FB6F894BD
:10A4D000DEBF0FBECDBF892B09F074CA540102C084
:10A4E000A12CB12C212F227030E040E050E060E040
:10A4F00070E080E090E0A0E00E941989D1F1C501F0
:10A5000002966FE976E0E1E0F0E0EC0FFD1F8E0FC0
:10A510009F1F0E948191F3E0AF0EB11C28E7622ECD
:10A5200025E3722E36E7832E33E0932E47E7542E31
:10A53000D3018D913D011F928F939F928F921F9215
:10A540005F92C5010296E1E0F0E0EC0FFD1F8E0F77
:10A550009F1F9F938F930E948F92A80EB91E0FB6D4
:10A56000F894DEBF0FBECDBF30E8631635E3730647
:10A57000F9F6212F247030E040E050E060E070E018
:10A5800080E090E0A0E00E94198909F450C0C50164
:10A59000029663EA76E041E050E04C0F5D1F840FC5
:10A5A000951F0E94819154E0A50EB11C2E018AE7EF
:10A5B000480E511C80E1D2011D928A95E9F728E0EE
:10A5C000A20168E980EB0E94A5173201B8E06B0E8A
:10A5D000711C96E7892E93E0992E27E7F20181916D
:10A5E0002F011F928F939F928F921F922F93C501DD
:10A5F000029641E050E04C0F5D1F840F951F9F9322
:10A600008F93C556DF4F2883CB59D0400E948F923D
:10A61000A80EB91E0FB6F894DEBF0FBECDBFC5564B
:10A62000DF4F2881CB59D04046145704B9F6CD5698
:10A63000DF4F9881C359D0409078C656DF4F98833A
:10A64000CA59D04020E030E040E0592F60E070E08F
:10A6500080E090E0A0E00E941989E1F480918713E6
:10A66000909188139F938F9388EA96E09F938F939E
:10A670001F9287E78F93CE018A0D9B1D03969F93B0
:10A680008F930E948F92A80EB91E0FB6F894DEBF6A
:10A690000FBECDBF20E030E040E050E0CC56DF4FB1
:10A6A0006881C459D040617070E080E090E0A0E023
:10A6B0000E94198909F496C9E3E0F0E0EC0FFD1F50
:10A6C000EA0DFB1D80E28083A50183E090E08A19FA
:10A6D0009B09FC01E40FF51FE252FF4C20814F5F04
:10A6E0005F4F222309F471C92081E1E0F0E0EC0F13
:10A6F000FD1FE40FF51F2283ECCFCE018A0D9B1DB9
:10A700006FEA76E003960E948191B7E0AB0EB11C30
:10A71000C5010E945E4C892B09F054C975C9E1142A
:10A72000F10409F4A1CAF89440905E3550905F3569
:10A73000609060357090613578948091E31C9091C1
:10A74000E41CA091E51CB091E61CA3019201281B1A
:10A75000390B4A0B5B0BCA01B9010E94BB8AC25775
:10A76000DF4F688379838A839B83CE58D040B701BB
:10A7700080E090E00E94BB8A9B01AC01C257DF4F92
:10A78000688179818A819B81CE58D0400E94098A54
:10A790004C019F928F937F936F9383EF96E09F93EB
:10A7A0008F931F9287E78F939E012A0D3B1D2D5F8C
:10A7B0003F4F3F932F93C456DF4F6883CC59D0400F
:10A7C000C556DF4F7883CB59D0400E948F92A80E98
:10A7D000B91EC456DF4F6881CC59D040C556DF4FF3
:10A7E0007881CB59D040862F972FA82DB92D8093F3
:10A7F000703590937135A0937235B0937335409254
:10A80000E31C5092E41C6092E51C7092E61C0FB6AB
:10A81000F894DEBF0FBECDBF27CAE114F10409F4DE
:10A8200031CAF8948091BA1C9091BB1CA091BC1CB9
:10A83000B091BD1C78949F938F9380916D028F93FC
:10A8400080916C028F9380E097E09F938F931F928B
:10A8500087E78F93C5010296A1E0B0E0AC0FBD1F62
:10A860008A0F9B1F9F938F930E948F92A80EB91EF1
:10A870000FB6F894DEBF0FBECDBF04CAF894809126
:10A88000623590916335A0916435B09165357894C7
:10A89000BF93AF939F938F9380E197E09F938F93A4
:10A8A0001F9287E78F93C501029621E030E02C0FBD
:10A8B0003D1F820F931F9F938F930E948F92A80E2C
:10A8C000B91EC5010E945E4C0FB6F894DEBF0FBEE4
:10A8D000CDBF892B09F076C8E3C9E114F10409F46E
:10A8E000EDC9F894409062355090633560906435BE
:10A8F0007090653578948091E71C9091E81CA09148
:10A90000E91CB091EA1CA3019201281B390B4A0BE8
:10A910005B0BCA01B9010E94BB8AC257DF4F688333
:10A9200079838A839B83CE58D040B70180E090E042
:10A930000E94BB8A9B01AC01C257DF4F68817981BD
:10A940008A819B81CE58D0400E94098A4C019F92F7
:10A950008F937F936F938BE197E09F938F931F92D9
:10A9600087E78F939E012A0D3B1D2D5F3F4F3F933D
:10A970002F93C456DF4F6883CC59D040C556DF4F64
:10A980007883CB59D0400E948F92A80EB91EC4562E
:10A99000DF4F6881CC59D040C556DF4F7881CB5905
:10A9A000D040862F972FA82DB92D80937435909382
:10A9B0007535A0937635B09377354092E71C509269
:10A9C000E81C6092E91C7092EA1C0FB6F894DEBF96
:10A9D0000FBECDBF73C9EF2809F47EC9F8948091EA
:10A9E000BE1C9091BF1CA091C01CB091C11C78945A
:10A9F0009F938F9380916B028F9380916A028F93C4
:10AA000088E297E09F938F931F9287E78F93C5010A
:10AA10000296A1E0B0E0AC0FBD1F8A0F9B1F9F9371
:10AA20008F930E948F92A80EB91E0FB6F894DEBFC6
:10AA30000FBECDBF51C98091B5309091B630A09175
:10AA4000B730B091B830BF93AF939F938F9388E3A3
:10AA500097E09F938F931F9287E78F93C50102968C
:10AA600021E030E02C0F3D1F820F931F9F938F93A7
:10AA70000E948F92A80EB91EC5010E945E4C0FB6AF
:10AA8000F894DEBF0FBECDBF892B11F00C94E24CC1
:10AA900031C98091C0308F938091BF308F93809166
:10AAA000BE308F938091BD308F938091BC308F9357
:10AAB0008091BB308F938091BA308F938091B93061
:10AAC0008F9383E497E09F938F931F9287E7982E4D
:10AAD0009F92C5010296A1E0B0E0AC0FBD1F8A0FA6
:10AAE0009B1F9F938F930E948F92A80EB91EC50142
:10AAF0000E945E4C0FB6F894DEBF0FBECDBF892B0F
:10AB000011F00C94E24C8091AF2C9091B02C90FFFE
:10AB100003C98091C4308F938091C3308F9380910B
:10AB2000C2308F938091C1308F9387E697E09F93D7
:10AB30008F931F929F92C501029621E030E02C0F67
:10AB40003D1F820F931F9F938F930E948F92A80E99
:10AB5000B91EC5010E945E4C0FB6F894DEBF0FBE51
:10AB6000CDBF892B11F00C94E24CD6C88091A62859
:10AB70008F938091A5288F938091A4288F938091A3
:10AB8000A3288F9389E797E09F938F931F9287E77E
:10AB90008F93C5010296A1E0B0E0AC0FBD1F8A0FF4
:10ABA0009B1F9F938F930E948F92A80EB91EC50181
:10ABB0000E945E4C0FB6F894DEBF0FBECDBF892B4E
:10ABC00011F00C94E24CB9C880916E358F9380914E
:10ABD0006D358F9380916C358F9380916B358F930A
:10ABE00084E897E09F938F931F9287E78F93C50127
:10ABF000029621E030E02C0F3D1F820F931F9F93A0
:10AC00008F930E948F92A80EB91EC5010E945E4CC0
:10AC10000FB6F894DEBF0FBECDBF892B11F00C9498
:10AC2000E24C9CC881E00E94511020918502309135
:10AC3000860240918702509188020E94B58C9F93B2
:10AC40008F937F936F9381E997E09F938F931F92E8
:10AC500087E78F93C5010296A1E0B0E0AC0FBD1F5E
:10AC60008A0F9B1F9F938F930E948F92A80EB91EED
:10AC7000C5010E945E4C0FB6F894DEBF0FBECDBF7B
:10AC8000892B11F00C94E24C7DC882E00E94511097
:10AC9000209181023091820240918302509184027E
:10ACA0000E94B58C9F938F937F936F938EE997E06B
:10ACB0009F938F931F9287E78F93C501029621E0A0
:10ACC00030E02C0F3D1F820F931F9F938F930E94A4
:10ACD0008F92A80EB91EC5010E945E4C0FB6F89463
:10ACE000DEBF0FBECDBF892B11F00C94E24C5CC8C7
:10ACF00083E00E9451109F938F937F936F938BEA11
:10AD000097E09F938F931F9287E78F93C5010296D9
:10AD1000A1E0B0E0AC0FBD1F8A0F9B1F9F938F93E4
:10AD20000E948F92A80EB91E8C98C5010E945E4C9D
:10AD30000FB6F894DEBF0FBECDBF892B11F00C9477
:10AD4000E24C43C88091AF2C87FF51C821E042E11B
:10AD500061E080ED0E94CD609F938F937F936F930E
:10AD600088EB97E09F938F931F9287E78F93C5019E
:10AD7000029621E030E02C0F3D1F820F931F9F931E
:10AD80008F930E948F92A80EB91EC5010E945E4C3F
:10AD90000FB6F894DEBF0FBECDBF892B11F00C9417
:10ADA000E24C25C88091AF2C87FF33C821E042E1F7
:10ADB00062E080ED0E94CD609F938F937F936F93AD
:10ADC00086EC97E09F938F931F9287E78F93C5013F
:10ADD0000296A1E0B0E0AC0FBD1F8A0F9B1F9F93AE
:10ADE0008F930E948F92A80EB91EC5010E945E4CDF
:10ADF0000FB6F894DEBF0FBECDBF892B11F00C94B7
:10AE0000E24C0C94094F8091AF2C87FF14C821E0CD
:10AE100042E163E080ED0E94CD609F938F937F932A
:10AE20006F9384ED97E09F938F931F9287E78F93A3
:10AE3000C501029621E030E02C0F3D1F820F931FC9
:10AE40009F938F930E948F92A80EB91EC5010E94F6
:10AE50005E4C0FB6F894DEBF0FBECDBF892B11F04C
:10AE60000C94E24C0C941B4F8091AF2C87FD02C0D8
:10AE70000C942E4F21E042E164E080ED0E94CD6011
:10AE80009F938F937F936F9382EE97E09F938F931F
:10AE90001F9287E78F93C5010296A1E0B0E0AC0F47
:10AEA000BD1F8A0F9B1F9F938F930E948F92A80EA6
:10AEB000B91EC5010E945E4C0FB6F894DEBF0FBEEE
:10AEC000CDBF892B11F00C94E24C0C942E4F809145
:10AED000AF2C82FD02C00C94434F46E061E083E05A
:10AEE0000E945A190C94434F8091921D8F93809128
:10AEF000911D8F938091901D8F9380918F1D8F93C3
:10AF000080EF97E09F938F931F9287E78F93C50100
:10AF1000029641E050E04C0F5D1F840F951F9F93F8
:10AF20008F930E948F92A80EB91EC5010E945E4C9D
:10AF30000FB6F894DEBF0FBECDBF892B11F00C9475
:10AF4000E24C20E030E040E0562D60E070E080E030
:10AF500090E0A0E00E94198911F40C94784F809140
:10AF6000AF2C82FD02C00C94784F8091961D8F9378
:10AF70008091951D8F938091941D8F938091931D47
:10AF80008F9388EF97E09F938F931F9287E78F931C
:10AF9000C5010296E1E0F0E0EC0FFD1F8E0F9F1F50
:10AFA0009F938F930E948F92A80EB91EC5010E9495
:10AFB0005E4C0FB6F894DEBF0FBECDBF892B11F0EB
:10AFC0000C94E24C0C94784F8091AF2C9091B02C63
:10AFD00090FD02C00C948B4F80E090E00E94802492
:10AFE0009F938F937F936F9383E098E09F938F93CA
:10AFF0001F9287E78F93C501029641E050E04C0F06
:10B000005D1F840F951F9F938F930E948F92A80EB0
:10B01000B91EC5010E945E4C0FB6F894DEBF0FBE8C
:10B02000CDBF892B11F00C94E24C0C948B4F809186
:10B03000AF2C9091B02C90FD02C00C949E4F81E0FB
:10B0400090E00E9480249F938F937F936F9383E17E
:10B0500098E09F938F931F9287E78F93C501029685
:10B06000E1E0F0E0EC0FFD1F8E0F9F1F9F938F9389
:10B070000E948F92A80EB91EC5010E945E4C0FB6A9
:10B08000F894DEBF0FBECDBF892B11F00C94E24CBB
:10B090000C949E4F8091AF2C9091B02C90FD02C0EB
:10B0A0000C94B14F81E090E00E9480242B013C0180
:10B0B00080E090E00E9480249B01AC01C301B201BA
:10B0C0000E947D229F938F937F936F9384E298E0F9
:10B0D0009F938F931F9287E78F93C501029641E05C
:10B0E00050E04C0F5D1F840F951F9F938F930E941C
:10B0F0008F92A80EB91EC5010E945E4C0FB6F8943F
:10B10000DEBF0FBECDBF892B11F00C94E24C0C9426
:10B11000B14F8091AF2C9091B02C90FD02C00C9457
:10B12000C44F81E090E00E9480242B013C0180E02C
:10B1300090E00E9480249B01AC01C301B2010E94F7
:10B14000DE229F938F937F936F938FE298E09F937C
:10B150008F931F9287E78F93C5010296E1E0F0E09D
:10B16000EC0FFD1F8E0F9F1F9F938F930E948F9256
:10B17000A80EB91EC5010E945E4C0FB6F894DEBF42
:10B180000FBECDBF892B11F00C94E24C0C94C44F30
:10B190008091AF2C9091B02C90FD02C00C94D74FB1
:10B1A00081E090E00E9480242B013C0180E090E04F
:10B1B0000E9480249B01AC01C301B2010E943F2385
:10B1C0009F938F937F936F938DE398E09F938F93DB
:10B1D0001F9287E78F93C501029641E050E04C0F24
:10B1E0005D1F840F951F9F938F930E948F92A80ECF
:10B1F000B91EC5010E945E4C0FB6F894DEBF0FBEAB
:10B20000CDBF892B11F00C94E24C0C94D74F809158
:10B21000AF2C9091B02C91FD02C00C94EA4F0E948B
:10B22000BF1D9F938F937F936F9380E598E09F93CB
:10B230008F931F9287E78F93C5010296E1E0F0E0BC
:10B24000EC0FFD1F8E0F9F1F9F938F930E948F9275
:10B25000A80EB91EC5010E945E4C0FB6F894DEBF61
:10B260000FBECDBF892B11F00C94E24C0C94EA4F29
:10B27000D10116968C9116971F928F9315968C91EB
:10B2800015971F928F9313968C9113971F928F93FC
:10B2900012968C911F928F9381E698E09F938F93E3
:10B2A0001F9287E78F93C5010296E1E0F0E0EC0F73
:10B2B000FD1F8E0F9F1F9F938F930E948F92A80E4A
:10B2C000B91EC5010E945E4C0FB6F894DEBF0FBEDA
:10B2D000CDBF892B11F00C94E24C0C94FC4F779A63
:10B2E0008091891390918A13A0918B13B0918C1344
:10B2F00092FD749A8091891390918A13A0918B1377
:10B30000B0918C1382FD0CC08091660280FD08C054
:10B3100081FD02C00C9428501D9902C00C94285045
:10B3200040E050E060E070E0CE0101960E94BC0E6B
:10B330008091981D90E020917F13309180138217A7
:10B34000930710F40C94285040E050E062E180E153
:10B3500092E00E94D26E0C9428508F2D0E941068AB
:10B36000739A8091871390918813892B11F00E9412
:10B3700035668091640A8F5F8093640A8091891397
:10B3800090918A13A0918B13B0918C1382FD02C00F
:10B390000C94E24C739A0C94E24C653811F00C94C6
:10B3A000D450A12CB12C0C94845088E59AE00E94D2
:10B3B000606D892B11F40C94D4500E9435668091F5
:10B3C000660287FD02C00C94E24C2B9A0C94E24C6E
:10B3D00020E030E0472D50E060E070E080E090E059
:10B3E000A0E00E94198911F00C94724F0C94784FD0
:10B3F000C456DF4F0FB6F894DEBF0FBECDBFDF914E
:10B40000CF911F910F91FF90EF90DF90CF90BF9061
:10B41000AF909F908F907F906F905F904F903F90F4
:10B420002F9008950C9484714F925F926F927F9247
:10B430009F92AF92BF92CF92DF92EF92FF920F93C3
:10B440001F93CF93DF93CDB7DEB760970FB6F89415
:10B45000DEBF0FBECDBF5B010E94F867E82FF0E0B2
:10B46000EE0FFF1FE455F34E808191810196918389
:10B4700080838091891390918A13A0918B13B0914E
:10B480008C1381FD74984090660250906702609022
:10B490006802709069020E9437736C01FC01808120
:10B4A000982F92959F70913099F48F7051F48091FC
:10B4B000901C9091911C01969093911C8093901CEC
:10B4C0003CC1B5018DE897E30E94F072892B51F0E1
:10B4D00080918E1C90918F1C019690938F1C80936D
:10B4E0008E1C2BC1D301C2013EE0B695A79597955E
:10B4F00087953A95D1F7F82FF1709F2E8BE79AE058
:10B500000E94AB6F7C01892B09F44BC0B501C701C8
:10B5100002960E94F072892B09F43FC087012BE646
:10B520003EE040E054E660E070E0C7010F960E9404
:10B53000E06BF6019181F7018481981321C0828527
:10B540008F5F828780918C1C90918D1C01969093C7
:10B550008D1C80938C1C84E00E942774F701208549
:10B5600030E02817390708F078C184E00E9427747A
:10B57000F7018087F60180818F70F7018187DDC038
:10B58000F701128684E00E942774F7018087F60194
:10B5900080818F70F701818761C1C7010E940C70A3
:10B5A000B1CF88E092E00E9433707C01892B09F4CE
:10B5B000C4C0B501C70102960E94E972F6018181FB
:10B5C0008150F701848380E091E0A0E0B0E08387C0
:10B5D0009487A587B687128684E00E942774F701B6
:10B5E0008087F60180818F70F7018187B7018BE733
:10B5F0009AE00E94E66F87012BE63EE040E054E6C9
:10B6000060E070E0C7010F960E94E06B11E0F60168
:10B610008181F7018483F60180818F70F701878330
:10B6200084E00E942774F701858383E00E942774D9
:10B63000F701868387818F3009F010E0F6014180A1
:10B64000F7018481481A512C612C712C86E0440C3E
:10B65000551C661C771C8A95D1F723853485458552
:10B660005685A0ECB0E00E944D87BB27A92F982FEC
:10B67000872F480E591E6A1E7B1E43865486658698
:10B680007686A501B701C6010E94BC0E8091981D67
:10B6900090E020917F13309180138217930738F048
:10B6A00040E050E062E180E192E00E94D26E809141
:10B6B0007F1390918013029708F44BC08091AF2CB8
:10B6C00086FF2AC00E941C60C60105960E94E85FA2
:10B6D000F60181811F928F93F70186811F928F93CC
:10B6E00085811F928F9389E898E09F938F931F9293
:10B6F00080E18F93CE0101965C019F938F930E940E
:10B700008F9282E00E940260C5010E94E85F0FB63E
:10B71000F894DEBF0FBECDBF8091660290916702A4
:10B72000A0916802B091690297FD4DC080917F138E
:10B7300090918013029708F47AC0809189139091B8
:10B740008A13A0918B13B0918C1381FF89C0749AD6
:10B7500087C08091660290916702A0916802B091C3
:10B76000690296FFABCF992009F4A8CFF60180813A
:10B77000982F9F709230E8F09150807F892B8083C2
:10B7800080E79AE00E94125A80918A1C90918B1C4B
:10B79000019690938B1C80938A1C809189139091C1
:10B7A0008A13A0918B13B0918C1396FF87CF739857
:10B7B00085CF8091901C9091911C01969093911C43
:10B7C0008093901C7BCF89E79CE12091791C2223F8
:10B7D00009F4ACCF9F938F938CE998E09F938F935C
:10B7E000CE0101963C019F938F930E94CC925C0105
:10B7F000B301C60102960E94A2910F900F900F9084
:10B800000F900F900F90009709F490CFEFEFAE1AC2
:10B81000BE0A8A0D9B1DAC010196FA0120812032DF
:10B82000D1F362E18AE192E00E94D26E7FCF1123D0
:10B8300009F483CF82E08093CA301092CC3010920A
:10B84000CB30F092CE30E092CD304AEC50E362E162
:10B8500082E492E00E94D26E70CF912C10E0D7CE9D
:10B8600060960FB6F894DEBF0FBECDBFDF91CF91CB
:10B870001F910F91FF90EF90DF90CF90BF90AF900E
:10B880009F907F906F905F904F90089581159105E4
:10B8900011F00197F1F70895E0918B35F0918C3517
:10B8A000908180918A3589230895E0918835F091BF
:10B8B0008935808190918A35892B8083E0918D35FF
:10B8C000F0918E35808190918A35892B80830895FF
:10B8D0001F93CF93DF93E0918835F0918935908164
:10B8E00080918A35809589238083E0918D35F09110
:10B8F0008E35808190918A35892B80838FE897E0FF
:10B900000E94465C1FB7F894E0918D35F0918E351A
:10B91000908180918A3580958923808389E091E0A8
:10B920000E94465CE0918B35F0918C35D081C091BE
:10B930008A351FBF789485E896E00E94465CE091C6
:10B940008B35F0918C35908180918A35982319F050
:10B950008D2F8C2301C081E0DF91CF911F9108953D
:10B9600050938E3540938D3570938935609388352B
:10B9700090938C3580938B3581E001C0880F2A9598
:10B98000EAF780938A350C94685CCF93DF93C82FD5
:10B99000DFB7F894E0918D35F0918E3580819091EC
:10B9A0008A35892B808387E090E00E94465CCC2317
:10B9B00051F0E0918D35F0918E35808190918A35EE
:10B9C00090959823908384E390E00E94465CE091F8
:10B9D0008B35F0918C35808190918A35892309F4DB
:10B9E000C0E085EB90E00E94465CE0918D35F091DF
:10B9F0008E35808190918A35909598239083DFBF12
:10BA000088E790E00E94465C8C2FDF91CF910895EB
:10BA1000CF93DF93C82FD8E08C2F81700E94C55C34
:10BA2000C6958111C068D150B9F78C2FDF91CF91A5
:10BA300008958FEF0C94085DDF92EF92FF920F93C1
:10BA40001F93CF93DF93E82EEB010E94685C811176
:10BA50002FC080EF0E94085DF12C10E488EFD82EF3
:10BA6000D10E81E00E94C55C082F81E00E94C55C78
:10BA7000882319F0002361F01DC0011109C01E15B3
:10BA800028F0888180FF04C0E11611F0F12E01E05A
:10BA9000802F0E94C55C98819695011190689883CB
:10BAA00011501D11DECF21961111D8CF8F2D03C05B
:10BAB0008FEF01C08EEFDF91CF911F910F91FF901B
:10BAC000EF90DF900895FF920F931F93CF93DF9332
:10BAD000F82EEB010E94685C209769F085E50E94D2
:10BAE000085D8E01085F1F4F89910E94085DC01795
:10BAF000D107D1F703C08CEC0E94085D8F2DDF9138
:10BB0000CF911F910F91FF900C94085D0F931F939D
:10BB1000CF93DF93DB01EC9111969C911197F0E0AC
:10BB2000F92B803181F4BF016E7FE3E0660F771F50
:10BB3000EA95E1F716969C911697ECE0F0E0E91B88
:10BB4000F109E60FF71FF7FF07C091E0EA019883BC
:10BB5000F195E195F10902C0EA011882883279F481
:10BB600014968C91982F9076903649F086FF02C0FB
:10BB7000EE7F05C085FF02C0EC7F01C0E87FCF01EA
:10BB800044E0969587954A95E1F7D9018C93EF703B
:10BB9000E801E88380E0DF91CF911F910F91089534
:10BBA0000F931F93CF93DF93EC018B01B801888132
:10BBB0000E941C5D888381508D3F30F4F8018081A4
:10BBC000883211F0803191F7DF91CF911F910F9161
:10BBD0000895CF93DF93EC010E94685CBE0184EB73
:10BBE0000E94635D81E00E94C55CC82F0E94685C72
:10BBF00081E0C11101C080E0DF91CF9108951F93D2
:10BC0000CF93DF931F921F92CDB7DEB7182F6983B2
:10BC10007A830E94685C0E944C5C69817A818823E7
:10BC200041F084E40E94635D113029F00E94555C6C
:10BC300002C082E001C080E00F900F90DF91CF91B1
:10BC40001F9108954F925F926F927F928F929F9271
:10BC5000AF92BF92CF92DF92EF92FF920F931F931A
:10BC6000CF93DF93CDB7DEB729970FB6F894DEBF39
:10BC70000FBECDBF6C015B014A0189010E94685C67
:10BC8000B6018EEB0E94635DCE0101967C013E0100
:10BC90009AE0690E711C27010E94195DF7018193DA
:10BCA0007F01E615F705C1F769E070E0C2010E9467
:10BCB000C677811109C09401A501B201F601808106
:10BCC0000E94865D80E001C083E029960FB6F8945B
:10BCD000DEBF0FBECDBFDF91CF911F910F91FF90BF
:10BCE000EF90DF90CF90BF90AF909F908F907F901C
:10BCF0006F905F904F900895EF92FF920F931F9374
:10BD0000CF93DF93CDB7DEB72B970FB6F894DEBF96
:10BD10000FBECDBFF82EE92E682F792F88E08F0D4A
:10BD20000E94FF5D882319F084E391E243C06CE830
:10BD300072E88EE190E00E94E75E8E01075F1F4F80
:10BD40009801AE01465F5F4FBE01655F7F4F8F2D4B
:10BD50009E2D0E94225E8111E7CF88E0E1EEF2E0A5
:10BD6000DE01119601900D928A95E1F7498521E750
:10BD700032E0429FC001439F900D112464E670E0C1
:10BD80000E94D2868A8594E6899F600D711D1124D8
:10BD9000FE0131968191481303C06F5F7F4F03C04E
:10BDA000E017F107B9F78B85882319F07195619534
:10BDB0007109CB012B960FB6F894DEBF0FBECDBF35
:10BDC000DF91CF911F910F91FF90EF900895DC01CB
:10BDD000CB0181159105A105B10529F08150904055
:10BDE000A040B040D9F708959B01AC011092B90072
:10BDF00060E074E284EF90E00E94E6862051310911
:10BE00004109510956954795379527952093B800D4
:10BE1000089594EA9093BC0040EA56E861E070E02F
:10BE20009091BC0097FD0BC0415051096109710907
:10BE3000411551056105710599F781E008959091CB
:10BE4000B900987F983011F09031B9F78093BB001A
:10BE500084E88093BC0080EA96E8A1E0B0E02091FD
:10BE6000BC0027FD08C00197A109B1090097A105F1
:10BE7000B105A9F7E2CF8091B900887F883111F030
:10BE80008034D9F680E0089524EA34E844E9209328
:10BE9000BC009091BC0097FFFCCF9091B900987FB7
:10BEA000983011F0903199F78093BB003093BC002B
:10BEB0009091BC0097FFFCCF9091B900987F903291
:10BEC00011F0983539F44093BC009091BC0094FD7A
:10BED000FCCFDDCF08950C94095F84E98093BC000A
:10BEE0008091BC0084FDFCCF08958093BB0084E862
:10BEF0008093BC008091BC0087FFFCCF9091B9007B
:10BF0000987F81E0983209F480E0089584EC809372
:10BF1000BC008091BC0087FFFCCF8091BB000895DE
:10BF200084E88093BC008091BC0087FFFCCF8091A7
:10BF3000BB000895E0E1DC01FD91CD01F0933F01EC
:10BF4000E150C9F780913C018F7D80933C01809145
:10BF50003C01877F80933C01FB0180E191919093AC
:10BF60003E018150D9F780913C01806880933C016B
:10BF700080913D0180FFFCCF4051510980913C01EF
:10BF8000806280933C0180913C01877F80933C01DB
:10BF9000141615069CF4FB0180E1919190933E01EB
:10BFA0008150D9F780913C01806880933C01809159
:10BFB0003D0180FFFCCF40515109EACFF90180E1FA
:10BFC00090913E0191938150D9F781E090E00895DE
:10BFD0000F931F93CF93DF93EC018CE70E94445F94
:10BFE0008CE70E94755F8E01005F1F4F89910E9450
:10BFF000755FC017D107D1F7DF91CF911F910F91D6
:10C000000C946D5F813019F440E050E002C040ECC8
:10C0100050E060E070E08CE790E00C948D17813088
:10C0200019F44EE050E002C048E050E060E070E0FB
:10C030008CE790E00C948D1741E050E060E070E0F8
:10C040008CE790E00E948D1764ED74E180E090E051
:10C050000C94E75E48E350E060E070E08CE790E02D
:10C060000E948D1749E350E060E070E08CE790E0BB
:10C070000E948D1744E150E060E070E08CE790E0B2
:10C080000E948D1748E750E060E070E08CE790E098
:10C090000E948D174EE550E060E070E08CE790E084
:10C0A0000E948D174DE650E060E070E08CE790E074
:10C0B0000E948D1768E374E38CE090E00E94E75ED5
:10C0C0004CE050E060E070E08CE790E00E948D175B
:10C0D00041E050E060E070E08CE790E00E948D1756
:10C0E00046E050E060E070E08CE790E00E948D1741
:10C0F00064ED74E180E090E00C94E75ECF93DF9311
:10C10000CDB7DEB7A2970FB6F894DEBF0FBECDBF96
:10C1100081E1EBE2F9E0DE01529601900D928A9501
:10C12000E1F781E1ECE3F9E0DE01119601900D9277
:10C130008A95E1F70E942A60CE0142960E94E85F4C
:10C1400082E00E94026064ED74E180E090E00E9471
:10C15000E75ECE0101960E94E85F60E27CE581E542
:10C1600090E00E94E75E80E00E940F6060E27CE564
:10C1700081E590E00E94E75E4EE050E060E070E014
:10C180008CE790E00E948D17A2960FB6F894DEBF60
:10C190000FBECDBFDF91CF910895CF92DF92EF9286
:10C1A000FF920F931F93CF93DF9300D0CDB7DEB7ED
:10C1B000F82E042F122F213031F0223031F02430AC
:10C1C00031F0283031F090E005C091E003C092E0FA
:10C1D00001C093E00C3059F00E3011F4946007C0A8
:10C1E000003111F4986003C0023109F49C606130A1
:10C1F00059F0623011F4906207C0633011F490641A
:10C2000003C0643009F490669068692F70E023E001
:10C2100030E0AE014F5F5F4F8F2D90E00E94A51779
:10C2200062E174E380E090E00E94E75E8F2D816020
:10C23000F82E0E94095F0E94865F89830E94865FB4
:10C240008A83023119F40E94865F8B830E94865F85
:10C2500087FDF1CF0E94905F0E946D5F62E174E301
:10C2600080E090E00E94E75E8F2D0E94095F0E94AF
:10C27000865F89830E94865F8A83023119F40E9457
:10C28000905F8B830E94905F0E946D5F39812A814D
:10C29000023149F5832F90E0A0E0B0E04B81772791
:10C2A000662731FF0EC030E0322F2227620F731F46
:10C2B000811D911D640F711D811D911D8C6F9F6FDC
:10C2C0000BC030E0322F2227620F731F811D911D9A
:10C2D000640F711D811D911D0E94BD8A20E83FEFF2
:10C2E0004FEF57E420C0632F70E0762F6627620F70
:10C2F000711D882777FD8095982F0E94BD8A0C308C
:10C3000029F420E030EE4FEF54E40DC00E3029F454
:10C3100020E038EF4FEF55E406C0003131F420E063
:10C320003EEF4FEF56E40E94098A2FE632E143E0E8
:10C3300050E40E94B58C6B017C01612F70E080E0BD
:10C3400090E00E94BD8A9B01AC01C701B6010E942A
:10C35000098A0F900F900F90DF91CF911F910F914D
:10C36000FF90EF90DF90CF900895CF93E6E4F1E057
:10C37000208190818081C081C295C695C695C37089
:10C38000207CC20F969596959073C90F82958C70FC
:10C39000C80F1F92CF938AEC92E19F938F930E94D4
:10C3A00037920F900F900F900F908C2FCF91089590
:10C3B0001F93CF93DF9346E069E180E00E94C06461
:10C3C00080E00E9415650E94A36304B600FE08C0C9
:10C3D00089EB92E19F938F930E9437920F900F9079
:10C3E00004B601FE08C088EA92E19F938F930E94F1
:10C3F00037920F900F9004B602FE08C087E992E1D1
:10C400009F938F930E9437920F900F9004B603FE74
:10C4100008C086E892E19F938F930E9437920F9015
:10C420000F9004B604FE08C089E792E19F938F93B2
:10C430000E9437920F900F908DE499E09F938F9315
:10C440008EE592E19F938F930E9437920E942D6F09
:10C450000E945E6E60E070E085EB92E00E94006FEB
:10C460000E94D46BE0919109F091920919950E9474
:10C47000B56190E00E9441650E94017382E0809363
:10C480008D3780938E370E949B634DE857E3BC0144
:10C490008DEC9BEA0E9415680E940B630E94FB676B
:10C4A0000E949F630E9422690E944074E091070AE3
:10C4B000F091080A1995E091DF09F091E0091995CA
:10C4C000E091D109F091D20919950E942469182FA1
:10C4D000C091130AD091140AFE0119950F900F9084
:10C4E0000F900F90892B49F0FE011995BC0180E84F
:10C4F00090E00E94BE86EB0102C0C0E8D0E00E943E
:10C50000F8671F921F93DF93CF931F928F938091B1
:10C51000060A8F938091050A8F938091DE098F938D
:10C520008091DD098F938CE292E19F938F930E941B
:10C5300037928FE192E19F938F930E9437928EE022
:10C5400092E19F938F930E94379260E070E087EDB5
:10C5500092E00E94006F89E199E00E945F6B86E0A3
:10C5600092E19F938F930E9437928DB79EB7429628
:10C570000FB6F8949EBF0FBE8DBFDF91CF911F9174
:10C58000089580E880936100109261000E94D86154
:10C59000C4EFD1E103EE11E182EDE82E81E1F82E46
:10C5A00091ECC92E91E1D92E23EBA22E21E1B22EDE
:10C5B00004B600FE06C0DF93CF930E9437920F901F
:10C5C0000F9004B601FE06C01F930F930E9437928E
:10C5D0000F900F9004B602FE06C0FF92EF920E94E9
:10C5E00037920F900F9004B603FE06C0DF92CF92F1
:10C5F0000E9437920F900F9004B604FE06C0BF92BF
:10C60000AF920E9437920F900F9014BE0E946E6EF0
:10C610000E943665CDCFDF92EF92FF920F931F936A
:10C62000CF93DF93CDB7DEB7A0970FB6F894DEBFF8
:10C630000FBECDBF83E690E00E94FC94182F282FF8
:10C6400035EF380F303108F0982F9095291709F4FD
:10C6500063C089ED92E19F938F930E943792EEE140
:10C66000F3E18E010F5F1F4F0F900F90D801D02E76
:10C67000E12EF02E88E0800F94919D9331968A13DD
:10C68000FBCFF89448E050E06FE770E0C8010E94EB
:10C690000295E0E1F3E1D8018EE08F0D94919D9336
:10C6A00031968A13FBCF4EE050E061E770E0C8019D
:10C6B0000E940295E6E0F3E12AE02F0D8491D80173
:10C6C0008D938D0131962A13F9CF4AE050E067E649
:10C6D00070E08D2D9E2D0E9402956DEC7BEA81E627
:10C6E00090E00E941A9560E070E08FE590E00E9473
:10C6F0001A9560E08EE590E00E940C9560E070E095
:10C7000085E690E00E941A951AE16AE175EE83E6EB
:10C7100090E00E941A957894812FA0960FB6F89415
:10C72000DEBF0FBECDBFDF91CF911F910F91FF9064
:10C73000EF90DF9008958FE590E00C94FC948EE5E7
:10C7400090E00C94F494F8941092B60016BC89E72B
:10C7500087BD82E084BD95E095BD95B395BB809380
:10C760006E00789408950F931F9360918F137091CA
:10C770009013809191139091921300918F131091C7
:10C7800090132091911330919213601771078207D3
:10C79000930759F71F910F9108950F931F9360917D
:10C7A0009735709198358091993590919A3500918F
:10C7B0009735109198352091993530919A356017B9
:10C7C00071078207930759F71F910F9108951F92E0
:10C7D0000F920FB60F9211240BB60F922F933F9327
:10C7E0004F935F936F937F938F939F93AF93BF9379
:10C7F000EF93FF9380918F1390919013A0919113D9
:10C80000B09192130196A11DB11D80938F13909347
:10C810009013A0939113B093921380918E138F5F16
:10C8200080938E1387FF15C010928E1380919735D9
:10C8300090919835A0919935B0919A350196A11DA6
:10C84000B11D8093973590939835A0939935B09307
:10C850009A35809136378823E1F080918D138F5F70
:10C8600080938D1387FF15C010928D1380918F35A3
:10C8700090919035A0919135B09192350196A11D7E
:10C88000B11D80938F3590939035A0939135B093DF
:10C8900092350E946B6D892B11F00E948C6CFF9178
:10C8A000EF91BF91AF919F918F917F916F915F9128
:10C8B0004F913F912F910F900BBE0F900FBE0F9095
:10C8C0001F9018951F920F920FB60F9211240BB65E
:10C8D0000F922F933F934F935F936F937F938F9319
:10C8E0009F93AF93BF93EF93FF938091C600E09126
:10C8F0009D35F0919E35309709F01995FF91EF9194
:10C90000BF91AF919F918F917F916F915F914F9167
:10C910003F912F910F900BBE0F900FBE0F901F9065
:10C9200018951F920F920FB60F9211240BB60F920B
:10C930002F933F934F935F936F937F938F939F9327
:10C94000AF93BF93EF93FF938091CE00E0919B351F
:10C95000F0919C35309709F01995FF91EF91BF91B7
:10C96000AF919F918F917F916F915F914F913F9187
:10C970002F910F900BBE0F900FBE0F901F90189528
:10C9800081110EC01092C5006093C40088E98093A5
:10C99000C1004093C20010929E3510929D350895BB
:10C9A000813069F41092CD006093CC0088E98093C7
:10C9B000C9004093CA0010929C3510929B3508958F
:10C9C000811107C08091C00085FFFCCF6093C60035
:10C9D0000895813031F48091C80085FFFCCF6093C9
:10C9E000CE000895CF93C82F8A3031F46DE0809146
:10C9F00093130E94E06402C08D3029F06C2F809167
:10CA000093130E94E06480E090E0CF91089581113B
:10CA100005C070939E3560939D350895813021F453
:10CA200070939C3560939B3508958093931383E9AD
:10CA300092E09093E2398093E139089584B7877F3B
:10CA400084BF88E10FB6F894809360001092600074
:10CA50000FBE08952FE088E190E00FB6F894A895F6
:10CA6000809360000FBE209360000895A8950895FC
:10CA700088E10FB6F89480936000109260000FBEBA
:10CA800008950C94D38D0C94CF8D8091A43590E0B3
:10CA900008958091390181FF09C0809139018D7F0E
:10CAA0008093390189E190E00197F1F723E040E0BC
:10CAB0006FE182E491E00E947F6A85E090E0019757
:10CAC000F1F708959091390191FD0AC0282F803126
:10CAD00008F02FE040E06FE085E491E00C947F6A7D
:10CAE00008958091390181FD0EC040E06FE181E43D
:10CAF00091E00E94746A282F2F7E81E090E021301F
:10CB000021F080E0089580E090E00895809139015F
:10CB100081FF02C081E0089540E06FE181E491E08F
:10CB20000E94746A8F3121F08F7E8150823090F79D
:10CB300080E008958091390181FD04C00E948665DE
:10CB40008823C1F30895109236378091390181FD11
:10CB50008BC00E949A658091390181FD85C00E9439
:10CB600049658091390182608093390180916E37E7
:10CB70008823D9F1809194009091950040917F375E
:10CB80005091803784179507A0F480914B3790918E
:10CB90004C37A0914D37B0914E37875F924CAF4FD5
:10CBA000BF4F80934B3790934C37A0934D37B09342
:10CBB0004E372091940030919500241B350B8091C5
:10CBC0004B3790914C37A0914D37B0914E37820F33
:10CBD000931FA11DB11D80934B3790934C37A093A9
:10CBE0004D37B0934E3710926E378091703788234F
:10CBF000D9F18091940090919500409183375091A4
:10CC0000843784179507A0F4809153379091543757
:10CC1000A0915537B0915637875F924CAF4FBF4FB9
:10CC20008093533790935437A0935537B09356372A
:10CC30002091940030919500241B350B809153373F
:10CC400090915437A0915537B0915637820F931F6A
:10CC5000A11DB11D8093533790935437A09355373E
:10CC6000B0935637109270370895809136378823E5
:10CC700021F00E9486650E94A36580E090E00895FF
:10CC800022E0260F27FF0CC0809134379091353772
:10CC9000019690933537809334378FEF9FEF089547
:10CCA000AB01BC0184E993E10E94689180E090E0CF
:10CCB000089540E06FE181E491E00C94746A282FBC
:10CCC00040E06FEF86E591E00E947F6A0895CF9380
:10CCD000DF9398EF980F923038F0982F9F7E963020
:10CCE00019F0893109F049C09091390191FD48C08E
:10CCF000C82F0E949A650E945966D82FC81709F458
:10CD000042C0C83029F4809139010E94496527C08A
:10CD1000C93119F4863181F404C0C63169F489310E
:10CD200059F429E040E06FE182E491E00E947F6ADB
:10CD300085E090E00197F1F72C2F40E06FE182E46D
:10CD400091E00E947F6AD83031F48FEF0E945F66D5
:10CD500081ED92E002C085E090E00197F1F70E943A
:10CD600059668C1781F0C63019F4813079F40BC004
:10CD7000C63161F4813151F406C082E490E008C00C
:10CD800084E490E005C080E490E002C083E490E099
:10CD9000DF91CF91089580919400909195009093A8
:10CDA00084378093833781E0809370378093363760
:10CDB0009091390191FF1EC020919400309195000F
:10CDC0003093803720937F3780936E37809331374D
:10CDD0002FB7789480913901809139018D7F8093AC
:10CDE000390180E197E230913137332311F0019717
:10CDF000D1F72FBF86E10E9467660C949A658091F7
:10CE00003637811102C00E94CB6681E090E0089520
:10CE10000F931F93CF93DF931F92CDB7DEB780910F
:10CE20003637882361F08091390181FF02C080E0AC
:10CE30007BC00E9486658823D1F300E003C00E9476
:10CE4000FF6601E0809194009091950090937E3769
:10CE500080937D3711E010936D3780E88093550102
:10CE600086E00E9467661093A5358FB78983789412
:10CE7000109247018091A5358111FCCF89818FBF28
:10CE80008091470111E08E3008F010E0119586E1A5
:10CE90000E9467661092550180916D378823D9F101
:10CEA000809194009091950040917D3750917E370C
:10CEB00084179507A0F48091473790914837A09147
:10CEC0004937B0914A37875F924CAF4FBF4F80933D
:10CED000473790934837A0934937B0934A3720910A
:10CEE000940030919500241B350B80914737909129
:10CEF0004837A0914937B0914A37820F931FA11D3F
:10CF0000B11D8093473790934837A0934937B0932A
:10CF10004A3710926D3701110E943566812F829534
:10CF2000869586958370817090E00F90DF91CF9108
:10CF30001F910F9108958FEF80934E0121E044E0FF
:10CF400060EF8CE691E00E947F6A25E041E06EE0B0
:10CF50008CE691E00E947F6A80E880936F01809167
:10CF6000460180936D0121E045E060E284E491E0B8
:10CF70000C947F6ACF93DF93C9EFD7E0CE0101977E
:10CF8000F1F70E94736A1092AB3510922D36109211
:10CF9000AF361092AA351092A935E9E3F1E080810D
:10CFA0008E7F808380818D7F808381EC93E00197E9
:10CFB000F1F780818160808323E040E06FE182E4CB
:10CFC00091E00E947F6A2197F1F780915D01809145
:10CFD0005E010E949B6760E070E081EA92E00E943F
:10CFE000006F0E94CB6681E090E0DF91CF910895C1
:10CFF000809115140895CF93DF931F92CDB7DEB7BC
:10D0000089830E949A65898180931514282F40E0B6
:10D010006FE188E491E00F90DF91CF910C947F6AEB
:10D020000E94FB6786E00C946766EF92FF920F9375
:10D030001F93CF93DF931F921F92CDB7DEB78C0162
:10D040007A017F936F931F938F9387E699E09F9365
:10D050008F9369837A830E942392009362011093D5
:10D0600063016981609360017A81709361010F901F
:10D070000F900F900F900F900F90E114F104C9F0F2
:10D08000F701808180936B01818180936A018281A5
:10D090008093690183818093680184818093670113
:10D0A0008581809366018681809365018781809365
:10D0B00064010F900F90DF91CF911F910F91FF901E
:10D0C000EF90089581EA92E00E94216F81E08093C1
:10D0D000A4358091A6359091A73501969093A735F8
:10D0E0008093A63581E090E008950F931F93CF932E
:10D0F0002091AA35C2E8C29F90011124F901E5559B
:10D10000FA4C4081442309F451C047FD09C0433023
:10D1100038F050E08A01025011096017710710F4CD
:10D12000108244C0B90164557A4C0E946891809184
:10D13000AA35C89FF0011124E555FA4CDF01A0582B
:10D14000BF4F9C9190939F3510828F5F833018F46E
:10D150008093AA3502C01092AA35E091AA3582E8E0
:10D16000E89FF0011124E555FA4C8081882319F0DD
:10D170000E94626802C01092A4358091470180939A
:10D18000A0359091A335992311F0891710F480935D
:10D19000A3356091A03570E084E00E941C7460911A
:10D1A0009F3570E083E00E941C7402C000E010E034
:10D1B000C801CF911F910F9108950F931F93CF93A3
:10D1C000DF931F92CDB7DEB78C01FC018081918186
:10D1D000009709F18334954029F0F80111821082FB
:10D1E00083E02AC06238E1F40E94C8738FB7898354
:10D1F000F8940E94377360E870E00E947568298196
:10D200002FBF1816190674F40E943273E0910D0AAC
:10D21000F0910E0A199583E495E0F80191838083DB
:10D2200081E00AC08091A1359091A235019690933A
:10D23000A2358093A135EFCF0F90DF91CF911F9151
:10D240000F9108950C9462658091390181FD06C0AB
:10D2500040E06FE085E491E00C94746A80E1089509
:10D26000EF92FF921F93CF93DF931F92CDB7DEB75C
:10D27000182F8091390181FD07C00E949A65809125
:10D28000363781111CC05AC080919400909195004E
:10D290009093803780937F3781E080936E378093BF
:10D2A0003137809139018D7F8093390180E197E298
:10D2B00020913137222309F30197D1F7DECF8091F6
:10D2C00070378823D9F18091940090919500409116
:10D2D00083375091843784179507A0F48091533792
:10D2E00090915437A0915537B0915637875F924C43
:10D2F000AF4FBF4F8093533790935437A093553718
:10D30000B09356372091940030919500241B350B33
:10D310008091533790915437A0915537B09156373B
:10D32000820F931FA11DB11D8093533790935437E3
:10D33000A0935537B09356371092703789E10E9409
:10D34000676686E00E942774892B51F00E94246949
:10D35000E82E86E00E94277481500E94626502C018
:10D36000E12CF12C8091940090919500909382375C
:10D370008093813781E080936F378FB78983F894EA
:10D3800080913901826080933901809139018D7FCC
:10D390008093390162E0610F84E993E10E94C66ADB
:10D3A00089818FBF80913237909133370196909366
:10D3B0003337809332370E949A6545E060EE82E40D
:10D3C00091E00E94746A182F86E00E942774892BCE
:10D3D00019F08E2D0E94626580916F378823D9F1F4
:10D3E00080919400909195004091813750918237BF
:10D3F00084179507A0F480914F3790915037A091F2
:10D400005137B0915237875F924CAF4FBF4F8093E7
:10D410004F3790935037A0935137B09352372091A4
:10D42000940030919500241B350B80914F379091DB
:10D430005037A0915137B0915237820F931FA11DE1
:10D44000B11D80934F3790935037A0935137B093CD
:10D45000523710926F3780913637882371F0809160
:10D46000940090919500909384378093833781E066
:10D47000809370370E94CB6602C00E94A365123071
:10D4800028F48CE00E94277410E00BC0133031F0B8
:10D49000153031F0173029F411E003C012E001C05B
:10D4A00013E0812F90E00F90DF91CF911F91FF90BB
:10D4B000EF900895CF93DF93EB010E9440660097B1
:10D4C00029F4CE010E943069009751F02091343741
:10D4D000309135372F5F3F4F3093353720933437B6
:10D4E000DF91CF9108950895FC0180816823862FF4
:10D4F00090E002C0959587954A95E2F70895CF93FD
:10D50000DF931F92CDB7DEB7FC01922F8FB78983CF
:10D51000F8942081362F3095522F5323292F01C0A4
:10D52000220F4A95EAF72623252B208389818FBF76
:10D530000F90DF91CF910895CF93DF93E0917B011E
:10D540002DEF2E0F2D3740F0FC011082E058FF4FD9
:10D5500010823196108217C0EC01E993A0E8B1E087
:10D5600020E82E0F3C91399311962A13FBCFE150FE
:10D57000F0E0E058FE4F2181FC01E058FF4F20838E
:10D58000319681E08083DF91CF910895609380018F
:10D59000E1E8F1E06158DC012D91CD012083319665
:10D5A0006E13F9CF08951F920F920FB60F921124A8
:10D5B0000BB60F922F933F934F935F936F937F938D
:10D5C0008F939F93AF93BF93EF93FF938091470106
:10D5D0008093A0358091A93522E8829FC001112453
:10D5E00085559A4C0E949C6A8091A9358F5F833043
:10D5F00018F48093A93502C01092A9350E94626880
:10D60000FF91EF91BF91AF919F918F917F916F911A
:10D610005F914F913F912F910F900BBE0F900FBED6
:10D620000F901F9018951F920F920FB60F92112412
:10D630000F900FBE0F901F9018951F920F920FB66C
:10D640000F9211240F900FBE0F901F9018951F92EC
:10D650000F920FB60F9211240F900FBE0F901F90D4
:10D6600018951F920F920FB60F9211241092313716
:10D670000F900FBE0F901F9018951F920F920FB62C
:10D680000F9211241092A8350F900FBE0F901F908B
:10D6900018951F920F920FB60F9211240F900FBE84
:10D6A0000F901F9018951F920F920FB60F92112492
:10D6B0001092A5350F900FBE0F901F901895CF9325
:10D6C000DF93EC0189919991009729F060E070E077
:10D6D0000E94006FF7CFDF91CF910895EF92FF92F4
:10D6E0000F931F93CF93DF938C017A01FC0180810C
:10D6F0009181009741F08A34910511F1F80111826E
:10D70000108283E04AC087E194E10E94AB6FEC0194
:10D71000209761F04E815F8168857985CE01029600
:10D720000E94426D0990D881C02DF2CF81E0809394
:10D7300016148AE490E0F8019183808381E02DC083
:10D740006838E1F787E194E10E94AB6FEC01209724
:10D7500081F3CE010296E816F906D9F4BE0187E1FD
:10D7600094E10E94CB6FE090CB14F090CC148E85A6
:10D770009F859093CC148093CB14E889F9893097D6
:10D7800019F08A899B891995F092CC14E092CB14F8
:10D79000D0CF0990D881C02DDACFDF91CF911F91E2
:10D7A0000F91FF90EF9008951092161487E194E185
:10D7B0000E94A76F60E070E08BEA92E00C94006F2B
:10D7C000EF92FF920F931F93CF93DF93EC01E090C2
:10D7D000CB14F090CC14FF86EE86398B288B1B8BF4
:10D7E0000A8B80911614882379F08BEA92E090934B
:10D7F000CC148093CB14CE0102960E94426DF0921D
:10D80000CC14E092CB1404C04E835F836887798781
:10D81000BE0187E194E10E94CB6FBE0187E194E1F4
:10D82000DF91CF911F910F91FF90EF900C94E66FD5
:10D83000CF93DF93EC0180911614882329F0CE0159
:10D8400002960E94766D04C01B861A861D861C8671
:10D85000BE0187E194E1DF91CF910C94CB6FCF9221
:10D86000DF92EF92FF920F931F9380911D1490917E
:10D870001E14892B49F41092191410921A14109244
:10D880001B1410921C1441C00E94B3638B019C01B5
:10D89000E0911D14F0911E144481558166817781B9
:10D8A00080819181A281B381840F951FA61FB71F2C
:10D8B000801B910BA20BB30B0084F185E02D3097F8
:10D8C000C1F0C480D580E680F780408151816281BB
:10D8D00073814C0D5D1D6E1D7F1D401B510B620B36
:10D8E000730B481759076A077B0730F7DB01CA013A
:10D8F000E3CF800F911FA21FB31F80931914909341
:10D900001A14A0931B14B0931C141F910F91FF9035
:10D91000EF90DF90CF90089585EB92E00C94216F0B
:10D92000EF92FF920F931F93CF93DF938C01FC0133
:10D9300080819181009799F089359105D9F0F8019E
:10D940001182108283E068C08285938584179507D1
:10D9500009F049C00084F185E02D3097A9F71092B5
:10D960001E1410921D1489E590E0F80191838083C4
:10D9700081E052C0673891F16238A9F7C0911D1457
:10D98000D0911E14E12CF12C209769F3CE010E9456
:10D990007C6F892BF1F0AE0168E88A859B850E9437
:10D9A000D26E892BA1F41B861A8688859985E1148D
:10D9B000F10421F0F7019187808704C090931E1431
:10D9C00080931D14198618860E942F6CD7CF0E9451
:10D9D0008C6C7E010884D985C02DD6CFE0911D14B2
:10D9E000F0911E14BACFF0931E14E0931D14A0857D
:10D9F000B185109709F4B7CF1A968D919C911B971A
:10DA00008417950739F418968D919C9119979187F1
:10DA10008087EDCFFD01EBCFDF91CF911F910F916B
:10DA2000FF90EF900895CF93DF93EC010E948C6CF0
:10DA30002A853B8590911D1480911E14232B91F013
:10DA4000E92FF82F309771F0EC17FD0739F480912A
:10DA5000CB149091CC149387828710C00084F185F9
:10DA6000E02DF0CF2091CB143091CC143B872A8746
:10DA700098878987D0931E14C0931D14DF91CF918E
:10DA80000C942F6CCF93DF93EC010E944E6FCE016C
:10DA9000DF91CF910C94136DCF93DF93EC010E9433
:10DAA0005E6FCE01DF91CF910C94136DCF93DF9316
:10DAB000EC010E94706FCE01DF91CF910C94136D39
:10DAC00021E030E0FC0182859385892B11F020E074
:10DAD00030E0C901089581E090E020911D1430915B
:10DAE0001E14232B11F480E090E00895CF93DF9370
:10DAF000EC01E0911D14F0911E148E179F0769F43C
:10DB00008885998590931E1480931D140DC080857F
:10DB100091858C179D0721F0FC013097C1F706C055
:10DB200088859985918780870E942F6C1986188631
:10DB30001B861A86DF91CF9108951F93CF93DF93B1
:10DB4000DC011496ED91FC9115973097E1F0162FBA
:10DB5000EC019093CC148093CB1482E08887CD01A4
:10DB600006961995082E000C990B0297029710F053
:10DB7000133839F4BE01CE01DF91CF911F910C947F
:10DB8000CD6D81E08887DF91CF911F910895FC01D1
:10DB9000208520FD0C949D6D0895CF92DF92EF9229
:10DBA000FF920F931F93CF93DF93E090CB14F090ED
:10DBB000CC14C090CD14D090CE14F601E817F9071C
:10DBC00039F0309709F44BC00190F081E02DF6CF89
:10DBD000009709F444C08B01EC018885882309F182
:10DBE0001886C114D10461F0CC15DD0529F0AE0111
:10DBF00067E8C6010E94C76DF601C080D180F1CFF1
:10DC0000EC81FD81309769F0C017D10751F0D093B6
:10DC1000CC14C093CB1440E050E063E8CE010696EC
:10DC20001995E091CD14F091CE14CE17DF0741F491
:10DC3000888199819093CE148093CD140CC0FC01FF
:10DC4000309749F0808191818C179D07C1F78881B9
:10DC5000998191838083F092CC14E092CB14DF9170
:10DC6000CF911F910F91FF90EF90DF90CF9008958B
:10DC70001F93CF93DF9310922714C091CD14D091AE
:10DC8000CE1411E0209779F08985882341F0188718
:10DC9000198640E050E062E8CE010E949D6D099037
:10DCA000D881C02DEFCFDF91CF911F910895809142
:10DCB000CA1491E0980F9093CA1408958AE880934B
:10DCC000CA141092C8141092C9141092CE14109253
:10DCD000CD141092CC141092CB1408958091271477
:10DCE00081110E94386E5091C914552309F452C015
:10DCF000E091C8142E2F30E085E0E89FF001112458
:10DD0000E85DFB4E608160932614A181B281B093DF
:10DD10002514A093241483819481909323148093D9
:10DD200022142F5F3F4F2F7133272093C814515077
:10DD30005093C914009731F58091CD149091CE1471
:10DD40009093211480932014809120149091211499
:10DD5000892B01F18091271481110E94386E409126
:10DD600024145091251460912614809120149091D0
:10DD700021140E94C76DE0912014F091211480813C
:10DD80009181DECF613819F421E0FC012087AD01DB
:10DD90000E94C76D809127142091C91490E0820FD2
:10DDA000911D08959C019091C9149032B9F0E091B1
:10DDB000C814E90FEF71E0931F1485E0E89FF001AC
:10DDC0001124E85DFB4E60835283418334832383B7
:10DDD0009F5F9093C91480E090E0089581E090E007
:10DDE0000895CF93DF93C091CB14D091CC140E94AF
:10DDF000C76DD093CC14C093CB14DF91CF9108950D
:10DE0000AB013091CD142091CE14E32FF22FE817FF
:10DE1000F907B1F0309721F00190F081E02DF7CFB4
:10DE2000009771F0FC01308321839093CE1480938E
:10DE3000CD1421E020871782168261E80C94F16EE0
:10DE40000895009749F0FC0120852150223020F4EC
:10DE500021E021872093271408950C94567880910F
:10DE6000CF149091D0140097C1F01092D01410925A
:10DE7000CF14DC0114966D917C9115971296ED915B
:10DE8000FC9113971995E091CF14F091D01430972D
:10DE900021F0808191810C9470780895CF93DF9365
:10DEA000EC014C835D836E837F830E94B363688340
:10DEB00079838A839B83DF91CF910895FC01408110
:10DEC00051816281738184819581A681B781840F9C
:10DED000951FA61FB71F80839183A283B3830895E4
:10DEE000CF93DF93EC010E94B363688379838A83C5
:10DEF0009B83DF91CF910895CF92DF92EF92FF92B3
:10DF0000CF93DF93EC010E94B363C880D980EA808D
:10DF1000FB80DC01CB018C199D09AE09BF0901967C
:10DF2000A11DB11D21E030E0CC80DD80EE80FF80BE
:10DF3000C816D906EA06FB0610F020E030E0C90159
:10DF4000DF91CF91FF90EF90DF90CF900895FC018B
:10DF5000118210820895FC01808191810895DC0175
:10DF6000ED91FC91309731F080819181009729F0FB
:10DF7000FC01FACF80E090E00895CF010895DC0124
:10DF8000ED91FC911197309721F0208131812D93F3
:10DF90003C93CF010895DC01ED91FC913097A9F0FD
:10DFA000A0E0B0E020813181E617F70741F4109737
:10DFB00009F4DC012D933C93118210820895211500
:10DFC000310519F0DF01F901EDCF08950F931F938B
:10DFD000CF93DF938C01EB010E94CB6F19821882E3
:10DFE000C8010E94AF6F009711F4F80101C0FC0155
:10DFF000D183C083DF91CF911F910F910895DC01F0
:10E00000ED91FC9180E090E0309729F0019601902D
:10E01000F081E02DF9CF0895009721F0FC01808177
:10E020009181089580E090E00895CF93DF93EC0113
:10E030004A815B8160E070E08C819D810E947191DA
:10E040002A813B8188819981289FA001299F500DB9
:10E05000389F500D112460E070E08E819F81DF9128
:10E06000CF910C947191FC018281938120E030E08A
:10E0700028173907D1F0A481B581A20FB31F4C91A5
:10E08000411110C081E08C9380819181289FA00173
:10E09000299F500D389F500D112486819781840F40
:10E0A000951F08952F5F3F4FE3CF80E090E00895E4
:10E0B000FC01868197814281538120E030E0241762
:10E0C0003507D1F08617970781F4A481B581A20F97
:10E0D000B31F8C91181614F481508C938481958110
:10E0E000FC01E20FF31F80810895A081B1818A0FA6
:10E0F0009B1F2F5F3F4FE3CF8FEF0895FC012681D9
:10E10000378162177307A0F0A081B18142815381EA
:10E11000A49FC001A59F900DB49F900D1124280FBE
:10E12000391F81E090E06217730720F080E00895C6
:10E1300080E090E008952F923F924F925F926F920D
:10E140007F928F929F92AF92BF92CF92DF92EF9287
:10E15000FF920F931F93CF93DF93CDB7DEB76897EE
:10E160000FB6F894DEBF0FBECDBFE7E3F7E324A5FB
:10E1700035A546A557A550A441A432A423A4948C48
:10E18000858C768C678C808D8983918D9A83828D26
:10E190008B83938D9C8384898D8395899E838689C7
:10E1A0008F83978998878089898791899A878289BF
:10E1B0008B8793899C8784858D8795859E878685A7
:10E1C0008F879785988B8085898B91859A8BB28470
:10E1D000A384F480E580D680C78080818F8B918175
:10E1E000988F128103812B8B3C8B4D8B5E8B0E9411
:10E1F000CD635E895F934D894F933C893F932B8913
:10E200002F932F923F924F925F926F927F928F92B5
:10E210009F922C812F932B812F932A812F932981D9
:10E220002F9328852F932F812F932E812F932D812C
:10E230002F932C852F932B852F932A852F93298518
:10E240002F9328892F932F852F932E852F932D85FC
:10E250002F93AF92BF922A892F9329892F93CF9220
:10E26000DF92EF92FF920F931F93288D2F932F89A8
:10E270002F939F938F937F936F93EDE8F7E38181C3
:10E280001F928F9380811F928F9386E293E19F93D9
:10E290008F930E9437920FB6F894DEBF0FBECDBFAA
:10E2A00068960FB6F894DEBF0FBECDBFDF91CF9159
:10E2B0001F910F91FF90EF90DF90CF90BF90AF90A4
:10E2C0009F908F907F906F905F904F903F902F9096
:10E2D0000895EF92FF920F931F93CF93DF938C01DA
:10E2E000EB017A010E94FF71F801F086E78260EC91
:10E2F00079E0CE01DF91CF911F910F91FF90EF90C8
:10E300000C9423720C9407720C94BB72DC01179668
:10E31000ED91FC9118970190F081E02D309709F074
:10E3200019940895DC011796ED91FC9118970280DD
:10E33000F381E02D309709F019940895DC011996C6
:10E34000ED91FC911A970280F381E02D309709F04E
:10E35000199408950F931F93CF93DF931F921F92E9
:10E36000CDB7DEB78C0188E10E943A74BC01CE01C2
:10E3700001960E94E972D8011996ED91FC911A97C5
:10E380000190F081E02D309729F0BE016F5F7F4F43
:10E39000C80119950F900F90DF91CF911F910F91A8
:10E3A0000895EF92FF920F931F93CF93DF938C0109
:10E3B000EB017A0142EC59E00E946971F801F286A2
:10E3C000E18666EC79E0CE01DF91CF911F910F914C
:10E3D000FF90EF900C9423720C948271CF93DF9393
:10E3E000EC016DE877E388E10E943074CE01DF91A3
:10E3F000CF910C94847181ED94E10C94A76FFC0192
:10E4000073836283BC0181ED94E10C94E66FBC01DF
:10E4100081ED94E10C94CB6FCF93DF93EC0181ED10
:10E4200094E10E94AB6F009749F0FC012281338197
:10E430002C173D0729F00E940C70F5CF80E090E08A
:10E44000DF91CF9108950F931F93CF93DF938B01AB
:10E450000E940C72EC01892B31F01D830C83C801E2
:10E460000E9423828E83DF91CF911F910F91089597
:10E47000CF92DF92EF92FF920F931F93CF93DF9390
:10E480007C018B016A0183ED94E10E94AB6FEC018A
:10E49000892B51F0EC81FD81309711F0C80119955D
:10E4A000CE010E940C70F3CFA601B801C701DF9125
:10E4B000CF911F910F91FF90EF90DF90CF900C9430
:10E4C00092710F931F93CF93DF931F921F92CDB73B
:10E4D000DEB70E94F5818C0183ED94E10E94AB6F61
:10E4E000009779F0DC011296ED91FC91139730972B
:10E4F00029F089839A8319959A8189810E940C70E9
:10E50000EFCF0115110549F0C8010F900F90DF9171
:10E51000CF911F910F910C9486710F900F90DF9106
:10E52000CF911F910F910895CF92DF92EF92FF92BA
:10E530000F931F930E9440740E94C8730E948A80A8
:10E540000E94F381C12C88E0D82E87E0E82EF12CC0
:10E5500000E01EE120E030E040E052E060E070E0EA
:10E5600082E090E00E94BA811F910F91FF90EF909E
:10E57000DF90CF900895CF93DF93EC010E94088243
:10E58000009761F00E945073E091E109F091E20977
:10E59000BE0188E392E7199581E090E0DF91CF9189
:10E5A0000895E091090AF0910A0A1994E091D309BB
:10E5B000F091D4091994E0910F0AF091100A19947E
:10E5C000E091110AF091120A199480E090E0089508
:10E5D0000895FB0120813181FC013183208308955E
:10E5E00042E050E00E945B9121E030E0892B11F085
:10E5F00020E030E0C9010895BC018DE897E30C9458
:10E60000E972E0919109F09192091995E091070A58
:10E61000F091080A1995E091DF09F091E009199548
:10E62000E091D109F091D209199420918C15309183
:10E630008D152817390798F040918A1550918B1540
:10E64000480F591F50938B1540938A15281B390B7F
:10E6500030938D1520938C1581E090E0089580E033
:10E6600090E0089590938D1580938C150895809176
:10E670008A1590918B15895F9A4E0895809189151E
:10E6800090E089529B4E089581E090E02091D5144E
:10E690003091D6142750354111F480E090E0089570
:10E6A0000E944473892B61F06091D5147091D61447
:10E6B00040918C1550918D1587E095E10C946891EF
:10E6C00020918A1530918B1521153105B9F0809173
:10E6D0008C1590918D15C096E7E0F5E1AF01475D8F
:10E6E00054414817590734F4DF01A20FB31F4C916E
:10E6F0004193F4CF10928B1510928A150895809152
:10E700008C1590918D1508958091891590E3981B33
:10E7100020918C1530918D15A901490F511DCA0109
:10E7200008950F931F93CF938C01C09189158C2F5F
:10E7300090E0801791076CF00E948473800F911F06
:10E740008138910530F4C01BC093891581E090E0B9
:10E7500002C080E090E0CF911F910F910895CF9378
:10E76000DF93E7E9F7E31192119287E3E73CF807BB
:10E77000D1F7CFE8D7E36BEE79E0CE010E94E972E2
:10E78000229687E3C739D807B1F7DF91CF91089573
:10E7900010928B1510928A1510928D1510928C156F
:10E7A00080E38093891587E095E19093D614809358
:10E7B000D5140C94AF73EF92FF920F931F93CF93E6
:10E7C000DF931F921F92CDB7DEB78C0169837A83E6
:10E7D0000E94C8736981E62E7A81F72E81E8E816D7
:10E7E000F10418F080E8E82EF12CA701B80180911F
:10E7F000D5149091D6140E946891F0928D15E092F4
:10E800008C15C7010F900F90DF91CF911F910F9141
:10E81000FF90EF900895FC0190E3A7E9B7E3019022
:10E820000D929A95E1F788E0FB01AFE8B7E301901C
:10E830000D928A95E1F70895E82FF0E0EE0FFF1FA3
:10E84000E956F84C7183608381E090E00895E82FE9
:10E85000F0E0EE0FFF1FE956F84C8081918108959A
:10E8600090E0880F991F815A984C0E94E97281E0CC
:10E8700090E0089590E0880F991F815A984C089570
:10E880008FEB92E00E9415708FEC92E00E94157061
:10E8900087EC92E00C9415700F931F93CF93DF9346
:10E8A000EC01BC018FEC92E00E947E70892BA9F0F4
:10E8B0000990D881C02DFE0161917191CF010E9414
:10E8C000DB73BE016E547F4FCE018E579F4FDF9199
:10E8D000CF911F910F910C940B74BE0187EC92E0C5
:10E8E0000E947E70892BD1F00E94C8736881798163
:10E8F0008A819B810E94DB738CA990E00E949173B6
:10E900000CA910E00E943E73BE016C5F7F4FA8010E
:10E91000DF91CF911F910F910C946891DF91CF916E
:10E920001F910F91089581E09CE10E94606D892BF9
:10E9300021F081E09CE10C94566D0895E091ED1B6F
:10E94000F091EE1B309709F0199480E00895EF9252
:10E95000FF920F931F93CF93DF938C01EA01FC0189
:10E9600080819181009741F08A33934081F1F801D1
:10E970001182108283E0F8C080E024E0829FF001E1
:10E980001124E151F44E118210828F5F8430A9F777
:10E990008093EC1B8091CB149091CC149093001C2D
:10E9A0008093FF1B0E94576E8093C73740E450E06E
:10E9B00060E070E081E09CE10E94426D0E94377946
:10E9C0008AE393E0F8019183808381E0CDC06230D7
:10E9D000D9F48091C8379091C937892B89F38091F8
:10E9E000D937863029F48091F13781FD0E949374E4
:10E9F00081E00E947E798091C8379091C937892B38
:10EA0000F9F20E940176DCCF633060F5611114C029
:10EA10002097B1F2D093C638C093C53883E00E94E6
:10EA20007E798091C8379091C937892B11F00E9467
:10EA30009E740E949374C4CF613011F6209709F43C
:10EA4000BFCFD093C238C093C13885E00E947E7991
:10EA50008091C8379091C937892B09F4B1CF0E94B2
:10EA60009E74AECF673809F040C01092EB1B8FEE5A
:10EA7000E82E8BE1F82E8091EB1B8430C0F4F70177
:10EA8000828193818C179D0749F4808191810E9436
:10EA90006379F7011182108213821282F4E0EF0E83
:10EAA000F11C8091EB1B8F5F8093EB1BE4CFE0EEBA
:10EAB000F8E3838194818C179D0719F414821382E3
:10EAC0001082B09629E3E036F20799F7EDE5F9E315
:10EAD000818592858C179D0711F4158214823D96CD
:10EAE00089E3EF3DF807A1F76BCF683809F068CFED
:10EAF000C150DC4109F064CF81E09CE10E94606D6F
:10EB0000892B09F45DCF1092EB1BE091EB1BE430F5
:10EB100008F056CF20E2E29FF0011124E953F74CB0
:10EB2000818D8823D9F081E09CE10E94566D80910F
:10EB3000EB1BE0E28E9FC00111248953974C909308
:10EB4000C6388093C53882E00E947E798091C837AC
:10EB50009091C937892B11F00E949E748091EB1B14
:10EB60008F5F8093EB1BD1CFDF91CF911F910F91DE
:10EB7000FF90EF900895CF93DF93A091C538B091A7
:10EB8000C638109719F0ED016C9605C0C091C138D8
:10EB9000D091C23829968091C03886FF23C0109248
:10EBA000EA1B80E0EFEEFBE18430C1F0408151814F
:10EBB00014962D913C9115974217530761F42281C9
:10EBC00033812115310539F08093EA1B398328837D
:10EBD0001B821A8205C034968F5FE6CF8093EA1BB2
:10EBE0000E94937488819981009741F04A815B81EA
:10EBF0006091C737DF91CF910C94F16EDF91CF9187
:10EC000008950F931F93CF93DF938091D937863068
:10EC100009F07AC08091C8379091C937803F91053B
:10EC200008F472C08897EC01D695C7959E01220F13
:10EC3000331F8E012817390710F40F5F1F4FCE01C5
:10EC400088969093C9378093C8379093D237809332
:10EC5000D3371092F5371092F4370E9431798095AE
:10EC600090959093F5378093F4371092DB3710929C
:10EC7000DA370E942079809590959093DB378093C6
:10EC8000DA370E949E74C80188969093C9378093A2
:10EC9000C8379093D2378093D3378091C3389091FF
:10ECA000C438BC016C0F7D1FA8010E946891BE0191
:10ECB00088EE97E30E94CD788091CC378093E83737
:10ECC0008091CD378093E9378091CE378093EA37B2
:10ECD0008091CF378093EB371092F5371092F4374D
:10ECE0000E943179809590959093F5378093F43711
:10ECF0001092DB371092DA370E9420798095909538
:10ED00009093DB378093DA37DF91CF911F910F918A
:10ED10000C949E74E091A109F091A209199480E0ED
:10ED200090E00895AF92BF92CF92DF92EF92FF9260
:10ED30000F931F93CF93DF93CDB7DEB7E1970FB655
:10ED4000F894DEBF0FBECDBF7C016B01CE010196F2
:10ED50005C0181E3F50111928A95E9F781E08983ED
:10ED60008CE00E9427748C831D821F8280910D1C71
:10ED700091E0980F90930D1C898713E018878DEC14
:10ED80009BEA9B878A8789E10E943A746BEE79E05F
:10ED90000E94F072892B31F082E08E838FEF8C8796
:10EDA0008D8709C089E10E943A74BC01CE010C969E
:10EDB0000E94E9721E838DEC9BEA9D8B8C8B6DE823
:10EDC00077E3CE0146960E94E9720E9437739FA7AF
:10EDD0008EA70E947F7399AB88ABC5010E946B829E
:10EDE0008C011127C8010E949173892B31F10E9477
:10EDF0003E73A801BC01C5010E948E820091970953
:10EE0000109198090E9484735C010E943E73B501C1
:10EE1000F8011995E114F10481F0009739F0019798
:10EE200061F441E050E064E070E004C041E050E093
:10EE300060E070E0C601F7011995E1960FB6F8940D
:10EE4000DEBF0FBECDBFDF91CF911F910F91FF901D
:10EE5000EF90DF90CF90BF90AF9008950F931F93E6
:10EE6000CF93DF934115510579F0FA018B01EC0145
:10EE7000828193810E944C74B801CE01DF91CF91C1
:10EE80001F910F910C949276DF91CF911F910F916A
:10EE900008950F931F93CF93DF93CDB7DEB7E1971C
:10EEA0000FB6F894DEBF0FBECDBF0E947F738C01FA
:10EEB0000E943773AE014F5F5F4FB8010E9481839C
:10EEC000892B09F443C088A999A99801281B390BFB
:10EED000C9010E941573892BC9F18E8181110CC063
:10EEE000BE016A5E7F4F88E10E943074E091E309C1
:10EEF000F091E40919952AC02A853B852D3C9BEAAF
:10EF0000390719F02F3F3F4F09F5823019F088E09B
:10EF100090E002C082E090E0019710F3E1E0F0E0C1
:10EF2000EC0FFD1FE80FF91F23852F3FA9F3BE014A
:10EF3000645F7F4F89E10E94307489E10E943A74D6
:10EF40006DE877E30E94F072892B51F6E1960FB6D7
:10EF5000F894DEBF0FBECDBFDF91CF911F910F910F
:10EF600008950E94436580930D1CE091A109F091E2
:10EF7000A2091994892B29F0E091A109F091A20925
:10EF800004C0E091A309F091A4091994FC01680F51
:10EF9000791F80E048E1E617F70781F0219198E0BA
:10EFA000322F3827532F517030FD842786955130EA
:10EFB00009F480682695915099F7EDCF08951F9236
:10EFC0000F920FB60F9211240BB60F922F933F930F
:10EFD0004F935F936F937F938F939F93AF93BF9361
:10EFE000EF93FF93809194009091950090937A37DE
:10EFF0008093793781E080936B3780917100807DB9
:10F00000809371000E942F6F80916B378823D9F114
:10F0100080919400909195004091793750917A3782
:10F0200084179507A0F480913F3790914037A091C5
:10F030004137B0914237875F924CAF4FBF4F8093BB
:10F040003F3790934037A0934137B0934237209198
:10F05000940030919500241B350B80913F3790919F
:10F060004037A0914137B0914237820F931FA11DC5
:10F07000B11D80933F3790934037A0934137B093B1
:10F08000423710926B37FF91EF91BF91AF919F91F3
:10F090008F917F916F915F914F913F912F910F9041
:10F0A0000BBE0F900FBE0F901F9018959FB7F8944E
:10F0B000E1E7F0E08081807D808388B38F6288BB48
:10F0C00010929000E1E9F0E010821092920010920C
:10F0D0009500109294008081856080839FBF089581
:10F0E0009C019FB7F894309399002093980088B3BF
:10F0F0008F6288BBE1E7F0E08081826080839FBF00
:10F100000895FB0141505109460F571FE417F507B9
:10F1100078F4208130E0322F22276181260F311DC3
:10F12000820F931F8217930708F401963296EECF51
:10F13000E417F50751F4208130E0322F2227820FA7
:10F14000931F8217930708F401960895CF93DF93D6
:10F15000C091D337D0E064972091D23730E0322F7E
:10F160002227C20FD31F48E050E06CED77E39E01E9
:10F17000280F311DC9010E948178AE0164EE77E34A
:10F180000E948178009721F098278927982702C04C
:10F190008FEF9FEFDF91CF910895FC012381260F20
:10F1A0002093CF37A72FBB2792819A0F9093CE370A
:10F1B00031813093CD3740814093CC37E92FF0E057
:10F1C000EA17FB0748F481E0830F8093CD37811164
:10F1D00003C04F5F4093CC3730E0772726173707BF
:10F1E00088F49F5F9093CE3791110CC08091CD37FA
:10F1F0008F5F8093CD37811105C08091CC378F5FB1
:10F200008093CC3708952091C5383091C638BC0121
:10F21000C90108960E94CD78E091C538F091C638B2
:10F22000ACECB7E38C91808711968C911197818714
:10F2300012968C911297828713968C9183870895EA
:10F2400044E150E060ED77E380E090E00E94817857
:10F25000009721F098278927982708958FEF9FEF2F
:10F26000089586E00C94A67881E10C94A67880E05D
:10F27000E82FF0E0EE0FFF1FE95BF64C11821082E1
:10F280008F5F8430A9F780E090E2899FF00111241C
:10F29000E953F74C118E8F5F8430B1F780E094E032
:10F2A0009093131C8093121C80E09DE0989FF001C6
:10F2B0001124E35AF64C158214828F5F8A30B1F71D
:10F2C0008093111C08959C0190E09430A1F0E92FE7
:10F2D000F0E081E0890FEE0FFF1FE95BF64C408103
:10F2E00051814217530729F49093111C1182108207
:10F2F0000895982FEACF9093111C0895AF92BF9272
:10F30000CF92DF92EF92FF920F931F93CF93DF93F1
:10F31000C091C538D091C638843009F4DBC128EFDC
:10F3200037E33093C4382093C3383093CB372093DE
:10F33000CA37833059F4898D8F70833009F06AC0E1
:10F3400088899989892B09F0D4C67EC0823009F05A
:10F350007FC08091171C8F5F8093171C811113C091
:10F360008091161C8F5F8093161C81110CC08091B8
:10F37000151C8F5F8093151C811105C08091141C92
:10F380008F5F8093141C1092C9371092C837109267
:10F390005C3910925B39898D982F9D7F953041F4AF
:10F3A0008A8D8F5F8A8F843109F0A3C6198EA1C61A
:10F3B000882309F49EC628893989232B09F440C083
:10F3C0009A8D2FEF290F2A8F911193C69B8D98301C
:10F3D00031F02FEF280F223048F4953039F4198E90
:10F3E00080E88093C0380E94BB753DC5953038F4E5
:10F3F00023E0092E01C0220F0A94EAF701C020E39E
:10F400002A8F9F5F9B8F8F708330A1F048F48130EB
:10F4100009F444C3823009F06CC61092F13741C33D
:10F42000863009F4BCC4883009F4B9C4843009F0CA
:10F4300060C6B5C484E08093C0380E94BB7545C5E2
:10F440008F70833009F055C688E08093C03800C5BE
:10F45000853019F5E091C138F091C23884819581E9
:10F46000892B09F446C61092C6381092C5388CEE26
:10F4700097E39093C4388093C3389093CB378093AD
:10F48000CA3710925C3910925B391092C9371092CA
:10F49000C83788E08093C0381BC18091D03785344D
:10F4A00009F027C60091D23710E0102F0027809175
:10F4B000D337080F111D8091C8379091C937801735
:10F4C000910708F416C61093C9370093C837809186
:10F4D000D6378F7309F00DC6F090D737F11009C6F3
:10F4E0008091573990915839C091150AD091160AD8
:10F4F0008C179D0759F44091593950915A392091F0
:10F50000170A3091180A42175307A1F02091E037EB
:10F510003091E1372817390709F0EBC52091E23720
:10F520003091E3378091593990915A39281739072A
:10F5300009F0DFC50E942079019609F0DAC58091B3
:10F54000D937863009F429C18131E9F1813009F0D8
:10F55000D0C58091E437883009F0CBC51092E437EC
:10F560008091E6379091E737873F6FEF960710F06D
:10F57000099601C008969093E7378093E63780910B
:10F58000DC379091DD37A091DE37B091DF37809383
:10F59000E0379093E137A093E237B093E33780915F
:10F5A000573990915839A0915939B0915A3980936F
:10F5B000DC379093DD37A093DE37B093DF3780E4FC
:10F5C0008093D83773C50C5111091093C937009334
:10F5D000C8378CEE97E39093C4388093C3388091FA
:10F5E000EA379091EB37892B29F00E943479019604
:10F5F00009F07FC52091E6373091E73721153105B5
:10F6000009F477C58DE599E39093C2388093C138AA
:10F61000A090E437B090E5374091190A50911A0A4A
:10F6200060911B0A70911C0AA091DC37B091DD3704
:10F630000091DE371091DF37E090170AF090180A3A
:10F64000E091C138F091C23889E3EF3DF80708F046
:10F6500050C584819581009721F12817390709F554
:10F6600086819781009719F0A816B906D1F4808198
:10F6700091818C179D0729F4C280D380CE14DF04BA
:10F68000B1F08417950729F4C280D380C616D70637
:10F6900071F0A817B90729F4828193810817190717
:10F6A00031F03D96F093C238E093C138C9CF109243
:10F6B000C6381092C53882E08093C0388CEE97E34C
:10F6C0009093CB378093CA3710925C3910925B3994
:10F6D0000E94BB7580915B3990915C39009709F469
:10F6E00008C59C01245E3F4F3093C9372093C8372B
:10F6F0003093D2372093D337E091C138F091C2389C
:10F7000020852093D83721E12093D9370896982770
:10F71000892798279093E9378093E8371092EB3741
:10F720001092EA37848195819093E5378093E4378E
:10F73000868197819093E7378093E6378091573998
:10F7400090915839A0915939B0915A398093DC374A
:10F750009093DD37A093DE37B093DF3780819181BE
:10F76000A281B3818093E0379093E137A093E23791
:10F77000B093E33788EF97E39093C4388093C3380E
:10F780000E94347980959095009711F48FEF9FEF48
:10F790009093EB378093EA3789C40E9431790196C0
:10F7A00009F0A7C44091E6375091E737411551055C
:10F7B00009F49FC48091E4379091E537009709F4EC
:10F7C00098C46091DC377091DD37E091DE37F091BD
:10F7D000DF37C7ECD8E3298D2223A9F0AC81BD81A6
:10F7E0004A175B0781F4AE81BF818A179B0759F4E2
:10F7F000A881B9816A177B0731F4AA81BB81EA1716
:10F80000FB0709F466C1A09629E3C734D20719F7AC
:10F810008091F1378F738230D9F450930F1C40934D
:10F820000E1C80E0843091F0E82FF0E0EE0FFF1F17
:10F83000E95BF64C208131818F5F4217530791F7C6
:10F840001092111C80E0C0E0D0E07CC08093111CBD
:10F850008091F13782FD4DC484E18093F13788E2D5
:10F8600090E09093C9378093C83780E58093F03754
:10F870003091EB378091EF378093EB372091EA3767
:10F880008091EE378093EA372093EE379091E937F5
:10F890008091ED378093E9379093ED378091E83789
:10F8A0008093111C4091EC374093E8378093EC37FC
:10F8B0003F5F3093EF3731110DC02F5F2093EE374C
:10F8C000211108C09F5F9093ED37911103C08F5FA6
:10F8D0008093EC378091E4379091E53790930F1C3B
:10F8E00080930E1C2091E6373091E7373093E5374F
:10F8F0002093E4379093E7378093E6378091DC37A5
:10F900009091DD37A091DE37B091DF378093E037FB
:10F910009093E137A093E237B093E3378091573962
:10F9200090915839A0915939B0915A398093DC3768
:10F930009093DD37A093DE37B093DF379CC39730C9
:10F9400089F08F5F8430C1F060E2869F90011124BE
:10F95000F901E953F74C918D9111F1CF8093111C6E
:10F96000EF010CC0209721F0428D9A8D941748F733
:10F97000E901C953D74CE5CF8093111C209709F4B6
:10F98000B8C3D093C638C093C53883E08A8F888FB8
:10F990001E8A84E08F8B1B8E8091E6379091E7372B
:10F9A0009D838C838091E4379091E5379F838E838C
:10F9B0008091DC379091DD37A091DE37B091DF3751
:10F9C00088839983AA83BB8381E0898F8091141CEB
:10F9D0008C878091151C8D878091161C8E87809155
:10F9E000171C8F8781E090E0998B888B8091EB3793
:10F9F0008B878091EA378A878091E9378987809160
:10FA0000E837888781E090E00E9403798091F037A1
:10FA1000982F907F913508F441C082958F7090E0C7
:10FA20000597880F991F880F991F2091101CEF2DA3
:10FA3000F0E0E817F90774F5E053F84C20A5211120
:10FA400003C01092101C28C0213011F4F394EFCFA2
:10FA50002230D9F431A53430C1F42093101CF09237
:10FA6000111C82A590E0982F882723A5822B9093C4
:10FA70000F1C80930E1C893C910510F088EC90E0DF
:10FA80009B8B8A8B9D8B8C8B09C031A5332311F006
:10FA9000F30ECDCF2093101CF092111C80E18093C7
:10FAA000F1378091F13782608093F13782E0809363
:10FAB000F83784E08093F9371092FA3788EC809316
:10FAC000FB378CE290E09093C9378093C83780E68B
:10FAD00080C2D093C638C093C5381092C038809188
:10FAE000F137782F7470F72E82FF03C0198E80E2F1
:10FAF00019C29091F03792959F70990F990F90933A
:10FB0000111C091B1109045111091093C9370093E5
:10FB1000C837922F9F70923029F4982F9F7392319B
:10FB200039F41FC0913021F4982F9F739230C9F09F
:10FB3000012B19F4982F9370A1F02091E837988544
:10FB400029133DC22091E9379985291338C22091A4
:10FB5000EA379A85291333C22091EB379B85291305
:10FB60002EC284FF49C0688979896115710509F43D
:10FB700043C0CE010C960E94CD783091EC37809135
:10FB8000CC37381339C02091ED378091CD37281309
:10FB900033C09091EE378091CE3798132DC080916D
:10FBA000EF374091CF37841327C03C872D879E873E
:10FBB0008F878B8D811119C09E89888D2A8D821B1C
:10FBC000292F269526952695821B980F9E8B87FDBB
:10FBD00081952F89322F36953695231B820F8F8B77
:10FBE000969596959695890F888F81E08093C03879
:10FBF000888D8A8F198A188A298DE22FEF708E2FAF
:10FC000090E0FC013197E830F10508F072C28827D6
:10FC1000E656FF4F8F4F0C9427878091C03880FFA6
:10FC200014C083E0898F80E48093C038198A188AD1
:10FC30008091C8379091C937009709F405C122E433
:10FC40002093C0380E940379FFC08091F1378F73F1
:10FC5000823009F04EC222CF8091C03880FF6AC046
:10FC60008091F1378F73823109F064C08091F03751
:10FC7000982F907F913508F441C082958F7090E065
:10FC80000597880F991F880F991F2091101CEF2D41
:10FC9000F0E0E817F90774F5E053F84C20A52111BE
:10FCA00003C01092101C28C0213011F4F394EFCF40
:10FCB0002230D9F431A53430C1F42093101CF092D5
:10FCC000111C82A590E0982F882723A5822B909362
:10FCD0000F1C80930E1C893C910510F088EC90E07D
:10FCE0009B8B8A8B9D8B8C8B09C031A5332311F0A4
:10FCF000F30ECDCF2093101CF092111C83E0898F5E
:10FD00008091E83788878091E93789878091EA3741
:10FD10008A878091EB378B8781E090E00E9403799E
:10FD200082E48093C038198A188A1092C9371092D9
:10FD3000C8378AC080E28093C0380E94BB75E091CA
:10FD4000C538F091C638118E83CD8091F13780FF90
:10FD500028C024FD26C088899989892B09F0C9C14A
:10FD60008091C8379091C93701960E94037980919C
:10FD7000C038982F90619093C0382091C837309147
:10FD8000C937232B19F082618093C0380E94BB755C
:10FD900081E090E0998B888B88E0898F1B8E81E1D0
:10FDA0000FC185FF1DC08091F63790E0982F8827FE
:10FDB0003091F737832B4091C3385091C438480FA6
:10FDC000591F5093C4384093C3384091C83750915D
:10FDD000C937BA01681B790B7093C9376093C8376C
:10FDE0004091C8375091C9374115510551F024FD54
:10FDF00008C09091C03892609093C038CA010E94A8
:10FE000003798091F23790E0982F88272091F3377B
:10FE1000820F911D90930F1C80930E1C2C893D899D
:10FE20002817390710F0892B21F430930F1C2093E9
:10FE30000E1C80910E1C90910F1C9B8B8A8B8091C5
:10FE4000C038837009F455C110925C3910925B3947
:10FE50000E94BB758091C03885FF07C010925C3945
:10FE600010925B39198E84E1ABC084FF0AC01092F6
:10FE70005C3910925B3981E090E0998B888B84E04B
:10FE80008CCF20915B3930915C3921153105E1F03F
:10FE900080FF02C0198A188A88899989009781F49D
:10FEA0008A899B898217930720F490935C39809309
:10FEB0005B3980915B3990915C39998B888B04C058
:10FEC00090935C3980935B391B8E8091CA379091F7
:10FED000CB379093C4388093C33880915B3990912D
:10FEE0005C39892B59F088899989009739F088966F
:10FEF0009093C9378093C83788E10BC08091C03890
:10FF000081FFF7C088E290E09093C9378093C837AB
:10FF100080E18093F1375CC08091C03880FFE9C0F8
:10FF2000198E80E18093C0380E94BB75E2C0809139
:10FF3000C8379091C937009711F00E9403799091CA
:10FF4000F1378091C03890FF0BC080FF06C087E07A
:10FF5000898F1A8E198A188A19C086E0898F16C06F
:10FF600080FF1EC085E0898F198A188AC2C08091DF
:10FF7000C8379091C937009711F00E94037980919A
:10FF8000F13780FF0DC087E0898F1A8E81E090E005
:10FF90000E94037980E18093C0380E94BB750FC036
:10FFA0008091C8379091C937892B49F4A2C08091BC
:10FFB000C03880FF9EC087E0898F1A8E9AC080E18A
:10FFC0008093F13788E290E09093C9378093C837E7
:10FFD00080E58093F03788858093EC37898580931E
:10FFE000ED378A858093EE378B858093EF378C854C
:10FFF0008093E8378D858093E9378E858093EA3743
:020000021000EC
:100000008F858093EB3786E08093D9378C819D81F3
:100010009093E5378093E4378E819F819093E73703
:100020008093E6378091573990915839A09159398A
:10003000B0915A398093DC379093DD37A093DE3747
:10004000B093DF3788819981AA81BB818093E037A3
:100050009093E137A093E237B093E337898D84FF23
:1000600005C01092F3371092F23705C01092F237A4
:1000700088EC8093F33780E48093D8378091C83739
:100080009091C9379093D2378093D3371092F73736
:100090001092F6371092F5371092F4370E943179AA
:1000A000809590959093F5378093F43785E480930D
:1000B000D0371092D1371092D7371092D63780911F
:1000C000181C9091191C01969093191C8093181C70
:1000D0009093D4378093D5371092DB371092DA376C
:1000E0000E942079809590959093DB378093DA3742
:1000F00004C01092C9371092C8371092C038DF91EF
:10010000CF911F910F91FF90EF90DF90CF90BF9014
:10011000AF9008958CE19CE10C94A76F90931B1C09
:1001200080931A1C08958CE19CE10C94AB6FEF92C4
:10013000FF920F931F93CF93DF938C01EB017A0112
:100140008CE19CE10E94AB6F0097D9F0DC01129624
:100150002D913C9113972C173D0781F41696ED9144
:10016000FC911797309769F09701AE01B801DF91C4
:10017000CF911F910F91FF90EF9019940E940C70F6
:10018000E3CFDF91CF911F910F91FF90EF900895F2
:1001900008950F931F93CF93DF93CDE5DCE1488162
:1001A00059816A817B8100E010E023EF30E88DE324
:1001B0009CE10E94E06B0E944365BC0180E090E0FE
:1001C000288139814A815B810E94E686AB01BC01AE
:1001D00028E131E889E29CE10E94E06BDF91CF9158
:1001E0001F910F91089580915D1C90915E1CA091CC
:1001F0005F1CB091601C4091591C50915A1C609139
:100200005B1C70915C1C880F991FAA1FBB1F4817AD
:1002100059076A077B0710F4DB01CA0180935D1C54
:1002200090935E1CA0935F1CB093601C0C94C980DB
:10023000CF93DF930E94C8730E943773EC01198239
:1002400018820E94938028813981009719F1FC015E
:1002500040854423F9F0FC0142815381F901EE0FFE
:10026000FF1FEE0FFF1FEC0FFD1F53834283FC01A6
:10027000448155812F5F3F4FF901EE0FFF1FEE0FB5
:10028000FF1FEC0FFD1F51834083398328830E9499
:100290000C70D9CFC901880F991F880F991F02963A
:1002A0000E94327388819981892B31F08EE19CE123
:1002B000DF91CF910C94EE71DF91CF910895AF92C1
:1002C000BF92CF92DF92EF92FF920F931F93CF9343
:1002D000DF931F921F92CDB7DEB75B010E94377389
:1002E0008C01FC01E080F180FA82E9820E947F7338
:1002F0009701220F331F220F331F2E5F3F4F8217AC
:10030000930798F0C12CD12CCE14DF0471F0F801C2
:100310004481558162817381C5010E949780FFEFFE
:10032000CF1ADF0A0C5F1F4FEFCF0F900F90DF91B6
:10033000CF911F910F91FF90EF90DF90CF90BF90E2
:10034000AF9008950F93013099F48091511C9091D2
:10035000521CA091531CB091541C80935D1C90932F
:100360005E1CA0935F1CB093601C0F910C94C9801D
:100370000F9108954F925F926F927F928F929F920A
:10038000AF92BF92CF92DF92EF92FF920F931F93A3
:100390002A013B01480159014DE15AE0BC018EE1BF
:1003A0009CE10E94D171EEE1FCE143AA54AA65AA46
:1003B00076AA87AA90AEA1AEB2AEC3AED4AEE5AE79
:1003C000F6AE82EA91E81F910F91FF90EF90DF90D7
:1003D000CF90BF90AF909F908F907F906F905F90E5
:1003E0004F900C948E800C94FB71CF93DF93E0912F
:1003F000210AF091220A1995EC01892B29F06A81D2
:100400007B8181E00E941C74CE01DF91CF91089521
:100410000F931F93CF93DF93EC01E091230AF091A8
:10042000240A19958C016A817B8181E00E941C74E9
:1004300081E090E0012B11F480E090E0DF91CF911A
:100440001F910F910895E091250AF091260A1994C1
:10045000CF93DF93FC01DB0185E0EB0119928A95D4
:10046000E9F78581837011F082E08C938781837036
:1004700021F082E012968C9312978581837081F02F
:100480008781837069F02389348981859285281753
:10049000390731F481E0848312961C92129701C0CF
:1004A000148285818370823029F0833011F488E0D2
:1004B00001C080E011968C93119787818370823000
:1004C00029F0833011F488E001C080E013968C930A
:1004D000DF91CF910895CF93DF9300D01F921F92A9
:1004E000CDB7DEB7BE016F5F7F4F0E942882898142
:1004F00090E003962A81820F911D2B81820F911D1E
:100500002C81820F911D2D81820F911D0F900F90D4
:100510000F900F900F90DF91CF9108953F924F92DF
:100520005F926F927F928F929F92AF92BF92CF9283
:10053000DF92EF92FF920F931F93CF93DF9300D040
:100540001F921F92CDB7DEB78C017B013A01BE012D
:100550006F5F7F4F0E94288269817A81472F50E028
:10056000EB813C80232D30E0862F90E00396840FB2
:10057000951F8E0F911D820F931FAD818A0F911DC4
:10058000681679060CF4A4C0D80111968C911197C5
:1005900080FB882480F8912C83E0880C991C8A9534
:1005A000E1F712968C91129780FBAA24A0F8B12C47
:1005B00094E0AA0CBB1C9A95E1F78A288C9187706D
:1005C000882A13968C91139780FBCC24C0F8D12CE9
:1005D000F5E0CC0CDD1CFA95E1F7C82814968C9157
:1005E00080FB442440F8512CA6E0440C551CAA95ED
:1005F000E1F74C28D7014C92D80115968C91837065
:10060000B4E08B9F60011124D80116969C919370E1
:10061000B0E19B9FC00111248C29D8011796FC9151
:1006200090E4F99FD00111248A2BD70111968C9365
:10063000D80118968C91D70112968C93623071F480
:10064000D80119968C91D70113968C93D8011A96DC
:100650008C91D70114968C9385E001C083E0780FCC
:10066000872F972F941B4115510561F04150510977
:10067000D801A40FB51F1B968C91D701A90FB11DEE
:100680008C93EECFE23071F4D701A70FB11DF801C2
:1006900093899C9391E0970FD701A90FB11D8E5FAD
:1006A00094899C93F32DF80F8F2F821B2115310510
:1006B00061F021503109D801A20FB31F55969C91CA
:1006C000D701A80FB11D9C93EFCF8F2F90E002C0F0
:1006D00080E090E00F900F900F900F900F90DF91BF
:1006E000CF911F910F91FF90EF90DF90CF90BF902F
:1006F000AF909F908F907F906F905F904F903F90C2
:100700000895AF92BF92CF92DF92EF92FF920F9334
:100710001F93CF93DF93633071050CF4B3C0EA01EC
:100720006B017C01FC01908196FBAA24A0F88181D9
:10073000282F269526952370B82EB294B694B69499
:1007400053E0B522392F3770388393FB332730F9C4
:10075000398394FB332730F93A8395FB992790F935
:100760009B83AC822D83829583708E83BF8282812E
:100770008887222379F13381848190E0982F88271C
:10078000830F911D9A87898787010B5F1F4F223046
:1007900071F46BEE79E0CE010B960E94E972F701DD
:1007A00086818B8785818C870E5F1F4F1EC023300B
:1007B000E1F4F7013D96DE011B969E012D5E3F4F51
:1007C0009E2F8F2F42914D93A217B307D9F7092F70
:1007D000182F0BC087010D5F1F4F6BEE79E0CE0124
:1007E0000B960E94E9721A861986BB20A1F1A1100E
:1007F0000DC0F8012081818190E0982F8827820F19
:10080000911D9C8B8B8B0E5F1F4F04C089859A8531
:100810009C8B8B8BF2E0BF120EC06BEE79E0CE01A9
:1008200045960E94E972F80181818D8B80818E8BC3
:100830000E5F1F4F18C0F3E0BF1215C0085F1F4FB7
:10084000D801FE017596CE014D962E912193E817A1
:10085000F907D9F708C06BEE79E0CE0145960E9402
:10086000E9721C8A1B8A98012E193F09C601821B56
:10087000930B98AB8FA71EA70DA7C216D30614F033
:10088000C90102C080E090E0DF91CF911F910F91EC
:10089000FF90EF90DF90CF90BF90AF90089520E051
:1008A00030E00296FC0132974081442331F0FC0194
:1008B00031974081240F311DF4CFC9010895FC0107
:1008C000208130E0322F22278181282B02C0220F85
:1008D000331F6A95E2F7232F3327FA01E95DF54FBD
:1008E000808190E08223932328E030E0241B350BA5
:1008F00002C0969587952A95E2F708956F927F92A8
:100900008F929F92AF92BF92CF92DF92EF92FF921F
:100910000F931F93CF93DF937C018B015A01E90161
:100920002830310544F4A901B501C8010E945F8453
:10093000F701808346C0690183E0D594C7948A9506
:10094000E1F7452B21F04701612C712C06C0FB011A
:10095000D701CB018C0D9D1D1FC048E050E0B501B3
:10096000C801860D971D0E945F84F40181934F0199
:10097000FFEF6F1A7F0A6C147D0479F7AE014770A0
:10098000552741155105E9F0E701C60DD71DB50101
:10099000C801860D971D12C0E817F90719F02191BB
:1009A0002D93FACFAE01477055274115510549F0F7
:1009B000E701CC0DDD1D60E070E0CF010E945F8497
:1009C0008883DF91CF911F910F91FF90EF90DF907F
:1009D000CF90BF90AF909F908F907F906F90089531
:1009E0008F929F92AF92BF92CF92DF92EF92FF923F
:1009F0000F931F93CF93DF931F921F92CDB7DEB754
:100A00000E9437738C0182E090E00E941573892B5D
:100A100019F480E090E05FC0F801218130E0322FCE
:100A200022278081A901480F511DCA010E940C7222
:100A30007C01892B71F30E9437734C01F701968179
:100A4000292F26952695269530E0977041E050E0B5
:100A500011F440E050E0C901840F951F0E94157306
:100A6000892BB9F2F70104811581A12CB12CF80171
:100A70008081882379F1F801C180D12CA5014770CC
:100A80005527B50193E0759567959A95E1F7680D3F
:100A9000791D883168F09601CE0101960E947E840E
:100AA000BE016F5F7F4FF80180810E9430740DC0DE
:100AB0001A8219829601CE0101960E947E84698174
:100AC0007A81F80180810E941C74AC0CBD1C0E5F01
:100AD0001F4FCDCFC7010F900F90DF91CF911F9186
:100AE0000F91FF90EF90DF90CF90BF90AF909F90CD
:100AF0008F900895DC0150E0E0E1F0E0CF01861B2B
:100B0000970B821B930B02C0440F551F8A95E2F787
:100B10008C91852B8C9311968C911197482B119663
:100B20004C9308956F927F928F929F92AF92BF9253
:100B3000CF92DF92EF92FF920F931F93CF93DF93A9
:100B4000283031051CF4FA0140815AC05901E3E014
:100B5000B594A794EA95E1F76115710541F0390163
:100B6000EA018B017C014A01C12CD12C05C0EA01AC
:100B7000FC014A0D5B1D2AC0F40141914F0128E0A0
:100B800030E0B801C7018C0D9D1D0E947A85FFEFF2
:100B9000CF1ADF0ACA14DB0479F7930127703327D1
:100BA00021153105E9F1CC0DDD1D488150E0021B16
:100BB000130B085F1F4F02C0559547950A95E2F742
:100BC00060E070E0C7018C0D9D1D1AC0C417D507E9
:100BD00019F069916193FACF2770332721153105F8
:100BE000F9F0488150E068E070E0621B730B02C0CE
:100BF000559547956A95E2F760E070E08A0D9B1D78
:100C0000DF91CF911F910F91FF90EF90DF90CF90E8
:100C1000BF90AF909F908F907F906F900C947A854B
:100C2000DF91CF911F910F91FF90EF90DF90CF90C8
:100C3000BF90AF909F908F907F906F9008956F922C
:100C40007F928F929F92AF92BF92CF92DF92EF925C
:100C5000FF920F931F93CF93DF931F921F92CDB7F5
:100C6000DEB77C01FC018681082F06950695069566
:100C7000202F30E0877001E010E011F400E010E078
:100C8000020F131FC80102960E949173009709F486
:100C900048C00E943E73F7012281FC012083F701C6
:100CA0002381FC0121830E943E7302965C01A8010E
:100CB00060E070E00E947191F701048115810F5F7F
:100CC0001F4F812C912CF80131978081882339F1B5
:100CD000F801C080D12C3401F7E06F227724740131
:100CE00093E0F594E7949A95E1F7EA0CFB1C8831C0
:100CF00028F00E943A749601AC0108C00E94277443
:100D00009A8389839601AE014F5F5F4FB301C7019C
:100D10000E9492858C0C9D1C0E5F1F4FD4CF81E0EA
:100D200090E00F900F90DF91CF911F910F91FF9066
:100D3000EF90DF90CF90BF90AF909F908F907F907B
:100D40006F900895DB018F939F930E944D87BF9111
:100D5000AF91A29F800D911DA39F900DB29F900D0A
:100D600011240895991B79E004C0991F961708F083
:100D7000961B881F7A95C9F780950895AA1BBB1BFF
:100D800051E107C0AA1FBB1FA617B70710F0A61B8B
:100D9000B70B881F991F5A95A9F780959095BC01AC
:100DA000CD01089597FB072E16F4009407D077FD28
:100DB00009D00E94BE8607FC05D03EF4909581952F
:100DC0009F4F0895709561957F4F0895A1E21A2E67
:100DD000AA1BBB1BFD010DC0AA1FBB1FEE1FFF1FDF
:100DE000A217B307E407F50720F0A21BB30BE40B2F
:100DF000F50B661F771F881F991F1A9469F7609576
:100E00007095809590959B01AC01BD01CF0108952F
:100E1000052E97FB1EF400940E941F8757FD07D0F4
:100E20000E94E68607FC03D04EF40C941F87509571
:100E30004095309521953F4F4F4F5F4F08959095C6
:100E40008095709561957F4F8F4F9F4F0895EE0F5E
:100E5000FF1F881F8BBF0790F691E02D19940E9409
:100E60003787332312F48A1B9B0B0C944887A29F6D
:100E7000B001B39FC001A39F700D811D1124911D6E
:100E8000B29F700D811D1124911D08950E94378716
:100E9000B7FF0895821B930B08950E943787A59F83
:100EA000900DB49F900DA49F800D911D1124089565
:100EB000B7FF0C944D870E944D87821B930B0895BA
:100EC000DF93CF931F930F939A9DF02D219FF00DE9
:100ED0008B9DF00D8A9DE02DF10D039FF00D029F7B
:100EE000E00DF11D4E9DE00DF11D5E9DF00D4F9D3D
:100EF000F00D7F936F93BF92AF925F934F93D501A5
:100F00000E9437878B01AC01D7010E943787EB0124
:100F1000E80FF91FD6010E94B0872F913F91D601AB
:100F20000E943787C60FD71FE81FF91FAF91BF91E7
:100F30000E94B0872F913F910E943787C60FD71F1D
:100F4000E81FF91FD6010E943787E60FF71F9801A7
:100F5000BE01CF0111240F911F91CF91DF91089510
:100F60000E943787460F571FC81FD91F08F43196B4
:100F70000895E894DF93CF93FC01DB010E9437874B
:100F80007F936F93E9019A01AC01BF93AF933F93B5
:100F90002F93DF010E94378726F46C1B7D0B820B99
:100FA000930B9E01EB01FC010E94B087AF91BF91B2
:100FB0002F913F910E94B087BE01CF01F9012F917F
:100FC0003F91CF91DF910895689401C0E894F92F83
:100FD000F12B12F00C941888A0E0B0E0E2EFF7E8F3
:100FE0000C948A88092E059422F40E947488112397
:100FF00092F4F0E80F26FFEFE094F094009510953E
:10100000B094C094D094A194BF0ACF0ADF0AEF0A2B
:10101000FF0A0F0B1F0B0E94238807FC0E94748895
:10102000CDB7DEB7ECE00C94A688689401C0E894D4
:101030008F929F92CF93DF930E942388DF91CF916D
:101040009F908F90089588249924F401E401B0E4DE
:101050009F93AA279A158B049C04ED05FE05CF05E6
:10106000D007A10798F4AD2FDC2FCF2FFE2FE92D4D
:10107000982C892E982F872F762F652F542F432F4A
:10108000322F2227B85031F7BF9127C01B2EBF91B6
:10109000BB27220F331F441F551F661F771F881F52
:1010A000991F881C991CEE1FFF1FCC1FDD1FAA1F54
:1010B000BB1F8A149B04EC05FD05CE05DF05A007C8
:1010C000B10748F08A189B08EC09FD09CE09DF0931
:1010D000A00BB10B21601A94E1F62EF49401AF013C
:1010E000BE01CD01000C0895609570958095909596
:1010F00030954095509521953F4F4F4F5F4F6F4F23
:101100007F4F8F4F9F4F08952F923F924F925F9244
:101110006F927F928F929F92AF92BF92CF92DF9207
:10112000EF92FF920F931F93CF93DF93CDB7DEB76C
:10113000CA1BDB0B0FB6F894DEBF0FBECDBF1994F0
:101140002A88398848885F846E847D848C849B8457
:10115000AA84B984C884DF80EE80FD800C811B8165
:10116000AA81B981CE0FD11D0FB6F894DEBF0FBE94
:10117000CDBFED0108950F93083090F0982F872F81
:10118000762F652F542F432F322F22270850F4CF6C
:10119000220F331F441F551F661F771F881F991F7B
:1011A0000A95B2F70F91089597FB10F8169400086E
:1011B0000F93083098F00850232F342F452F562FC7
:1011C000672F782F892F902DF4CF059497958795C9
:1011D0007795679557954795379527950A95AAF777
:1011E0000F9108952A0D3B1D4C1D5D1D6E1D7F1D29
:1011F000801F911F08950024A7FD00942A0F301D21
:10120000401D501D601D701D801D901D08952A19E0
:101210003B094C095D096E097F09800B910B08950C
:101220002A153B054C055D056E057F058007910776
:1012300008950024A7FD00942A17300540055005A5
:10124000600570058005900508955058BB27AA27B2
:101250000E943D890C94A88B0E949A8B38F00E94C2
:10126000A18B20F039F49F3F19F426F40C94608B85
:101270000EF4E095E7FB0C945A8BE92F0E94B98B92
:1012800058F3BA17620773078407950720F079F4BB
:10129000A6F50C94DB8B0EF4E0950B2EBA2FA02D47
:1012A0000B01B90190010C01CA01A0011124FF2713
:1012B000591B99F0593F50F4503E68F11A16F0400E
:1012C000A22F232F342F4427585FF3CF469537950D
:1012D0002795A795F0405395C9F77EF41F16BA0BD2
:1012E000620B730B840BBAF09150A1F0FF0FBB1F80
:1012F000661F771F881FC2F70EC0BA0F621F731FC9
:10130000841F48F4879577956795B795F7959E3F25
:1013100008F0B0CF9395880F08F09927EE0F9795B6
:10132000879508950E949A8B60F080E891E009F417
:101330009EEF0E94A18B28F040E851E071F45EEF2F
:101340000CC00C94608B0C94DB8BE92FE0780E942E
:10135000B98B40F3092E052AB1F326173707480742
:10136000590738F00E2E07F8E02569F0E025E06413
:101370000AC0EF6307F8009407FADB01B9019D0189
:10138000DC01CA01AD01EF930E94208A0E94A88B64
:101390000E94D5895F91552339F02BED3FE049E458
:1013A00050FD49EC0C9426890895DF93DD27B92F71
:1013B000BF7740E85FE31616170648075B0718F487
:1013C000D92F0E94E78B9F938F937F936F930E94F7
:1013D000728DE4E4F1E00E94738B0E94A88B2F9140
:1013E0003F914F915F910E94C88CDD2351F090583E
:1013F000A2EA2AED3FE049EC5FE3D0785D270E9446
:101400003D89DF910C94A88B0E94368B08F481E013
:1014100008950E941D8A0C94A88B0E94A18B58F0FD
:101420000E949A8B40F029F45F3F29F00C945A8B6C
:1014300051110C94DC8B0C94608B0E94B98B68F377
:101440009923B1F3552391F3951B550BBB27AA277D
:1014500062177307840738F09F5F5F4F220F331FB7
:10146000441FAA1FA9F335D00E2E3AF0E0E832D07F
:1014700091505040E695001CCAF72BD0FE2F29D082
:10148000660F771F881FBB1F261737074807AB0754
:10149000B0E809F0BB0B802DBF01FF2793585F4FC9
:1014A0003AF09E3F510578F00C945A8B0C94DC8BEB
:1014B0005F3FE4F3983ED4F3869577956795B795AB
:1014C000F7959F5FC9F7880F911D9695879597F9B6
:1014D0000895E1E0660F771F881FBB1F621773072F
:1014E0008407BA0720F0621B730B840BBA0BEE1F44
:1014F00088F7E095089529F416F00C945A8B0C9413
:10150000DB8B0C94608B0E94C18BA8F39638A0F7FC
:1015100007F80F92E8942BE33AEA48EB5FE70E9462
:10152000CB8C0F920F920F924DB75EB70F920E9425
:10153000818CE1E7F1E00E94738B4F915F91EF9115
:10154000FF91E595EE1FFF1F49F0FE57E068442725
:10155000EE0F441FFA95E1F74195550B0E94F38B6E
:101560000F9007FE0C94E78B089597FB16F40E94EA
:10157000638B0C94F98AE89409C097FB3EF490952C
:101580008095709561957F4F8F4F9F4F9923A9F05C
:10159000F92F96E9BB279395F695879577956795EB
:1015A000B795F111F8CFFAF4BB0F11F460FF1BC02F
:1015B0006F5F7F4F8F4F9F4F16C0882311F096E9C2
:1015C00011C0772321F09EE8872F762F05C0662370
:1015D00071F096E8862F70E060E02AF09A95660F29
:1015E000771F881FDAF7880F9695879597F90895E2
:1015F000E894F92F96EBFF2381F0121613061406D8
:10160000440B9395F6958795779567955795404048
:10161000FF23B9F71BC099270895882351F49850E8
:10162000D2F7872B762F652F542F432F322F20E0B0
:10163000B1F3121613061406440B88233AF09A9558
:10164000440F551F661F771F881FCAF755234AF49A
:10165000440F551F11F460FF04C06F5F7F4F8F4F21
:101660009F4F880F9695879597F90895990F0008D1
:10167000550FAA0BE0E8FEEF16161706E807F90764
:10168000C0F012161306E407F50798F0621B730BFF
:10169000840B950B39F40A2661F0232B242B252B80
:1016A00021F408950A2609F4A140A6958FEF811D23
:1016B000811D089597F99F6780E870E060E00895C4
:1016C0009FEF80EC0895909580957095609550956A
:1016D0004095309521953F4F4F4F5F4F6F4F7F4F54
:1016E0008F4F9F4F0895DF93CF931F930F93FF92D8
:1016F000EF92DF927B018C01689406C0DA2EEF0135
:101700000E94C88CFE01E894A591259135914591E0
:101710005591A6F3EF010E943D89FE019701A801B2
:10172000DA9469F7DF90EF90FF900F911F91CF91BE
:10173000DF91089500240A94161617061806090664
:10174000089500240A941216130614060506089537
:10175000092E0394000C11F4882352F0BB0F40F4BF
:10176000BF2B11F460FF04C06F5F7F4F8F4F9F4FFF
:10177000089557FD9058440F551F59F05F3F71F081
:101780004795880F97FB991F61F09F3F79F08795E8
:101790000895121613061406551FF2CF4695F1DF71
:1017A00008C0161617061806991FF1CF8695710501
:1017B000610508940895E894BB2766277727CB0135
:1017C00097F908950E94368B08F48FEF08959B01D6
:1017D000AC0160E070E080E89FE30C94098A0C940F
:1017E0005A8B0C94768D0E94C18BD8F39923C9F340
:1017F000940F511DA3F39150504094F059F0882359
:1018000032F0660F771F881F91505040C1F79E3FFE
:1018100051052CF7880F911D9695879597F9089596
:101820005F3FACF0983E9CF0BB2786957795679517
:10183000B79508F4B1609395C1F7BB0F58F711F451
:1018400060FFE8CF6F5F7F4F8F4F9F4FE3CF0C94C8
:10185000DC8B0E94398C29ED3BE54EED5EE30C9468
:10186000B58C16F00C94768D0C94608B68940C9467
:101870005A8B0E94C18BA8F39923C1F3AEF3DF9377
:10188000CF931F930F93FF92C92FDD2788232AF050
:101890002197660F771F881FDAF720E030E040E8D5
:1018A0005FEB9FE3883920F0803E38F021968F77F8
:1018B0000E942689E9E9F1E004C00E942689E6EC4D
:1018C000F1E00E94738B8B01BE01EC01FB2E6F5780
:1018D00071097595771F880B990B0E94BD8A28E1C5
:1018E00032E741E35FE30E94C88CAF2D9801AE015F
:1018F000FF900F911F91CF91DF910E943D890C9431
:10190000A88BFA01DC01AA0FBB1F9B01AC01BF57DA
:1019100028F4222733274427507820C0B75190F469
:10192000AB2F0024469537952795011CA395D2F33C
:10193000002071F0220F331F441FB395DAF30ED04D
:101940000C94258961307105A0E88A07B94630F406
:101950009B01AC016627772788279078309621F085
:10196000208331834283538308950E94C88C0C9452
:10197000A88B0E949A8B38F00E94A18B20F09523AF
:1019800011F00C945A8B0C94608B11240C94DC8B0A
:101990000E94B98B70F3959FC1F3950F50E0551FCE
:1019A000629FF001729FBB27F00DB11D639FAA27B4
:1019B000F00DB11DAA1F649F6627B00DA11D661F03
:1019C000829F2227B00DA11D621F739FB00DA11D24
:1019D000621F839FA00D611D221F749F3327A00DDE
:1019E000611D231F849F600D211D822F762F6A2F7A
:1019F00011249F5750409AF0F1F088234AF0EE0FDF
:101A0000FF1FBB1F661F771F881F91505040A9F70B
:101A10009E3F510580F00C945A8B0C94DC8B5F3FF9
:101A2000E4F3983ED4F3869577956795B795F79547
:101A3000E7959F5FC1F7FE2B880F911D96958795BF
:101A400097F90895FA01EE0FFF1F30962105310531
:101A5000A1F16115710561F48038BFE39B0749F17D
:101A600068949038810561F08038BFEF9B0741F0A2
:101A700099234AF5FF3FE1053105210519F1E89465
:101A80000894E795D901AA2329F4AB2FBE2FF85F5C
:101A9000D0F310C0FF5F70F4A695E0F7F73950F06F
:101AA00019F0FF3A38F49F779F930DD00F9007FC01
:101AB0009058089546F00C94608B60E070E080E8E8
:101AC0009FE308954FE79F775F934F933F932F9343
:101AD0000E94398C2F913F914F915F910E94B58C5C
:101AE0000C94838A9B01AC010C94B58C9F3F31F020
:101AF000915020F4879577956795B795880F911D3C
:101B00009695879597F908958F929F92AF92BF927D
:101B1000CF92DF92EF92FF92CF93DF93EC01688137
:101B200079818A819B81611571058105910521F477
:101B300064E279ED8BE597E02DE133EF41E050E091
:101B40000E94088749015A019B01AC01A7EAB1E450
:101B50000E944D876B017C01ACEEB4EFA5019401AE
:101B60000E945B87DC01CB018C0D9D1DAE1DBF1D4E
:101B7000B7FF03C00197A109B04888839983AA835E
:101B8000BB839F77DF91CF91FF90EF90DF90CF9055
:101B9000BF90AF909F908F9008950C94848D80E0BB
:101BA00092E00C94848DA0E0B0E0809300029093CA
:101BB0000102A0930202B093030208952F923F9274
:101BC0004F925F926F927F928F929F92AF92BF924D
:101BD000CF92DF92EF92FF920F931F93CF93DF93F9
:101BE0005C016B017A016115710519F0FB019183AC
:101BF0008083E114F10429F0C7010297839708F06C
:101C0000F1C0E5012196F5011081812F90E00E943D
